:020000040800F2
:20000000F0FF0120C1B5060845F50008D1CF040839B6060839B6060839B606080000000067
:2000200000000000000000000000000041F500083DF500080000000039F50008C10605083E
:2000400039B6060839B6060839B6060839B6060839B6060839B606087917050841170508B0
:2000600009170508D116050899160508F9700608E9700608D9700608C9700608B5700608F4
:20008000A17006088D70060839B606080000000000000000000000000000000061160508B5
:2000A000EDD404083DD50408DDD4040865D504082DD504081DD504080DD50408B5AD0608E8
:2000C000BDAD0608A9AD0608B1AD060839B6060839B6060895080508DD0705080000000043
:2000E0002916050839B60608FD0D01080000000000000000000000000000000079700608AD
:2001000000000000E54C0608FDD4040839B6060800000000000000000000000000000000C6
:2001200065700608517006083D700608297006081570060800000000000000000000000018
:20014000000000000000000000000000D9EE000801700608ED6F0608D96F06082507050858
:200160009DAD0608A5AD0608000000000000000000000000000000000000000000000000C7
:200180000000000039B60608000000000000000039B6060839B6060860B106000100000050
:2001A0000E02010002000000D07400203475002000000000C0F10708307500201402010063
:2001C00005000000F03900203C75002000000000C2F1070838750020130201000400000057
:2001E000D82B00204875002000000000C8F1070844750020031101000A0000001874002093
:200200005075002000000000491A01084C7500200D1001004C000000B06F0020607500200E
:2002200000000000DD4C04085C7500200902010001000000186F0020B0750020000000009F
:20024000CCF10708AC750020FD01010024000000D06E0020B875002000000000DBDF0408FD
:20026000B4750020FB01010001000000E0690020E07500200000000009590508DC75002079
:20028000FC01010009000000AC680020E87500200000000011590508E4750020F7010100BD
:2002A00006000000A0680020F875002000000000CEF10708F4750020F9010100040000002D
:2002C0009C680020047600200000000085E0040800760020160215003F0000008C2D002014
:2002E0000C7600200000000029590508087600203400010010000000CC67002050760020B1
:2003000000000000219C02084C7600201102010008000000A46700206476002000000000F3
:20032000D4F107086076002012120100040000009C6700207076002000000000DCF10708C5
:200340006C7600201830010038000000646700207876002000000000C163050874760020E6
:20036000000201000B000000E8630020B4760020000000004D590508B0760020FF210100A0
:200380000500000094630020C476002000000000E9580508C0760020081203000F00000017
:2003A000A0630020D07600200000000075590508CC760020FA01010003000000005D0020FB
:2003C000E4760020000000006D590508E07600202A020100080000000C520020EC76002025
:2003E00000000000E0F10708E8760020205201000800000068500020F876002000000000BE
:20040000459C0208F47600200610010024000000A82C00200477002000000000F159050846
:20042000007700200C02010004000000F84800202C77002000000000F958050828770020D2
:20044000FE01010014000000203B0020347700200000000055590508307700202610010089
:200460000E00000018E6002008E6002000000000251F010804E600200B3001001A00000095
:20048000B0DC00205CE6002000000000E8F1070858E600201F50010024000000DCDB00209D
:2004A0007CE600200000000004F2070878E60020050201000400000098DE0020A4E60020EB
:2004C0000000000028F20708A0E60020010201000B000000A0EC002028F600200000000054
:2004E0003D59050824F60020020201000300000098EC002038F60020000000000000000025
:2005000034F600201B0201001000000084EC002040F6002000000000DD5905083CF60020E8
:200520001B2001000C000000B4E9002054F6002000000000CD83010850F600202102010069
:20054000F0000000E8E7002064F6002000000000D59B010860F600203710010030000000DB
:200560003CEF002058F70020000000002CF2070854F70020161001000600000040EC0020B0
:200580008CF70020000000005CF2070888F700202F1001002200000000F6002098F7002095
:2005A0000000000062F2070894F7002023220100100000007CEB0020C0F700200000000079
:2005C00084F20708BCF700201E0001000900000068EB0020D4F700200000000094F20708A8
:2005E000D0F70020052001000C00000014EC0020E4F7002000000000A0F20708E0F700202F
:20060000123001001000000050EB0020F4F7002000000000ACF20708F0F70020FD07010068
:200620007C000000ACE6002008F8002000000000517D010804F80020F59101006C00000086
:200640006CE7002088F80020000000007991010884F8002023200100100000009EEE0020D8
:20066000F8F8002000000000890D0208F4F80020F62101000C00000014160120AC1701206B
:2006800000000000BCF20708A81701201C0202001C000000A415012000180120000000006E
:2006A000615E0508FC1701202830010016000000C01501202018012000000000591B0208FE
:2006C0001C18012014000100050000009C1501203C18012000000000C8F20708381801202A
:2006E000012001000C000000F40E01204818012000000000CEF20708441801200C4006008A
:20070000E4000000140D0120581801200000000055E30308541801200A9001002400000093
:20072000D00C01204019012000000000410D02083C1901200E300300BC0100000C0B01203E
:2007400068190120000000005D9C02086419012013100100040000002C130120281B01206A
:2007600000000000DCF20708241B01200101010004000000500A0120301B0120000000004E
:20078000000000002C1B01200001010004000000480A0120381B012000000000E0F2070823
:2007A000341B01200201010003000000440A0120401B01200000000095E303083C1B0120DC
:2007C000220201001C01000014110120481B01200000000069600508441B01201500100092
:2007E00070000000E42701209029012000000000000000008C2901200300010001000000A8
:20080000DC270120042A01200000000000000000002A01202A00080060000000182201202D
:200820000C2A012000000000F99B0208082A01202C00040010000000802A0120702A0120AA
:2008400000000000E19502086C2A0120292014007800000054250120942A01200000000013
:2008600000000000902A01201A0001000E000000AC240120102B012000000000E4F2070842
:200880000C2B01202B0012002400000088240120242B012000000000B5950208202B0120A2
:2008A0001902010010000000782401204C2B0120000000002D590508482B012025201E002D
:2008C0002C010000D02F0120A43301200000000000000000A0330120031201003D0000008C
:2008E00068320120D434012000000000F2F20708D0340120F831010006000000702C01200F
:20090000183501200000000030F30708143501201010010002000000742F0120243501206C
:200920000000000036F30708203501201900010005000000EC2B01202C3501200000000030
:2009400038F3070828350120020001000C000000343E01204C3E0120000000000000000092
:20096000483E012029020100400000005C3701205C3E0120000000003EF30708583E0120FE
:200980002C02010004000000043E0120A03E0120000000007EF307089C3E01200A0201003A
:2009A00014000000A83C0120C83E01200000000021E30308C43E01201A0201003C0000006C
:2009C000E84301203049012000000000AD5D05082C49012038200100030000009441012032
:2009E000704901200000000082F307086C4901200400080080000000F04A0120704B012000
:200A00000000000000000000F04B01202802040004000000B0490120F84B012000000000CA
:200A2000D9590508F44B01202702040004000000AC490120004C012000000000CD59050830
:200A4000FC4B01201F020800100000009C490120084C012000000000C5580508044C0120DF
:200A60001D02020006000000B0540120DC5401200000000000000000D85401200612030071
:200A800012000000C05401206865012000000000E95E0508646501202700010004000000B7
:200AA000004E0120806501200000000086F307087C6501200B2201003D00000034880120EF
:200AC000BC8E0120000000008CF30708B88E01200D12010014000000988D0120008F01208C
:200AE00000000000CCF30708FC8E01201E02010006000000188C0120188F012000000000C9
:200B0000E0F30708148F0120100201000100000074A0012070A0012000000000E6F30708CD
:200B20006CA001200403090412010002EF0201408304563200020102030100001201000200
:200B400002020040830440570002010203010000FFFFFFFF0000000000000000010000002D
:200B60000000000000000000EC39002000000000010000000000000000000000000000002F
:200B8000000000000000000000000000000000000000000000000000000000000000000055
:200BA000000000000060024010600240000000000000000000000000000B000000000000D6
:200BC00000000000000000000060024028600240010000000000000000000000060C000096
:200BE00000000000000000000000000000600240406002400200000000000000000000006F
:200C0000100D00000000000000000000000000000060024058600240030000000000000018
:200C200000000000160E0000000000000000000000000000006002407060024004000000D8
:200C40000000000000000000200F0000000000000000000000000000006002408860024099
:200C6000050000000000000000000000261000000000000000000000000000000060024097
:200C8000A060024006000000000000000000000030110000000000000000000000000000CB
:200CA00000600240B8600240070000000000000000000000362F00000000000000000000CC
:200CC000000000000064024010640240000000000000000000000000003800000000000080
:200CE000000000000000000000640240286402400100000000000000000000000639000040
:200D0000000000000000000000000000006402404064024002000000000000000000000045
:200D2000103A000000000000000000000000000000640240586402400300000000000000C2
:200D400000000000163B000000000000000000000000000000640240706402400400000082
:200D60000000000000000000203C0000000000000000000000000000006402408864024043
:200D800005000000000000000000000026440000000000000000000000000000006402403E
:200DA000A06402400600000000000000000000003045000000000000000000000000000072
:200DC00000640240B86402400700000000000000000000003646000000000000000000008C
:200DE000000000007D0000001D8500081985000815850008098500080585000811850008BE
:200E00000D85000800000000B9910008F5A90008E98F000851AB000889920008A18500086B
:200E2000798500085D8500086DA3000889880008798A000875900008F1900008AD940008A7
:200E40008D8500086585000855850008010000000000803FE53E0108E9430108613F0108DA
:200E60004D130108311501085D13010879130108251301081513010800000000000000003A
:200E800009022000010104C03209040000020806500507058102400000070501024000009F
:200EA00009026400030100C03209040000010300000009211101000122360007058303098C
:200EC000000A080B0102020201000904010001020201000524001001052401000204240249
:200EE000020524060102070582030800FF09040200020A000000070501024000000705812F
:200F00000240000009024300020100C03209040000010202010005240010010524010001D4
:200F2000042402020524060001070582030800FF09040100020A0000000705010240000054
:200F40000705810240000000FF000000140000FF0000000000000000AA550701000001AAFE
:200F600055050100002D202D2D202D2D2D2D202D2D2D2D00000000000000000000000000C7
:200F8000000000000800000080DC0608FF1FFF1F05010905A101A100050109300931093298
:200FA000093309350934093609371581257F750895088102050919012908150025019508F3
:200FC00075018102C0C0000009022200010100E03209040000010301020009211101000106
:200FE0002236000705830309000A000000000000010203040102030406070809AA550B01B7
:201000000000AA5505010000AA550902000000AA5503009F01000000C0120000FFFFFFFF51
:2010200050E600200000000028E6002000000000010000000100000000000100E0017EFFCB
:20104000FFFFFFFFFF000000FFFFFFFF08FF0101FF0100000100000075020208000000000E
:20106000000000002CE30608000000000000000000000000D0FA060800000000000000007B
:201080000000000088FB060800000000000000000000000034FB0608000000000000000082
:2010A000E90D0208EA0F01200101000031230208000000000000000050FC0608912602089B
:2010C000000000000000000008FC06082D202D2D202D2D2D2D202D2D2D00000000000000DC
:2010E000000000000000000000000000FFFFFFFF21130208000000000000000060FA06084E
:2011000001000000FA00000001000000010000000101000000010101000000005A0E012044
:201120000000F40101000000580E01200000F40101000000560E01200000F40101000000C1
:20114000540E01200000F40101000000520E01200000F40101000000500E01200000F4012B
:20116000010000004E0E01200000F40101000000210B0208E50A020800000000F4E40608E6
:201180003E0E0120053201004C0E01206400F401010000004A0E01206400C409010000002A
:2011A0003C0E0120E803D007010000003A0E0120E803D00701000000380E0120E803D007AC
:2011C00001000000360E01201E00B80B01000000440E012005000F0001000000460E0120CA
:2011E00003000A0001000000340E01201E00F40101000000480E01200200000080E506087E
:20120000320E01201400640001000000400E01203200E80301000000300E01200000C80040
:2012200001000000110D012000C80100100D0120005001000F0D0120005A01000D0D012043
:2012400002000000E8E40608046807080C680708E80F01200100C40900000000E60F0120B8
:201260000100C40900000000E40F01200100C40900000000E20F01200100C40900000000DE
:20128000DE0F01200100C40900000000E00F01200100C40900000000DC0F01200100C409BA
:2012A00000000000DA0F01200100C409000000006F0A012000C801006E0A012000C8010091
:2012C0006C0A01200000FFFF0A0000006A0A01200100C80001000000680A012032003075A6
:2012E00032000000660A01207EFF140005000000640A012005002C0105000000630A012041
:20130000055A0500600A012000FF0100620A012002000000BC0800205E0A012003000000DF
:2013200038DE06085F0A012000FF0100610A012002000000BC0800205D0A01200300000002
:2013400038DE0608BC090120FF7F0100B809012000000000FFFFFFFF01000000B409012047
:2013600000000000FFFFFFFF01000000B009012000000000FFFFFFFF01000000750A020810
:20138000050A020800000000D0E50608040F0120EE02CA0801000000020F012000C801007F
:2013A00064000000010F012002C8010064000000000F0120020000008CE50608560A012037
:2013C0000000803E05000000540A012080C1803E050000004E0A01200083007D0500000049
:2013E0004C0A012080C1803E05000000470A012000FF0100400A01206400F401010000003B
:201400003E0A01206400F401010000003C0A01206400F401010000003A0A012004000000DF
:20142000DCE60608390A012002000000F0E60608FB0A01200D000000FCE60608F80A01204C
:2014400000640100F60A0120320010270A000000F40A01200D000000FCE60608F30A012059
:201460000D000000FCE60608F20A01200200000098E50608000000000000000000000000C5
:2014800034E70608090F0120460000006CE70608070F01200300000088E80608080F012053
:2014A00004000000A4E50608FD0A01200300000098E80608FC0A01200300000098E8060820
:2014C000FE0C0120000A0100FC0C01200000E80301000000FA0C01200000E80301000000AE
:2014E000F80C0120000A0100F60C01200000E80301000000F40C01200000E80301000000A0
:20150000C80C0120C800E80301000000CE0C01203C00FA0001000000CC0C01200100E8030B
:2015200001000000CA0C0120000501000C0D012002000000B8E506080A0D01200000F40199
:2015400001000000080D01200000F40101000000060D01200000F40101000000040D012002
:201560000000F40101000000020D01200000E80301000000000D01200000E803010000003F
:201580001E0E0120006401000A0000001D0E0120006401000A0000000B0E0120196401001C
:2015A0000A0E012002000000C4E50608080E0120E803D0070A000000060E0120006401009C
:2015C0000A000000FB0D012000640100FA0D012000640100020E0120006401000A00000046
:2015E000010E0120006401000A000000000E0120006401000A000000050E012000FF01007A
:201600000A000000040E012000FF01000A000000030E012000FF01000A000000FF0D01201A
:2016200001FF01000A000000FE0D012001FF01000A000000FD0D012001FF01000A00000032
:20164000060B01200000F40101000000040B01200000E80301000000020B01200000E8032D
:2016600001000000000B01200000E80301000000FE0A01200000E803010000003B100120D0
:20168000009601003210012000C80100311001200064010030100120006401002F1001209A
:2016A000006401002E100120006401002D100120FF0801002C10012001640100F5080208D1
:2016C000B908020800000000A8E806083510012001320100341001200100000018E9060892
:2016E000331001200400000020E906082B100120009601002A10012000640100281001205F
:201700001400E8030100000026100120000030750A0000002410012000C801002310012051
:2017200000C801002210012000C8010038100120003201003A10012000140100391001203E
:20174000004B0100371001200400000034E9060836100120006401000A0000002A0E012077
:201760000AC805000A000000290E01200100000044E906082C0E01200AC805000A000000B8
:201780002B0E01200100000044E90608210E012000C805000A000000280E012000C8050068
:2017A0000A000000220E012000C805000A000000230E012000C805000A000000260E012079
:2017C00000C805000A000000270E012000C805000A000000250E012000C805000A000000DA
:2017E000240E012000C805000A000000200E0120020000004CE906084A1001200000D007D9
:20180000010000004410012000C801004310012000C801004210012000C801004810012097
:201820000000D007010000004110012000C801004010012000C801003F10012000C8010022
:20184000461001200000D007010000003E10012000C801003D10012000C801003C1001205D
:2018600000C80100407907080000000000008C1701204C790708070800000000D00E002032
:2018800054790708070800000000C80E00205C790708070800000000C00E0020647907089A
:2018A000080800000000B40E002050630708070800000000AC0E00205863070807080000B2
:2018C0000000A40E0020606307080708000000009C0E00200C640708080800000000900E5E
:2018E00000206C790708071000000000880E002074790708071000000000800E00207C7951
:201900000708071000000000780E0020847907080810000000006C0E00206C67070801005A
:20192000000000000000000000000000100000000000000000000000890602086D06020881
:20194000FD12020858E90608EF0A0120005A0100EE0A012000C80100EC0A0120E803D007EF
:20196000010000000000000000000000290E0208F4E906085C0A01200300000048EA060870
:201980005B0A0120000301005A0A012000030100A90502085D0502080000000058EA0608C0
:2019A0001D050208D504020800000000F4EA0608F5050208E11202080000000074EB0608BE
:2019C000580A012001030100410202082102020800000000E8EE0608FD0B0208D10B020829
:2019E0000000000068EF060845040208ED03020800000000D8EF060899060208952E0208EA
:201A00000000000090F0060869180208290C02080000000038F10608E9060208000000003E
:201A200000000000D4F10608CD0702086D0702080000000038F20608750802083108020875
:201A400000000000F0F20608E574020831090208000000007CF306082E0E0120010601000D
:201A600031070208FD0602080000000094F4060801740208A91402080000000004F5060834
:201A800061090208C91502080000000080F60608297502088915020800000000D80E002010
:201AA0002D0E0120010301003D0602080D060208000000008CF7060881120208000000002D
:201AC00000000000F0F706089D040208C9120208000000008CF806080000000000000000EF
:201AE0000000000028F90608DD0902081517020800000000A8F906080000000000000000E2
:201B000000000000D0FB060870DC00209CFF2C0100000000C4120120E0150C1700000000A9
:201B2000C61201200200000008FF0608340A012088136F1701000000360A012088136F1792
:201B4000000000004C74002000000000000000004A740020000000000000000048740020EB
:201B60000000000000000000467400200000000000000000447400200000000000000000B3
:201B80004274002000000000000000008C0600200000000000000000BD09012003000000D3
:201BA000ECFC06082C0A012088136F17010000008EDE002088136F17000000002D030208CF
:201BC0000000000000000000FCFC0608A50F01200100000050FD060890DE0020010000003F
:201BE0005CFD060886DE00200200000064FD060800000000000000000000000070FD06080E
:201C00001503020800000000000000000CFE060800000000000000000000000060FE06081E
:201C2000000000000000000000000000D0FE0608380A01200200000008FF06088ADE0020C6
:201C4000E0150C1700000000D81D01202C1E012001F11F3FD601FF0048A70020FFFFFFFFBA
:201C60000000803F00000000000000000000000000000000000000000000000000000000A5
:201C800000000000000000000000803F0000000000000000000000000000803F00000000C6
:201CA00000000000000000000000803F000000000000000000000000010000000000FA4327
:201CC0000000FA430000803FFFFFFFFFFF000000A5AE0408000000000000000000000000AE
:201CE00000000000B43E01200800000000000000A43E012008000000254D04080000000040
:201D000000000000000000005DDE040800000000000000000000000001000000A00F0000CC
:201D2000B80B000002FFFF01685E0C00020000003D3E010841140108D53D0108000000000E
:201D400011130108BD460108253D0108713901080000000000000000D11201082D85000886
:201D600021850008758F0008918F0008598F00083D8F0008218F0008F53D01081D14010890
:201D8000293D010800000000E912010875390108F93C0108D13801080000000000000000C9
:201DA000DD1201087C9A0708AC640708000000001DE40308A0860100040000007C9A07088B
:201DC000849A0708000000003D890408E803000004000000186E0708000000000000000080
:201DE000E93A03087D000000FF0000001C6C0708000000000000000099BF03087D000000C2
:201E0000FF000000487107080000000000000000F55B03087D000000FF000000B06E0708F7
:201E20000000000000000000D9AE0408E8030000030000008C9A07080000000000000000EC
:201E4000A13E03081027000003000000F0DE07080000000025940208A5B804085F76000080
:201E600005000000A4E207080000000000000000D9DB04081027000002000000989A07088E
:201E80000000000000000000B14C0408E803000005000000A49A07080000000000000000FC
:201EA000F5EB0308204E000003000000B49A07080000000000000000DDE90308204E00002A
:201EC00003000000C49A0708000000000000000079B40408400D030003000000788B0708F4
:201EE000000000000000000021AC04081027000002000000D8640708000000000000000085
:201F00004DE701081027000003000000D49A070800000000000000001D840408A0860100F9
:201F200002000000C46C070800000000000000001987040850C30000020000006C6A0708BA
:201F40000000000000000000657F0408A861000002000000948B0708000000000000000058
:201F6000754D0408A00F000002000000DC9A0708000000000000000085D0010810270000C8
:201F800002000000647B070800000000057D0108D9C3010885450100020000002C6A0708AF
:201FA0000000000000000000811A01081027000002000000C0640708000000000000000011
:201FC0008937020850C3000002000000E89A070800000000000000007D260108400D030095
:201FE00001000000F09A070800000000000000006D4C0408400D030002000000F89A07088F
:020000040800F2
:20200000000000000000000031F7010850C3000003000000049B07080000000000000000CB
:20202000B505040840420F0001000000109B070800000000000000004D4D040850C30000D5
:20204000010000001C9B07080000000000000000D96901081027000002000000FFFF000037
:20206000FFFFFFFFCCDE0708000008020503030000000000D8DE07080100080205040300BA
:2020800000000000E4DE0708000008020503030000000000ECDE070801000802050403006A
:2020A00000000000C88A07080200FE010110030000000000606B07080300140200030000B4
:2020C00000000000F4DE070804001F020200080000000000FCDE070805001F0202010800D6
:2020E000000000001A030000000000000000000000000000000000000000000000000000C3
:20210000040309041201000200000040830420570002010203010100116A0508E56905086B
:2021200089690508995A0508A569050849690508955A050840190020056B05082561050841
:20214000F56A0508795A0508B16A0508696A0508695A05081C1900201D640508815A050890
:202160007D5A0508755A05086D640508715A05086D5A05084C53070859460108FD130108A6
:20218000394501080000000000000000D13C0108E13B01080000000000000000000000007D
:2021A000C5120108215B0508155B05085D6B0508796B0508CD5A0508416B0508256B0508E9
:2021C000020000000000000018190020D45401200200000001000000895C05081419002021
:2021E000000000000100000001000000C55C05083418002000000000000000000000000043
:202200000000000000000000000000000000000001000000000000000000000000000000BD
:2022200000000000010000000000000000000000000000000000000001000000000000009C
:20224000D8000000000000000500000006000000FFFFFFFF03000000000000000500000097
:20226000050000001F0000001C0000001F0000001E0000001F0000001E0000001F00000085
:202280001F0000001E0000001F0000001E0000001F0000000068214C0100000070530708FD
:2022A0000600000005000000008002021F00000053544D202020202050726F64757420201E
:2022C0002020202020202020302E3031008002021F00000053544D202020202050726F6473
:2022E000757420202020202020202020302E30310B0101010100000050C300000101FF01D2
:2023000025000000A057070800000000000000000000000001000000000000000000000091
:2023200000000000000000000100000000000000F40100002AFF0000A400000000000000DA
:2023400000000000000004010000020001000002100000000700000000000000000000005C
:202360000102030406070809C70000000500000006FF0000EC19002000000000000000003F
:2023800000000000000000000000000000000000000000000000000000000000000000003D
:2023A00000000000000000000000000000000000000000000000000000000000000000001D
:2023C000000000000000000000000000000000000000000000000000FFFFFFFFFFFFFFFF05
:2023E000FFFFFFFFFFFFFFFFFFFFFFFFFFFFFFFFFFFFFFFFFFFFFFFFFFFFFFFFFFFFFFFFFD
:20240000FFFFFFFFFFFFFFFFFFFFFFFFFFFFFFFFFFFFFFFFFFFFFFFFFFFFFFFFFFFFFFFFDC
:20242000FFFFFFFFFFFFFFFFFFFFFFFFFFFFFFFFFFFFFFFFFFFFFFFFFFFFFFFFFFFFFFFFBC
:20244000FFFFFFFFFFFFFFFFFFFFFFFFFFFFFFFFFFFFFFFFFFFFFFFFFFFFFFFFFFFFFFFF9C
:202800000828000800400008232042657461666C69676874202F2053544D33324634313157
:202820002028533431312920342E312E31204E6F762031352032303139202F2031323A3526
:20284000353A3137202831653565336433363929204D5350204150493A20312E34320A2371
:2028600020636F6E6669673A206D616E7566616374757265725F69643A20424546482C2074
:20288000626F6172645F6E616D653A2042455441465056463431312C2076657273696F6EA0
:2028A0003A2035373261316131392C20646174653A20323032332D30312D31365432333AA3
:2028C00035303A35315A0A0A236D63752053544D3332463431310A0A23646566696E652006
:2028E0005553455F4143435F5350495F4D5055363030300A23646566696E65205553455F5F
:202900004759524F5F5350495F4D5055363030300A23646566696E65205553455F41434349
:202920004759524F5F424D493237300A23646566696E65205553455F464C4153485F4D3236
:20294000355031360A23646566696E65205553455F4D4158373435360A0A626F6172645F50
:202960006E616D652042455441465056463431310A6D616E7566616374757265725F69646F
:2029800020424546480A0A23207265736F75726365730A7265736F75726365204245455022
:2029A00045522031204230320A7265736F75726365204D4F544F522031204230340A726550
:2029C000736F75726365204D4F544F522032204230350A7265736F75726365204D4F544FCB
:2029E000522033204230360A7265736F75726365204D4F544F522034204230370A726573D6
:202A00006F757263652050504D2031204130330A7265736F75726365204C45445F535452B7
:202A200049502031204130380A7265736F757263652053455249414C5F54582031204130A4
:202A4000390A7265736F757263652053455249414C5F54582032204130320A7265736F7593
:202A60007263652053455249414C5F5458203131204230330A7265736F75726365205345C0
:202A80005249414C5F5458203132204231300A7265736F757263652053455249414C5F52BA
:202AA000582031204131300A7265736F757263652053455249414C5F52582032204130333A
:202AC0000A7265736F757263652053455249414C5F5258203131204230330A7265736F751C
:202AE0007263652053455249414C5F5258203132204231300A7265736F7572636520493260
:202B0000435F53434C2031204230380A7265736F75726365204932435F53444120312042DC
:202B200030390A7265736F75726365204C45442031204331330A7265736F75726365204CCF
:202B400045442032204331340A7265736F75726365205350495F53434B2031204130350AF3
:202B60007265736F75726365205350495F53434B2032204231330A7265736F7572636520F7
:202B80005350495F4D49534F2031204130360A7265736F75726365205350495F4D49534F85
:202BA0002032204231340A7265736F75726365205350495F4D4F53492031204130370A7252
:202BC00065736F75726365205350495F4D4F53492032204231350A7265736F7572636520B0
:202BE0004144435F424154542031204230300A7265736F75726365204144435F435552527B
:202C00002031204230310A7265736F7572636520464C4153485F43532031204130300A721D
:202C200065736F75726365204F53445F43532031204231320A7265736F757263652047595B
:202C4000524F5F455854492031204130310A7265736F75726365204759524F5F435320310E
:202C6000204130340A7265736F75726365205553425F4445544543542031204331350A0ACD
:202C8000232074696D65720A74696D657220413033204146330A232070696E204130333A75
:202CA0002054494D39204348322028414633290A74696D657220423034204146320A2320B2
:202CC00070696E204230343A2054494D33204348312028414632290A74696D6572204230AD
:202CE00035204146320A232070696E204230353A2054494D33204348322028414632290AE3
:202D000074696D657220423036204146320A232070696E204230363A2054494D3420434872
:202D2000312028414632290A74696D657220423037204146320A232070696E204230373AD4
:202D40002054494D34204348322028414632290A74696D657220423033204146310A232019
:202D600070696E204230333A2054494D32204348322028414631290A74696D65722042310D
:202D800030204146310A232070696E204231303A2054494D32204348332028414631290A4D
:202DA00074696D657220413030204146320A232070696E204130303A2054494D35204348DF
:202DC000312028414632290A74696D657220413032204146320A232070696E204130323A40
:202DE0002054494D35204348332028414632290A74696D657220413038204146310A232073
:202E000070696E204130383A2054494D31204348312028414631290A0A2320646D610A6431
:202E20006D6120414443203120310A232041444320313A20444D41322053747265616D20CA
:202E400034204368616E6E656C20300A646D612070696E2042303420300A232070696E20A8
:202E60004230343A20444D41312053747265616D2034204368616E6E656C20350A646D6105
:202E80002070696E2042303520300A232070696E204230353A20444D4131205374726561DD
:202EA0006D2035204368616E6E656C20350A646D612070696E2042303620300A2320706941
:202EC0006E204230363A20444D41312053747265616D2030204368616E6E656C20320A64EA
:202EE0006D612070696E2042303720300A232070696E204230373A20444D41312053747271
:202F000065616D2033204368616E6E656C20320A646D612070696E2042303320300A2320FB
:202F200070696E204230333A20444D41312053747265616D2036204368616E6E656C20331A
:202F40000A646D612070696E2042313020300A232070696E204231303A20444D4131205394
:202F6000747265616D2031204368616E6E656C20330A646D612070696E2041303020300AFD
:202F8000232070696E204130303A20444D41312053747265616D2032204368616E6E656CD2
:202FA00020360A646D612070696E2041303220300A232070696E204130323A20444D413151
:202FC0002053747265616D2030204368616E6E656C20360A646D612070696E20413038205A
:202FE000300A232070696E204130383A20444D41322053747265616D2036204368616E6EFC
:20300000656C20300A0A2320666561747572650A666561747572652052585F5345524941B9
:203020004C0A6665617475726520534F465453455249414C0A666561747572652054454C37
:20304000454D455452590A66656174757265204F53440A66656174757265204149524D4F10
:2030600044450A0A232073657269616C0A73657269616C2030203634203131353230302023
:2030800035373630302030203131353230300A0A23206D61737465720A7365742062617207
:2030A0006F5F62757374797065203D204932430A736574206261726F5F6932635F646576E6
:2030C000696365203D20310A736574206261726F5F6861726477617265203D204E4F4E459D
:2030E0000A7365742073657269616C72785F70726F7669646572203D20534255530A73658A
:203100007420626C61636B626F785F646576696365203D20535049464C4153480A736574D9
:20312000206473686F745F69646C655F76616C7565203D203435300A736574206473686F9A
:20314000745F6275727374203D204155544F0A736574206473686F745F62697462616E67E8
:20316000203D204F46460A736574206D6F746F725F70776D5F70726F746F636F6C203D204F
:203180004453484F543630300A7365742063757272656E745F6D65746572203D20414443DD
:2031A0000A73657420626174746572795F6D65746572203D204144430A736574206D616732
:2031C0005F6861726477617265203D204E4F4E450A736574206265657065725F696E76659B
:2031E0007273696F6E203D204F4E0A736574206265657065725F6F64203D204F46460A739A
:2032000065742073797374656D5F6873655F6D687A203D20380A736574206D6178373435B2
:20322000365F7370695F627573203D20320A73657420666C6173685F7370695F627573205D
:203240003D20320A736574206779726F5F315F62757374797065203D205350490A736574EE
:20326000206779726F5F315F737069627573203D20310A736574206779726F5F315F73653C
:203280006E736F725F616C69676E203D2043573138300A736574206779726F5F315F616C5F
:2032A00069676E5F796177203D20313830300A00FFFFFFFFFFFFFFFFFFFFFFFFFFFFFFFFE0
:2032C000FFFFFFFFFFFFFFFFFFFFFFFFFFFFFFFFFFFFFFFFFFFFFFFFFFFFFFFFFFFFFFFF0E
:2032E000FFFFFFFFFFFFFFFFFFFFFFFFFFFFFFFFFFFFFFFFFFFFFFFFFFFFFFFFFFFFFFFFEE
:20330000FFFFFFFFFFFFFFFFFFFFFFFFFFFFFFFFFFFFFFFFFFFFFFFFFFFFFFFFFFFFFFFFCD
:20332000FFFFFFFFFFFFFFFFFFFFFFFFFFFFFFFFFFFFFFFFFFFFFFFFFFFFFFFFFFFFFFFFAD
:020000040800F2
:20400000AEBE08000E02000000000B0014020000000000FF000A00130200000000013F108D
:20402000000301010004040100A8160000010052000D000100010000001405040500000030
:204040000040000000000504050000000000080000010504050000000000000000050504ED
:204060000500000000000000001E05040500000000000000001F050405000000006400522C
:2040800000070009020000002A00FD01000019120000000000000000232A1A130000000041
:2040A00000000000232A0000000000000000000000000700FB010000130F00FC0100000091
:2040C00000000000000000000C00F70100002201000000000A00F90100003D3E00004500F5
:2040E000160200001303FF2401002501002601002701002301002A0100100200120200186C
:2041000001000000000000000000000000000000000000000000000000000000000000009E
:20412000000000160034000000DC0532000000000000000000000001040E001102000000FC
:20414000000000010101010A0012020100FFFFFFFF3E0018000300000103020405060709C2
:20416000000000000001006400DC051A046C070019750343080E000001000000001E1E1E23
:204180000101000000000000000000000000001100000200000000000000FF00000000000B
:2041A0000B00FF0102000000000000150008020100151617FFFF2D2E2FFFFF000000FFFF0C
:2041C0000900FA0100001002000E002A020000820058025E0102000E002002050003643284
:2041E00000F40196002A0006000100E001060000020124252627000000000001000001027F
:20420000030405060758022E04D007E8030C000A000C020000012C02001A00FE01000001CA
:2042200020000001210000010000000000000001FFFF0014002600010001000001000115E9
:20424000005802D903000020000B000300B3014A015E012C0164010100000001000A019A63
:2042600001001E0A0000022A001F00050000000000000100010005000001020300000000B8
:2042800000000000000000000000000000008017000A000502000000000000110001020062
:2042A00000000000000200000000000009000202000000000016001B02000006000000E8CE
:2042C000030000000000000000000012001B000200001800020301F40132000164F60021EB
:2042E0000200000000000000000000000000000000000000000000000000000000000000BC
:2043000000000000000000000000000000000000000000000000000000000000000000009D
:2043200000000000000000000000000000000000000000000000000000000000000000007D
:2043400000000000000000000000000000000000000000000000000000000000000000005D
:20436000000000000000000000FFFF000000FF1E0000FF3C0000FF5A0000FF780000FF9682
:204380000000FFB40000FFD20000FFF00000FF0E0100FF2C0100FF4A0100FF000000000027
:2043A000000000010B020D0A03050B030D0A030A0B040D0A03080B040D0A03070B030D0A18
:2043C00003000000000000060A0100000203060000000336003700010020003200C800D063
:2043E0000796001400320028004C0440060005500014000F00080064000100010005000A27
:20440000000000F40196000F000C0016000100C4090000B40028002F0001004D6574656F0C
:204420007236352070726F00000000000000000000000000000000000000000000160023F5
:20444000020200000000000000000000000000FF0000000F001E0000000005010000000026
:204460000000120005000200010100000000000000000000160012000300000000010001F4
:20448000055334313100000802008200FD070000E2008109CD084E00CE00820196097609A0
:2044A0008B0956092000EA00EA00EA00EA00EA00EA00EA00EA00EA00EA004A092C00EA005C
:2044C000EA00EA0061004100EA000B01EA006200EA00EA00EA00A30096002100EA00EA0038
:2044E0001601EA00EA00EA00EA00EA0041098200EA00EA00EA00EA00EA00EA00EA002109B7
:20450000EA002300EA00EA00CD00EA007200F5010900980864001401000A010A0000FF1F46
:204520000000142800002C3700008000FFFFFFFF4600010200000000000000000000000017
:2045400000000000000000000000000000000000000000000000000000000000000000005B
:2045600000000000000000005000C4FF00FFFFFFFF0100000005180B0C00000000001600E1
:20458000230002000A000000AEFFE4FF21000100000000001200F60102000000000001002E
:2045A00000000202000022001C020000000201140000110200000000840301020000000003
:2045C00000010000000000001C002800030000010200000000000000000000000000000090
:2045E000000000000B00140000000300002300120001000200E80364000F0A00010A001ED0
:2046000000EA000C000400320003070707000000434343460046050064CE07CE07CE070118
:2046200000000000000000000000000000320003070707000000434343410046050064CEA9
:2046400007CE07CE0701000000000000000000000000003200030707070000004343434154
:204660000046050064CE07CE07CE07010000000000000000000000000032000307070700C1
:204680000000434343410046050064CE07CE07CE07010000000000000000000000000032AF
:2046A0000003070707000000434343410046050064CE07CE07CE07010000000000000000A9
:2046C0000000000000320003070707000000434343410046050064CE07CE07CE0701000057
:2046E00000000000000000000000002A000A0009003000000000003F02000000000000000C
:20470000000000020000029E077D001F013F02000105017300C2010E00030064005200000E
:20472000000000284030007D00274034007C0023320000640032324B0000002800000000BD
:20474000000055F401900101374B000000FA00AC0D00000000320090015E01F40100000A27
:2047600064C8009001A50000050F00010F0114004B3200005A140B00005200A5000014009D
:20478000280100C8002D310025146400000000000000000000000032323296000119090FCF
:2047A0005A05000001695F5A91551464016E5F64004B00000000002D50280078002F542ECE
:2047C000007D002D500000780032324B0000002800000000000055F401900101374B000032
:2047E00000FA00AC0D00000000320090015E01F40100000A64C8009001960000050F00017D
:204800000F0114004B3200005A140B00004B009600001400280100C8001E220025146400BB
:20482000000000000000000000000032323296000019070F5A050000026464646464646400
:2048400001646464004B00000000002D50280078002F542E007D002D500000780032324BF1
:204860000000002800000000000055F401900101374B000000FA00AC0D000000003200903D
:20488000015E01F40100000A64C8009001960000050F00010F0114004B3200005A140B0037
:2048A000004B009600001400280100C8001E22002514640000000000000000000000003203
:2048C000323296000019070F5A05000002646464646464640164640A00130001000804445B
:2048E000100A0001010000000000000A0000010000900100000900020100006E0A01220158
:20490000220200000508E916D516C116AD169916851671165D16651678168B169E16B11679
:20492000C416D716EA164916351621160D16FD161117251739176C1680169416A816BC1693
:20494000D016E416F8161A163F1664168916AE16D316F8161D1700000000000000000000DC
:20496000000000000000000000000000000000000000000000000000000000000000000037
:20498000000000000000424F5343414D5F4100424F5343414D5F4200424F5343414D5F4513
:2049A00000464154534841524B005241434542414E440042414E44362020200042414E44B3
:2049C000372020200042414E4438202020004142454652363738310032003300340035008F
:2049E0003600370038000101010101000000050001000000020003000400000000000000FE
:204A000032352000504954003130300032303000343030004C5635004C5636004C563700E3
:204A20007600150000000000000000000000000000000000000000000000000000000000EB
:204A4000000000000000000000000000000000000000000000000000000000000000000056
:204A6000000000000000000000000000000000000000000000000000000000000000000036
:204A8000000000000000000000000000000000000000000000000700030000000066002A7C
:204AA00000000000000000E803D007DC0564FF00000000E803D007DC0564FF00000000E802
:204AC00003D007DC0564FF00000000E803D007DC0564FF00000000E803D007DC0564FF00AC
:204AE000000000E803D007DC0564FF00000000E803D007DC0564FF00000000E803D007DC0C
:204B00000564FF16002C000000E803D007E803D007E803D007E803D0077E0029000200003A
:204B200000203000000101203000000201102000001B022030000000000000000000000033
:204B4000000000000000000000000000000000000000000000000000000000000000000055
:204B6000000000000000000000000000000000000000000000000000000000000000000035
:204B8000000000000000000000000000000000000000000000000014001A0000007E05EA7A
:204BA00005B4053200E803D00700002A002B000000001E001E001E0005011E011E011E0131
:204BC0001E011E011E011E011E011E011E011E011E011E011E160019020000000000000050
:204BE00000000000000000000000003201250002000000000000000000000000000000005B
:204C0000000000000000000000000000000000000000000000000000000000000000000094
:204C2000000000000000000000000000000000000000000000000000000000000000000074
:204C4000000000000000000000000000000000000000000000000000000000000000000054
:204C6000000000000000000000000000000000000000000000000000000000000000000034
:204C8000000000000000000000000000000000000000000000000000000000000000000014
:204CA0000000000000000000000000000000000000000000000000000000000000000000F4
:204CC0000000000000000000000000000000000000000000000000000000000000000000D4
:204CE0000000000000000000000000000000000000000000000000000000000000000000B4
:204D000000000000000000000000000000000000000000000000000000000000004300034D
:204D2000020100000000000000000000000000000000000000000000000000000000000070
:204D4000000000000000000000000000000000000000000000000000000000000000000152
:204D60000C00F80103000101F401140008001000010000050B0019000000000028010012A3
:204D80000002000000000000000000000000000000460029020000000000000000000000A0
:204DA0000000000000000000000000000000000000000000000000000000000000000000F3
:204DC00000000000000000000000000000000000000000000000000A002C02000001000199
:204DE000001A000A02000000004A01B400D6010000C2010E0196004400000042001A0200AD
:204E0000000000000000000000000000000000000000000000000000000000000000000092
:204E2000004245464800424554414650564634313100000000000000000000010009003837
:204E4000000200000A078600040000000000000000000000000000000000000000000000B5
:204E6000000000000000000000000000000000000000000000000000000000000000000032
:204E8000000000000000000000000000000000000000000000000000000000000000000012
:204EA0000000000000000000000000000000000000000000000000000000000000000000F2
:204EC0000000000000000000000000000A0028020000000000000A0027020000000000006B
:204EE00016001F020000FFFFFFFFFFFFFFFFFFFFFFFFFFFFFFFF0C001D0200000000000060
:204F000000001800060201002829000020030000000020030000000020030A002700000085
:204F20002003000043000B02020000000000000000000000000000000000000000000000FC
:204F4000000000000000000000000000000000000000000000000000000000000000000051
:204F6000000000010000001A000D0201000000000000000000000000000000000000000006
:204F8000000C001E0200000000000000000700100200000000004E8BFFFFFFFFFFFFFFFFFB
:204FA000FFFFFFFFFFFFFFFFFFFFFFFFFFFFFFFFFFFFFFFFFFFFFFFFFFFFFFFFFFFFFFFF11
:204FC000FFFFFFFFFFFFFFFFFFFFFFFFFFFFFFFFFFFFFFFFFFFFFFFFFFFFFFFFFFFFFFFFF1
:204FE000FFFFFFFFFFFFFFFFFFFFFFFFFFFFFFFFFFFFFFFFFFFFFFFFFFFFFFFFFFFFFFFFD1
:20500000FFFFFFFFFFFFFFFFFFFFFFFFFFFFFFFFFFFFFFFFFFFFFFFFFFFFFFFFFFFFFFFFB0
:020000040800F2
:020000040800F2
:20800000134B0268196821EA02011960596821EA0201596019680A431A609968026821EA4A
:2080200002019960D96821EA0201D9604179102907D001F1804303F59E3319680A431A602C
:208040007047996811439960D9680A43DA607047003C0140024B9A6D136A002BFCD170479F
:20806000501A0020F0B401292D4C2E4D4FF0000694BF00230123EE62C4F81861C4F81C6117
:20808000C4F82831D4F82871D4F8F43047EA4207C4F82871EE63EC6B002A38D144F495748B
:2080A000EC631C6824F001041C601C68E407FCD4490289085960D8601968EAB921F04001D6
:2080C000196019498B421DD018494FF47410C860196841F01E011960596941F08001596143
:2080E000196841F00101196022B90E4AD36A43F00803D362F0BC704741F0400119600A49CF
:208100008B42E1D14FF0746041F8500CE0E744F01A04EC63EC6A44F00804EC62C1E700BF85
:20812000501A0020002C014058640240006402401248002302461178032902F1060218D047
:208140000133062BF7D10E4AD2F85031052B0FD0591C03EB4303C2F8501100EB4303032028
:2081600040F2EB3140F2FF32187059809A807047704703EB430300EB4303F0E77C1B002072
:20818000501A002030B5134A134B8DB0082102F1580082F8F0100693694400230DF1070517
:2081A0000124CDE9073302938DF8143009938DF828300B93CDE9035449F062FDFFF74AFF51
:2081C0009DF80700A0F1FF00B0FA80F040090DB030BD00BF501A0020DD810008826D136A4B
:2081E0005B681B78FF2B08D090F8F030013BDBB280F8F0301BB10120704700207047126A27
:20820000526802201370704770B4C3080D4CE25C00F00706B24004EBD004D2B20020C6F1B5
:2082200008038B4228BF0B46C3F108052A419840C91A40EA02004FF0000614F8012FEED1DB
:2082400070BC7047901A0020084AD2E9553199420AD0D118013391F85C110170C3F30A03E2
:20826000C2F854310120704700207047501A0020064AD2F85C39D2F86029934294BF4FF419
:2082800000600020013B9B1A18447047501A0020012380F85130704707B501A8FFF7D4FFCE
:2082A0000028FAD09DF8040003B05DF804FB044BD3E95503984288BF03F50063181A704764
:2082C000501A002001207047024BC3F86429C3F868197047501A0020024BC3F86C29C3F8D2
:2082E00070197047501A00207047704730B4134DD5E955239A4286BF03F50064A21A9A1ADF
:208300000A44B2F5006F13D8A9B101444A1E013810F8014FE918824203F1010381F85C41A3
:20832000C3F30A03F4D1C5F85831002030BC7047022030BC70470846F8E700BF501A002071
:20834000F8B51A4C94F87439002BFBD159B301444E1E451ED4F86029D4F85C1915F8017F97
:20836000531CC3F30A038B422CBF4FF400600020C91A22440144012982F87879C4F86039D8
:208380000FD1012048F0FCF8D4F85C39D4F860198B4294BF4FF4006200225B1A1344012B2B
:2083A000EFD0B542D6D10020F8BD00BF501A002010B5094CD4F88030084611465BB1D4F82F
:2083C0008030052B07D1002AD4F8843003DDFFF7B7FFD4F8843010BD482B002010B590F882
:2083E0005010002380F8503081B10B4CD4F8802072B1D4F88020052A0CD13C30D4F8843086
:20840000FFF79EFFD4F88430012010BD0120FCE71046FAE71846F8E7482B0020002280F8B6
:208420005120DBE790F85020531C0244DBB280F8503082F83C1090F851200AB1132B00D946
:20844000CCE77047212838B50C4605D022282FD0202813D0002038BD0029FBD0072AF9D1DD
:208460001A4BD3F8880093F88C1093F88D2093F88E30206021716271A371EBE70029E9D0EF
:20848000072AE7D1124AD2F868391BB1D2F86409096898470D4B256820796179A279C3F8AB
:2084A000885083F88C0083F88D1083F88E20D1E70029CFD0022ACDD1054AD2F87039002B65
:2084C000C8D00988D2F86C099847C3E7482B0020501A0020024B0020C3F88000704700BF70
:2084E000482B0020054B064A00200521C2F88010C3F87009C3F86809704700BF501A002059
:20850000482B0020704700BF704700BF704700BF704700BF704700BF704700BF704700BF8E
:20852000042301480B8070479801002010B4074A074B92F89000122403F114020C8001285A
:208540000CBF184610465DF8044B7047482B00209C01002000487047781A00200048704741
:20856000781A0020034B93F82400032894BF002001207047501A0020034B93F82400032824
:2085800094BF002001207047501A0020034B93F82400003818BF0120704700BF501A0020D9
:2085A000034B93F82400003818BF0120704700BF501A0020A0B182680D4B12B107229A7005
:2085C00070471978DA6003294FF004000CBF80214FF48071C3E901111A611A759870704783
:2085E000034B41F2E47101225A545A70704700BFF8BD00200378022B10D0006908B90120EC
:2086000070470C4B1B78032B0EBF0B4B80B24FF6F773984294BF0020012070470549436869
:2086200041F650028A58B3EB422F2CBF01200020704700BFF8BD0020F7FFFF0F0378022B9D
:2086400014D030B4104A4368006941F6480402F5C2511559096841F63C042B4012595B0AC6
:20866000023801FB0030104430BC7047064B426841F6340141F630005958185800EB410082
:2086800000EB5220704700BFF8BD002030B593B040F040020B0E0D0C04468DF80810080A6D
:2086A0008DF80420952101AA8DF805308DF80650002306258DF807008DF809100DF10300A2
:2086C00001210392134A0493CDE90733CDE90D33CDE909018DF818308DF82C300F938DF874
:2086E0004030119305950C92FFF74CFD00B974B9094B082203F1580003A983F8F02049F0CF
:20870000BFFAFFF7A7FC9DF8030013B030BDFF2013B030BD1D870008501A0020836D1B6A45
:208720005B681B78FF2B0AD190F8F030002B03F1FF3380F8F03014BF012002207047002060
:20874000704700BF30B5104A104B8DB0014682F8F01002F15800069302A900230DF107054F
:208760000124CDE9073302938DF8143009938DF828300B93CDE9035449F082FAFFF76AFC51
:208780009DF807000DB030BD501A00201D87000870B51C4D90B00024FD220DF1030305F152
:2087A0005800012601A98DF803200693CDE90144CDE90A44CDE90C442C628DF8104005944E
:2087C00007948DF824408DF838400F940396089649F056FAFFF73EFC3046FFF7B3FFFF2840
:2087E00009D0094BD3F884306B612046092385F8243010B070BD0423022085F8243010B0D7
:2088000070BD00BF501A0020482B002070B5064690B008200D46FFF795FFFF2821D0FE285B
:2088200002D0022010B070BD002402230E48089301A9CDE90265CDE90544CDE90A44CDE99D
:208840000C4401948DF8104007948DF824408DF838400F9449F014FAFFF7FCFB204610B0E0
:2088600070BD012010B070BDA81A002008B5FFF7F1FB0A2047F066FD024B186EBDE80840B8
:2088800048F064BE501A002070B50379254C002B14BF012200228AB084F8502003D184F829
:2088A00024300AB070BD054690F9001004F1580049F05CFBAD784DBB01261B482566C4F8BE
:2088C000EC4084F8646049F087FB03464FF47A70A4F85C3047F054FE206E48F037FE282205
:2088E0006846002164F0EDFF0A2310480293694649F0C6F9FFF7AEFB0D4B84F82460D3F8E6
:2089000084306361002323760AB070BD284648F033FB054608B11E23C3800921284647F011
:20892000E1F8C9E7501A0020801A0600A81A0020482B00202DE9F84F494B98420ED003F56E
:208940006853083398424ED0464B0020C3E94000A3F8FC00A3F80801BDE8F88F414C424F07
:20896000DFF810810223C4F8943004F198060025FB6AAB42294605F1010503D0D4F81801BD
:2089800053F056FD94F81C31D4F8182186F8243032623046414653F05FFFD4F894309D42F0
:2089A00006F13006E4DB002384F80A31D4E92803D4F89410B4F89C20B4F8A850C4F8283178
:2089C00012FB01F203FB01F3A4F8FC20B4F89E10264AA4F80851C4E94003A4F8FE10C4F8D8
:2089E000F8200120B8E71F4C1F4F0223C4F8943004F198054FF0000B4FF4806A4FF0400990
:208A00004FF40068FA6A01265A455946B34403D0D4F8180153F00CFDD4F8181194F81C2129
:208A2000296285F824204FF400314FF00062C5E90212A5F804A0A5F81090A5F80680AE7450
:208A4000FFF776FB28466E7653F052FED4F89420074B45F8303B9345D4DB84F80A61A5E756
:208A60001971EF00482B00209801002090D9060864D906081940EF002DE9F843194C94F8E5
:208A80002460042E0546894690461F4608D0082E02D00020BDE8F883FFF77AFE0228F8D14A
:208AA000206E48F04DFDA37E9BB969021120FFF7EDFDA0B90C4BC4F80090D3F88420656085
:208AC0000523C4E90387626184F824300120BDE8F88329461120FFF7D9FD0028EAD0FFF71F
:208AE000C5FED6E7501A0020482B00202DE9F04FCF4ED04D86468C4617460FCE05F596746E
:208B00002DED068B0FC40FCE0FC496E8070089B095F86231039784E80700CDE904EC042B67
:208B200000F24881DFE813F0B401460141010500C4019FEDC18ADFEDC18AC149C5F848119A
:208B4000C049C14BC14AC5F844110399002918BF134638EE887AF5EE006AC6EE879ABC4E9A
:208B6000C5F85031A6F1120B06F1C0080027DFEDB97A9FEDB99A28EE278AB0EE67AA059B29
:208B8000BB4200F00C811BF8013BEA1892F86741002C00F01481002202E0152A00F00F8164
:208BA00002EB42014FEA420918F80100A04202F10102F2D1294491F84512002900F0668108
:208BC0002046029344F02AFF029B82465046029344F044FF0178002940F0F180029BA94469
:208BE0000133DBB2032289F8853289F88422BAF1000F00F0E4804FEA141909F1FF39B9F1E0
:208C0000040F04F00F0000F20881944C04EB4901B1F884C04CFA00F111F0010100F0FD8016
:208C2000012101FA00F0013800EA0C00A144029362F04EFB99F890C0DFF838E2029B6044D0
:208C40000EEBC00C03228CF807308CF806205EF83000C6F814C000F13F4303F57E0304EBD2
:208C60009324012194F898309AF8082003F01F045B09032B01FA04F100F00381042B00F0E2
:208C8000FB80022B00F0CF80BCF804300693B3FA83F3C3F11F03C3F3CC0100EB810103F090
:208CA00007030C6A9B004FF00F0C0CFA03FC24EA0C040C620C6A02FA03F323430B6202234E
:208CC00006A907930CF00AF8039B002B00F08380B5F86031D5F8301507EE903AF8EEE77A3B
:208CE000FCEEE77A17EE900AB1FBF0F202F57F42FF32120CB1FBF2F295F86211B2FBF0F0D8
:208D0000042983B27ED007EE902AF8EE676A66EE887A29EE677A95F8630104990091A8EE3A
:208D2000A67A019051463046C6ED027A86ED037A36F0ECFF002F72DD7368D5F888219342A1
:208D40006FD0012F6BD0D5F8A021934269D0022F65D0D5F8B821934263D0032F5FD0D5F88B
:208D6000D02193425DD0042F59D0D5F8E821934257D0052F53D0D5F80022934251D0062F61
:208D80004DD0D5F81822D31A18BF012301370122082F3374727406F118067FF4F0AE30480A
:208DA00009B0BDEC068BBDE8F08F9FED2E8AF0EE488AC2E69FED2C8AF0EE488ABDE62B4AF6
:208DC000224BC5F848210020C5F8503109B0BDEC068BBDE8F08FB0EE690A63F0DFF9FCEE65
:208DE000C07A4FF6FF7317EE902AD5F83015B1FBF2F21A44120CB1FBF2F295F862110429E8
:208E0000184680D107EE900A07EE102AF8EE677AF8EE476A67EE8A7A7BE7716154E701239B
:208E2000B4E70023B2E7124B5C6C214359642BE7BCD90608482B0020ACC5A737ACC5A736B0
:208E4000B1E9030871E00408A5E0030865E00408CC2C00206F12833A00007A4464D90608D0
:208E6000742C0020282930386F120339F5E1030800380240F82D00200F4B1C6B214319635B
:208E800002E70D4B1C6C21431964FDE68A469DE69FED0A8A0A4A0B4BC5F84821C5F84431D0
:208EA00000220123CDE90332F0EE488A064B50E69FED068AEEE700BF003802406F12833AE2
:208EC000B1E9030871E0040865E0040800000000F8B5104ED6F83045054600680F4664087D
:208EE0000BF000FEB4FBF7F1B1F5803F03D3012CFAD96408F6E72246284689B244F02CFCF1
:208F0000054BC6F8983D28460449BDE8F840002244F030BB482B0020E9270208E0380020B0
:208F200010B5044C04480A4621460AF055FC204610BD00BFE8380020B85B070810B5044C65
:208F400004480A4621460AF047FC204610BD00BFE8380020C85B070810B5044C04480A46BC
:208F600021460AF039FC204610BD00BFE8380020D45B070810B5044C04480A4621460AF0D9
:208F80002BFC204610BD00BFE8380020E05B070810B5044C04480A4621460AF01DFC20469D
:208FA00010BD00BFE8380020EC5B070810B50C4C94F8F2200023236212B10A4AC2F8A03E7D
:208FC0005BF0F0FE20B10423022084F8243010BD044BD3F884306361092384F8243010BD46
:208FE000501A0020482B002070B50D4D95F82430042B04460E460AD0082B06D1EB6983422A
:209000000CD0FFF7D3FF022801D0012070BD0823C5E9074685F82430022070BD022070BDCE
:20902000501A002010B50AF0ABFB0F4C48B194F82430032B11D8237E0133DBB2072B2376C9
:2090400003D9002384F8243010BD084A0123D2F88420626184F8243010BD054848F0BCFFF0
:20906000A4F85C00E7E700BF501A0020482B0020801A060070B51D4C94F82430042B0646C5
:209080000D4608D0082B20D1E36983422BD0FFF77FFB022819D1206E48F052FA0021372067
:2090A000FFF7F4FA29461720FFF7F0FAA8B9A37E6BB971021920FFF7E9FA70B90823C4E91A
:2090C000076584F82430022070BD012070BD31461920FFF7DBFA0028F0D0FFF7C7FBFFF7A6
:2090E000A1FF032070BD022070BD00BF501A00202DE9F0412B4C0546884617461E4694F8C4
:209100002400042834D0082806D1E369AB4206D0FFF73EFB0228F2D00120BDE8F0814FF054
:20912000FC0CA26D2048117B204B80F8A4CEC3F8588051B1526942B194F8E020002A0CBF0B
:209140004FF480724FF4007201E04FF480721A661749184848F094FD01220623C4E9008588
:20916000C4E90376227284F824300020BDE8F081206E48F0E5F9A37E5BB969021820FFF7BD
:2091800085FA40B994F82430082BC8D04FF0FE0CC7E72946F2E7FFF769FBFFF743FF0320B8
:2091A000BBE700BF501A0020482B002098010020C8010020A81A002070B50379204C002B75
:2091C00014BF0123002384F8503003D1002384F8243070BD1B4D002195F9AB2E032047F03B
:2091E00089FD0028F2D04668304647F071FD84F8F1000028EAD095F8A93E003B18BF01233D
:20920000304684F8F2305CF027FD0AF0B9FA28B9237E84F824000133237670BD5BF0ACFE0C
:2092200030B1237E00220133237684F8242070BDD5F8843063610123207684F8243070BDD4
:20924000501A0020482B002010B55BF095FE48B10B4C237E0133DBB2072B237603D90023D2
:2092600084F8243010BD0AF08BFA0028F7D0054A0123D2F88420626184F8243010BD00BFE3
:20928000501A0020482B00202DE9F041844C94F85050002D00F0F28094F82420814E022717
:2092A000531E082B3FD8DFE803F035379C3E694F153E05005BF076FD002840F0E68063699B
:2092C000D6F88420FA3393422AD2FFF7BDFF94F82420E5E75BF066FD0028F0D0236A00228B
:2092E000012B227640F2D580E16994F8F200013B0131C4E9071310B16A4BC3F8A02E0822FD
:2093000084F82420A2F10805B5FA85F56D092846BDE8F08184F824705BF044FD002844D1F1
:2093200094F82420531EDBB2022B0AD85D4B6169D3F884305B1AC82BE4D9FFF785FF94F834
:209340002420042ADED1E2E7D4F82431002BD9D1544BE668D3F884306361072284F8242014
:20936000002ECFD0D4E9002123690120B047D7E76369D6F8841064338B42C3D2D4F820814C
:20938000B8F1000FF4D15BF00DFD00289FD0E66884F81880042384F82430002E73D0D4E9DD
:2093A000002123694046B047BAE75BF0A1F90028B6D196F8AD3E002BA3F10203B3FA83F3EE
:2093C00014BF022201225B096276A3765BF090F900287FF47AAF344A0323926CA26284F864
:2093E00024305BF085F900289AD12E4B206293F8DC6EB3F8DE0ED3F8E0EED3F8E0CED3F879
:20940000E07ED3F8E02E84F82E6093F8E41EA08593F8E56E84F8322093F8E50ED3F8E82E4E
:209420006263B3F8EE8EB3F8EE2E84F83310B3F8EE1EC2F30B1343EA182303F00F0301F0D2
:209440000F024FEA1E6E4FEA1C4C3F0A360900F00F0003F5FA63042184F8390084F82FE054
:2094600084F830C084F8317084F83860638784F83C2084F824102846BDE8F08184F8245069
:209480002846BDE8F081054641E7042384F824303DE7FAD1FFF78AFD94F82420531E42E708
:2094A000501A0020482B0020F83900202DE9F04FC64C94F8506095B0002E00F0818194F8AA
:2094C0002420C34F04F1580804F14009531E082B00F29680DFE813F034005A0020019400EA
:2094E0008300A500190094000900FEF74BFE002840F01A826369D7F88420FA3393427CD2CD
:20950000FFF790FD94F82420E0E7FEF73BFE0028F0D0236A0022012B227640F21B82E2698E
:20952000013B511CC4E90713082284F82420A2F10806B6FA86F67609304615B0BDE8F08F26
:20954000206E47F0FDFF00210846FFF79FF80546FFF78CF9012D50D1206E4FF0000A84F8E6
:2095600019A047F0EDFF40F2AB110820FFF78EF8052800F07A81012800F04281FFF776F924
:20958000627E002AD1D0022384F82430206E47F0D7FF637E022B0CBF4FF08045002500216D
:2095A0003720FFF773F829462920FFF76FF80546FFF75CF90DBB637E022B00F06981A5767D
:2095C000206E47F0BDFF00210920FFF75FF8002873D0FFF74BF994F82420531E10E0206815
:2095E0004FF40071FFF712F9012800F02681022800F02A81002800F03A8194F82420531E1D
:20960000DBB2022B0AD8724B6169D3F884305B1AC82B8CD9FFF706FD94F82420042A86D18D
:209620008AE7A26D117B136A002900F0D5805269002A00F0D18094F8E020002A00F0CC801B
:20964000B3FA83F35B09002BD7D004A900250DF10F0302220591404605A94FF0010ACDE9E1
:209660000B3A0792CDE90955CDE90E55CDE91055ADF8105006958DF820508DF834508DF8A1
:209680004850139548F0FCFAFEF7E4FC9DF80F3003F01F03052B00F05081FFF7C3FCD4F82C
:2096A0000CB0BBF1000F00F0DD802A46236961685046D84794F8242008E710214846FFF7F8
:2096C000A5F88246002884D101217F20FEF79CFD012805467FF47DAF50460221FEF794FD07
:2096E000002800F0038101287FF473AF16213A20FEF78AFD01308002A062FFF7B7F8206E1B
:2097000047F01EFF00210A20FEF7C0FF002840F0E680032384F82430102105A8FFF776F800
:2097200000287FF46AAF9DF821309DF822109DF81C209DF815009DF816501B01DBB243EA7C
:20974000111303F5FA636387DDF81D3001F00F0184F83C101BBA110902F00F0245EA00207A
:2097600084F8381084F839209DF814109DF817206363069B2363A08584F82E1084F82F2034
:20978000FFF774F8A37E6BB9206E47F0D9FE4FF400711020FEF77AFF0546FFF767F8002D67
:2097A0007FF4AEAE0B4848F017FC00220423A4F85C003046226284F8243015B0BDE8F08F48
:2097C000304684F8246015B0BDE8F08F501A0020482B002040787D012268217A4FF480737C
:2097E00002EB01214046002248F016FE237A0133DBB22372A3F10203B3FA83F35B0922E74A
:20980000042304AA05A9404607930692CDE909AACDE90BAACDF814A08DF820A08DF834A022
:20982000CDF838A048F02CFAFEF714FC9DF81330AB2B04BF02236376A0E66369D7F88420F4
:2098400064339342BFF4D9AEFFF710F8FFF7EAFBE5683DB10022104623696168A84794F806
:20986000242033E694F8242030E6657686E60190FEF7FCFFE56801982076042384F824306A
:20988000002D3FF459AED4E900212369A847B4E6206E47F055FE29463A20FEF7F7FE04AAF5
:2098A0008246042305A9404606920793CDE90955CDE90B5505958DF820508DF834500E95EE
:2098C00048F0DEF9FEF7C6FBBAF1000F07D1FEF7CDFF049B1BBAC3F38073A37670E6FEF7EF
:2098E000C5FFFFF79FFB94F82420EFE504212C20FEF78AFC032182464E20FEF785FC0C2187
:2099000083463620FEF780FC0BF1020B421C02FA0BF205FA0AF5A2FB0501420A42EAC1522B
:20992000A262FEF7A3FFEAE60190FEF79FFF01980423064684F82430FEE50E4BE568D3F868
:2099400084306361072284F82420002D3FF4EFAD504698E708D0042384F82430FEF786FF4C
:2099600094F82420531E4BE6FEF712FF02287FF444AE2EE6482B00202DE9F84FBA4C94F84A
:20998000081F0546C1F34001D4F8100F47F0E4FD94F8081FD4F80C0FC94301F0010147F08D
:2099A000DBFD002D00F0CD806E1EB04FB04D5FFA86FB4FF01008D4F8100F47F0B1FDD4F810
:2099C0000C0F47F0ADFDB4F8183F002B40F0438194F81A1FD4F81C0F47F0BEFD4FF0FA0979
:2099E0004FF47A704FF0010C7B68C3F30803002B40F00881EFF31183002B40F00381D4F845
:209A00008420A968D4F884309A42F8D1D4F8403F9942F4D8D4F83C6F00FB06F35B1AB3FBEC
:209A2000F6F300FB02327B68C3F30803002B40F0A880EFF31183002B40F0A380D4F8843073
:209A4000D5F808A0D4F884108B42F7D1D4F8401F8A45F3D8D4F83C6F00FB06F1A1EB0A01D7
:209A6000B1FBF6F100FB03139B1AB3F57A7FDAD3B9F10109B8D1D4F8100F47F051FDD4F8C6
:209A80000C0F47F04DFDB4F8183F002B40F0D78094F81A1FD4F81C0F81F0010147F05CFDB6
:209AA0004FF0FA0C4FF47A704FF0010E7B68C3F30803002B40F08680EFF31183002B40F010
:209AC0008180D4F88420A968D4F884309A42F8D1D4F8403F9942F4D8D4F83C9F00FB09F34F
:209AE0005B1AB3FBF9F300FB02327B68C3F308034BBBEFF3118333BBD4F88430D5F808A025
:209B0000D4F884108B42F7D1D4F8401F8A45F3D8D4F83C9F00FB09F1A1EB0A01B1FBF9F1C2
:209B200000FB03139B1AB3F57A7FDED3BCF1010CBCD10BF1FF365FFA86FBBBF1FF0F7FF48E
:209B40003AAFBDE8F88FEFF3118988F31288AE682B68DB0344BFC4F838EFAE68D4F884305C
:209B6000D4F8381F5FFA89F989F31188D4F83C9F0B4400FB09F1891BB1FBF9F100FB03139C
:209B8000D0E7EFF3118E88F31288D5F808A02B68D90344BFC4F838CFD5F808A0D4F88430D9
:209BA000D4F8381F5FFA8EFE8EF31188D4F83C6F0B4400FB06F1A1EB0A01B1FBF6F100FBA6
:209BC000031351E7EFF3118188F31288D5F808902B68DA0344BFC4F838EFD5F80890D4F8C2
:209BE0008430D4F8382FC9B281F31188D4F83C1F1A4400FB01F3A3EB0903B3FBF1F300FB5B
:209C0000023272E7EFF3118188F31288AE682B68DB0344BFC4F838CFAE68D4F88430D4F87F
:209C2000382FC9B281F31188D4F83C1F1A4400FB01F39B1BB3FBF1F300FB0232F3E6D4F8A5
:209C4000343F002B3FF42CAFD4F8203FC3F8009084F8319F24E7D4F8343F002B3FF4BEAE82
:209C600046F04EFDBAE600BF482B002000ED00E010E000E02DE9F84FB74CB84F94F8081FBA
:209C8000D4F8100FB64DC1F3400147F065FC94F8081FD4F80C0FC94301F0010147F05CFC21
:209CA0004FF0050B4FF01008D4F8100F47F038FCD4F80C0F47F034FCB4F8183F002B40F0FC
:209CC000438194F81A1FD4F81C0F47F045FC32264FF47A704FF0010C7B68C3F30803002BEC
:209CE00040F00781EFF31183002B40F00281D4F88420A968D4F884309A42F8D1D4F8403F67
:209D00009942F4D8D4F83CEF00FB0EF35B1AB3FBFEF300FB02327B68C3F30803002B40F067
:209D2000A780EFF31183002B40F0A280D4F88430D5F808A0D4F884108B42F7D1D4F8401FF4
:209D40008A45F3D8D4F83CEF00FB0EF1A1EB0A01B1FBFEF100FB03139B1AB3F57A7FDAD332
:209D6000013EB9D1D4F8100F47F0DAFBD4F80C0F47F0D6FBB4F8183F002B40F0DA8094F8F0
:209D80001A1FD4F81C0F81F0010147F0E5FB4FF0320C4FF47A7001267B68C3F30803002B69
:209DA00040F08780EFF31183002B40F08280D4F88420A968D4F884309A42F8D1D4F8403FA8
:209DC0009942F4D8D4F83C9F00FB09F35B1AB3FBF9F300FB02327B68C3F308033BBBEFF384
:209DE000118323BBD4F88430D5F808A0D4F884108B42F7D1D4F8401F8A45F3D8D4F83C9F9B
:209E000000FB09F1A1EB0A01B1FBF9F100FB03139B1AB3F57A7FDED3BCF1010CBCD10BF1C5
:209E2000FF3616F0FF0B7FF43FAFBDE8F88FEFF3118988F31288D5F808A02B68DB0344BFD6
:209E4000C4F8386FD5F808A0D4F88430D4F8381F5FFA89F989F31188D4F83C9F0B4400FBA6
:209E600009F1A1EB0A01B1FBF9F100FB0313CFE7EFF3118E88F31288D5F808A02B68D9037A
:209E800044BFC4F838CFD5F808A0D4F88430D4F8381F5FFA8EFE8EF31188D4F83CEF0B449F
:209EA00000FB0EF1A1EB0A01B1FBFEF100FB031352E7EFF3118188F31288D5F808902B68AB
:209EC000DA0344BFC4F8386FD5F80890D4F88430D4F8382FC9B281F31188D4F83C1F1A441A
:209EE00000FB01F3A3EB0903B3FBF1F300FB023271E7EFF3118188F31288D5F808E02B68EF
:209F0000DB0344BFC4F838CFD5F808E0D4F88430D4F8382FC9B281F31188D4F83C1F1A4428
:209F200000FB01F3A3EB0E03B3FBF1F300FB0232F1E6D4F8343F002B3FF429AFD4F8203F5B
:209F40001E6084F8316F22E7D4F8343F002B3FF4BEAE46F0D5FBBAE6482B002000ED00E04F
:209F600010E000E00E4B30B4DB68427801780D4CDB43C3F30223C3F10403DBB202FA03F3D2
:209F800060181B0101F01F050122490903F0F003AA4080F8003344F8212030BC704700BF49
:209FA00000ED00E000E100E000F01F0240090123032803FA02F304D004280CD0022805D09D
:209FC0007047074A116C0B4313647047044A516C0B4353647047024A116B0B431363704776
:209FE0000038024000285FD00368374A2DE9F04103F13F4404F57E0402EB9422012492F819
:020000040800F2
:20A00000982002F01F055209032A04FA05F456D0042A4FD0022A48D08588B5FA85F0C0F15A
:20A020001F00C0F3CC0603EB860600F0070082000F24306A944020EA04003062306A01FAB3
:20A0400002F20243002132624FF0010E0A464FF0030C02270EFA02F838EA050002F10102DE
:20A060001CD118680CFA01F420EA04001860186807FA01F606431E609E6826EA04069E6095
:20A0800098689860586820EA0800586058685860D86820EA0400D860D868D860102A01F19C
:20A0A0000201D7D1BDE8F0817047084A556C2C435464B1E7054A156B2C431463ACE7034AC1
:20A0C000156C2C431464A7E764D9060800380240144A154BD2F83025B3EB920F15D2B3EB24
:20A0E000D20F14D2B3EB121F13D2B3EB521F12D2B3EB921F11D2B3EBD21F10D2B3EB122F70
:20A1000034BF4FF480708020704702207047042070470820704710207047202070474020F1
:20A12000704700BF482B0020809698002DE9F04385B00D461746044647F06CFA002859DBF7
:20A140003B4EDFF8F88008EB000206EB800006F6847392F8A090C0F8443F002C60D0A28853
:20A160004FF00043B2FA82F2D34005D0314A116821EA0301116053612946204645F0B2FC75
:20A18000256805F13F4505F57E05AD0A204647F041FA00F0FC0303F1804303F59C3300F04F
:20A1A00003009A6880000F21814022EA01029A609A68EDB205FA00F0104398602CB1A08840
:20A1C0004FF00044B0FA80F0C44008EB87074E44D7F8B0308DF80D300021012302A88DF8E6
:20A1E0000E3002948DF80C10FDF70AFF96F8883FF02B02D805B0BDE8F0830F4B13F8093038
:20A200008DF80430F02103224FF4807301A886F8881F8DF80520ADF80630FFF7A3FEE9E75F
:20A220002946204645F05EFC4FF0FF35AEE700BF482B0020003C0140545C070864D90608D9
:20A24000002869D0F0B58388B3FA83F3202B85B00446C3F11F024AD0304E314D16444FF07C
:20A26000004005EB820230FA03F396F8A060C2F8441F05D02B4A116821EA03011160536168
:20A280002046002145F02EFCA3882268B3FA83F4C4F11F0303F0FC0101F1804101F59C31C2
:20A2A00003F0030398000F2702F13F438A68874022EA070203F57E038A60C3F3872383400E
:20A2C00088684FF000420343354422FA04F48B604FF40062012302A88DF80E300294ADF8DE
:20A2E0000C20FDF78DFE95F8883FF02B01D805B0F0BD0D4B9B5D8DF80430F02103224FF487
:20A30000807301A885F8881F8DF80520ADF80630FFF728FE05B0F0BD704700BF64D90608B9
:20A32000482B0020003C0140545C070810B4B8B10D4CD4F8903F102B05D15DF8044B052152
:20A34000002045F0B7BE03EB4302224482F8951F01210B4482F8940F82F8961FC4F8903F24
:20A360005DF8044B704700BF482B002080782021DCE700BF2DE9F04FDFF8ACA32DED028B53
:20A380009AF8D81F002297B0CAF8C82FCAF8CC2FCAF8D02FCAF8D42FCAF8C42F19B19AF8BE
:20A3A000D92F8AF8C42F9AF8DA2F1AB19AF8DB2F8AF8D32F9AF8DE2F1AB19AF8DF2F8AF80E
:20A3C000CE2F9AF8DC2F1AB19AF8DD2F8AF8C92F9AF8E03F05935A1ED3B257B203937B1C84
:20A3E00000F0AA80C54AC64E52F83790029602EBC70200231279019308EE102A1D46344672
:20A40000984626783946304648F09CFC83463046BBF1000F1ED046F0AFFDEA1D1321D2B272
:20A4200020B14FF0000E827180F807E045F05AFB207848F0B1FC4FF0070308F101022371CC
:20A440004FF0010384F802806070CDF804B05FFA82F8E3700135042D04F10504D1D118EE3F
:20A46000100A029ECDF81080FFF79EFDA549A64A4868024042F440324A600FB9019B5BB9A2
:20A48000A24C4820FFF790FD2046022160F0A8FCA26842F00102A2609A489C4A4168BAF802
:20A4A000E24F41F400014160516821F480515160916B21F4401141F480119163D16841F4BA
:20A4C0006001D160956B85F44011C1F3015101EB81011F2000FA01FC25EA0C0C112505FA1A
:20A4E00001F141EA0C019163D16841F0E061D160956BC5F30151C1F10401C9B201EB8101B8
:20A5000088404FF0120C25EA00000CFA01F108439063E4B1BAF8E41FCAF8EC4FA1B1BAF886
:20A52000E62FCAF8F01F62B1019B7948521A90FBF2F2CAF8F42F6BB917B0BDEC028BBDE83F
:20A54000F08F744A1288EFE7734A1188E7E7734A1488DFE74846049960F042FC684B01207E
:20A5600003F114080723F278441CE4B252B375783279A5F10A0101EB410105EB450C092D5E
:20A5800003FA01FE03FA0CFB02FA01F140F2A080D9F80C2022EA0E0E41EA0E01C9F80C103F
:20A5A000421E02EB82021F21062801FA02FC05FA02F273D8D9F8341021EA0C010A43204645
:20A5C000C9F834200536B045CDD1D9F80820039942F40072C9F80820D9F8082042F4807251
:20A5E000C9F80820D9F80820574442F00102C9F8082097F9E82F022046F07CFB04460028D8
:20A600009AD04668304646F063FB454A431E242101FB032393F89C50002D8DD1059983F8A6
:20A620009D10062283F89C20002885D0304646F04FFB5BF03DFA60680AF09CF907A80AF019
:20A640005BF9049EA26837480792012E8CBF4FF4806300230D9309F14C034FF48072CDE94B
:20A660000A56089309904FF4003360680C9507A94FF400674FF40056CDE91023CDE90E7651
:20A680000AF04CF96268136843F001031360D9F8083043F08043C9F808304DE7C11FA0F1EF
:20A6A0000D0201EB81014FF01F0E02EB82020C280EFA01FC0EFA02F005FA01F113D8D9F860
:20A6C000302022EA0C0211432046C9F8301079E7D9F8101002FA0CF221EA0B0B42EA0B02B0
:20A6E000C9F810205CE7D9F82C1005FA02F221EA00010A432046C9F82C2063E720DA060808
:20A700000C3B002000230140E030FCFF00200140803801002E7AFF1F2C7AFF1F2A7AFF1FFD
:20A7200098010020403B0020482B00202DE9F84F2E4F00EB800407EBC40454F8F46C2EB1A4
:20A74000054614F8DF0C00F0FF0820B14FF000084046BDE8F88F89469A46934645F0E4FE57
:20A760004FEA49010123C9B204F8DE1C04F8DDBC04F8DB3C04F8DA8C04F8DC3C04F8DF3C8C
:20A7800004F8E08CB28844F8D8AC9105814644F8D4AC1DD43388DA0510D442F20F7405E033
:20A7A00045F0C2FEA0EB0903A34215DC33889B05F6D433889BB243F480733380B3889BB2A5
:20A7C00043F440734FF00108B3804046BDE8F88F98464046BDE8F88F37F8803C01339BB266
:20A7E000284627F8803C5FF033FEB1E7403C002070B5464E16F87E4C04EB440306EBC303DE
:20A80000650013F87C3C032B6ED8DFE803F059291E02254406EBC50555F8780C002870D1E2
:20A8200016F81C3C9C425FD0013404F00302934206F87E2C58D002EB420406EBC4040223C1
:20A8400044F8780C04F87C3C70BD2B1906EBC30353F8782C72B1013A43F8782C002070BDE3
:20A860002B1906EBC30353F8782C002AF3D1022203F87C2C254406EBC50515F8703C013B20
:20A88000DBB205F8703C8BBB214B16F81C6CD3F8C01255F8740C621C02F003024B1E0324CB
:20A8A000B242034405F87C4CB3FBF1F045F8780C1AD0994218D8013845F8780C012070BD4B
:20A8C00047F074FF80B1124B2C44D3F8C02206EBC404012102F51C5304F87C1C0F33B3FB5E
:20A8E000F2F344F8783C70BD012070BD084BD3F8C022012002F2E733B3FBF2F345F8783C55
:20A9000070BD013845F8780C002070BD403C0020980100202DE9F84F3249DFF8D4B091F8B2
:20A92000AD1E01240229074619461046CBF820414FF000022C4C1D4618BF7F02FDF792FBE1
:20A940002A4B63626B02A362E36A40F2FF5943F093034FF400704FF48A62E3620121C4F8A6
:20A960003890A0601020E2605AF00EF8012D40F251434E46C4F83890CA4640F252488EBF18
:20A980004FF0120998464FF011090A25C4F838A00121A7604846C4F80C8059F0F5FF0346DE
:20A9A0004FF0000C40F2774201213720A6632BB900231846CBF81C31BDE8F88FA663C4F879
:20A9C00008C0E26059F0E0FF013DA6630028EFD015F0FF05DAD10346CBF82051CBF81C31D6
:20A9E000BDE8F88F482B0020002C014000E1F505501A00202DE9F843DFF8748098F82450A6
:20AA0000042D0446894617461E4608D0082D02D00020BDE8F883FEF7C9FA0228F8D101233D
:20AA20004A4620460021FFF775FF68B1FEF70CFCD8F80C40002CEBD00022D8F81030D8F87A
:20AA400004101046A047E3E7084BC8F80090D3F88420C8F804400523C8E90376C8F814207F
:20AA600088F824300120BDE8F88300BF482B0020501A00202DE9F84F3149DFF8CC9091F852
:20AA8000AD1E1E4602292F4B07464FF0010418BF4702012E40F25948C3F8244198BF4FF475
:20AAA0008B683B469346474640F2FF55B0468CBF4FF0190A4FF0180A0A241E4640F2FF531C
:20AAC000C9F838300121C9F808605046C9F80C7059F05AFF03464FF0000C40F277420121EC
:20AAE0003720C9F83850ABB9584641460122FDF7B9FA4646144A154B536276029662D36AB7
:20AB000043F09103D3620F4B00210846C3F81C11BDE8F88FC9F83850C9F808C0C9F80C209D
:20AB200059F032FF013CC9F838500028DCD014F0FF04C3D1034BC3F82441BDE8F88F00BF4D
:20AB4000482B0020501A0020002C014000E1F5052DE9F047364C82B005460E4617469846B5
:20AB600094F8240004280CD0082806D1E369AB4207D0FEF71BFA0228F2D0012002B0BDE898
:20AB8000F087DFF8B4A02660DAF8A09E6560C9F34F210F294FEA592222D8236A0193FBB1D9
:20ABA00094F8F200E0B1B9F5005F13D0214831464FF40072484462F023FE09F50072C2F3DD
:20ABC0004F211029CAF8A02E4FEA522202D0019B012B20D192B2013A164EAD1A0B4600E029
:20ABE000012332462846062601250021E760C4F81080257284F82460FFF73CFF0028BDD0C8
:20AC0000FEF722FBE66886B12846236961680022B0470320B2E7E269013B01320421C4E979
:20AC2000072384F824100220A8E70320A6E700BF501A002048770020482B0020F0B53B4CF2
:20AC400054F8185C2B78022B95B018D0012B02D0002015B0F0BD95F904506B1CF8D0022D47
:20AC6000F6DC0091134614F8141C024628465FF091FD0028ECD028465FF03CFEE9E72B6A09
:20AC8000002BE5D10DF10F0C8DF80F00002601200027CDE90833CDE90A12CDE90E67059332
:20ACA0008DF81C300D9310931293CDF810C006908DF830008DF84400EFF31180102383F316
:20ACC000128854F8183C1B6A13B3069B04AE32461BB1D3691432002BFBD12B6A13B3996883
:20ACE00039B993420AD0196829B15B6899680029F7D01433F3E70E4AC3E90026C0B280F374
:20AD0000118854F8182C136A002BFCD10120A0E704ABC0B22B6280F31188A4F118005CF03A
:20AD2000A5FAEEE7024A1A60FFDE00BF403C0020283C002003681A78012A01D0002070474D
:20AD400093F90430044A03EB830302EBC30313F8DF0CC0B2704700BF403C002070B50368B4
:20AD60001D78022D13D0012D01D0002070BD044693F904000A4B421C83F8B450F5D00228E5
:20AD8000F3DC0A46B4332179BDE87040CEE41B6A002BEAD1012247F09FFA012070BD00BFA1
:20ADA000403C002010B50B4C54F8183C1B78022B0FD154F8100C46F0C9FB54F8100C08B118
:20ADC0002123C380012144F08DFEFFF781F924F8140C10BD403C002038B505460A460C461C
:20ADE0000648294647F078FA45F08001034847F01DF9231A5842584138BD00BF283C0020F7
:20AE000030B583B00D46012301460DF107020446074847F0D1FB9DF8072035EA020304D005
:20AE200003482A43214647F05DFC03B030BD00BF283C002013B53A4C0023D4F8C4208DF8DA
:20AE40000730137803F0FD01012905D194F8C81011B90C2184F8C810022B1ED0032B2DD04A
:20AE600001220B212F4857F05FFE042045F088FB2C4801230DF10702002157F077FE0028E8
:20AE800038D09DF80730482B34D1274BC4F8B830264BC4F8BC3002B010BDD4F8CC0046F0EA
:20AEA00055FBD4F8CC0008B13523C380012144F019FEFFF70DF9A4F8C800D1E7D4F874355C
:20AEC000506846F2A8111961002380F888301222372157F0FDFDD4F8C4300D22586824213B
:20AEE00057F0F6FDD4F8C430302258686A2157F0EFFDB5E7D4F8C4301A78022A03D0032A6E
:20AF000007D00020C7E7D4F8CC0046F099FE0020C1E758681022372157F0DAFDF1E700BF60
:20AF2000403C0020043D0020CB2B06084D2C06082DE9F04FB54CB64E95B0002305464FF439
:20AF4000F0728B4604F6F800202184F8F43884F8F538019562F0B5FC202104F6D8204FF42B
:20AF6000F07262F0AEFCDFF8C0C2AA4932274FF0100E4FF47A704FF00108DCF80430C3F33E
:20AF80000803002B40F0BC80EFF31183002B40F0B780D6F884208D68D6F884309A42F8D179
:20AFA000D6F8403F9D42F4D8D6F83C9F00FB09F35B1BB3FBF9F300FB0232DCF80430C3F3FC
:20AFC0000803002B7BD1EFF31183002B77D1D6F88430D1F808A0D6F88450AB42F7D1D6F8EE
:20AFE000405FAA45F3D8D6F83C9F00FB09F5A5EB0A05B5FBF9F500FB03539B1AB3F57A7F72
:20B00000DBD3013FB9D194F8B92C002A52D094F8BA3C013B022B4DD803EB830004EBC001CA
:20B020007D4D91F8547D05EBC0004FF0010C022FC4F8BC0C84F844CD00F0C182DBB204EBFF
:20B040000313D3F8CC3DC1F8583D9BB302234FF4807081F8543DA5F188034C3DA1F8600D58
:20B06000C1F86C3DC1F8705D1509013D042D02F00F0200F28782694F07EB4503B3F884003C
:20B0800040FA02F3DB0740F17D82012303FA02F2013A10403D4460F01BF995F89020604B02
:20B0A000104403EBC000C4F8C40C8379002B47D0412B45D06FF0010015B0BDE8F08FEFF318
:20B0C00011898EF31288D1F808A00B68DD0344BFC6F8388FD1F808A0D6F88430D6F8385F17
:20B0E0005FFA89F989F31188D6F83C9F2B4400FB09F5A5EB0A05B5FBF9F500FB03537CE75E
:20B10000EFF311858EF31288D1F808900B68DB0344BFC6F8388FD1F80890D6F88430D6F8B1
:20B12000382FEDB285F31188D6F83C5F1A4400FB05F3A3EB0903B3FBF5F300FB02323CE7BC
:20B140002323C380092144F0CDFCD4F8C43C13B11A689B881383D6F83025324BB3EB920F95
:20B1600080F03382B3EBD20F80F03182B3EB121F80F03182B3EB521F80F03182B3EB921F95
:20B1800080F03182B3EBD21F80F03182B3EB122F80F02F824FF4807000230122FF210DF143
:20B1A0000F088DF80F10CDE90483CDE90833CDE90A33D4F8BC1CA4F8C00C0D9306928DF8EA
:20B1C0001C208DF83020EFF31180102383F31288D4F8BC3C1B6A002B00F0D881069B04AD99
:20B1E0002A461BB1D3691432002BFBD10B6A002B00F01582996839B99A421AD01968A9B1DF
:20B200005B6899680029F7D01433F3E7403C0020482B002010E000E09449002064D9060812
:20B22000F82D0020404B4C0000ED00E0B74AC3E90025C0B280F31188D4F8BC1C0B6A002B91
:20B24000FCD18C220120CDE908330DF10E0A05938DF81C300D93109312938DF80E20002324
:20B260000022CDE90E23CDF82880CDF810A006900B908DF830008DF84400EFF3118010238E
:20B2800083F31288D4F8BC3C1B6A002B00F08781069B2A461BB1D3691432002BFBD10B6A67
:20B2A000002B00F0BC81996839B993420AD0196829B15B6899680029F7D01433F3E7934A87
:20B2C000C3E90025C0B280F31188D4F8BC2C136A002BFCD19DF80F301B2B40F09081D4F8CF
:20B2E000C43C012284F8F4280BB12322DA80DFF81C92402248460A2146F0EEFF8A210023A7
:20B3000001228DF80E1000200021CDE90E01CDE90833D4F8BC1CCDF810A0CDF82880059352
:20B320008DF81C300D931093129306920B928DF830208DF84420EFF31180102383F31288AB
:20B34000D4F8BC3C1B6A002B00F03181069B2A461BB1D3691432002BFBD10B6A002B00F0F1
:20B360005B81996839B9934209D0196829B15B6899680029F7D01433F3E7C3E90095C0B26D
:20B3800080F31188D4F8BC2C136A002BFCD19DF80F2094F8B81CC2F3801284F8FC2D00293F
:20B3A00000F0D480022900F0B980D6F830355849B1EB930F80F01F81B1EBD30F80F009815B
:20B3C000B1EB131F80F00981B1EB531F80F00981B1EB931F80F00981B1EBD31F80F00D81C9
:20B3E000B1EB132F34BF4FF48076802694F8001EA4F8FE6D182914D1464F474800215B081E
:20B40000B3FBF6F3A7FB03730F465B0B66F30F076BF30F0163F31F4762F31F41C4F8081E92
:20B4200047603A48A4F8C06C0222002146F054FFC82044F087FFD4F8BC0C4FF0800B002627
:20B44000002700230122CDE90E67CDE908338DF80EB0CDF810A0CDF8288005938DF81C30D5
:20B460000D931093129306920B928DF830208DF84420EFF31182102383F31288D4F8BC3C75
:20B480001B6A002B38D0069B002B3DD02B46D96914330029FBD1006A002800F0BA80816887
:20B4A00039B9834209D0016829B1406881680029F7D01430F3E7C0E90095D2B282F311884A
:20B4C000D4F8BC0C036A002BFCD19DF80F3013F00203B6D1019841788278007884F8100EB2
:20B4E000C1F12001C2F11002184684F8111E84F8122E15B0BDE8F08F0562D2B282F311880D
:20B5000002485BF0B3FEDBE72B46C4E7FC480020809698005917B7D1484A0020D6F8303518
:20B520004048B0EB930F72D2B0EBD30F51D2B0EB131F52D2B0EB531F53D2B0EB931F54D2CC
:20B54000B0EBD31F34BF802640264FE7D6F830353549B1EB930F4ED2B1EBD30F39D2B1EBF5
:20B56000131F3AD2B1EB531F3BD2B1EB931F3CD2B1EBD31F41D2B1EB132F34BF4FF480766B
:20B58000802633E70020C4F8C40CDBE504ADC0B20D6280F3118825485BF068FE4CE60D6222
:20B5A000C0B280F3118821485BF060FE8DE60D62C0B280F3118848465BF058FEE2E691F81B
:20B5C000613D634481F8613D4EE50220E4E50420E2E504260AE70820DEE5082606E71020B5
:20B5E000DAE5102602E72020D6E52026FEE64020D2E58020D0E50226F8E64026F6E6D4F8C8
:20B60000C40C202144F06EFA4FF0FF3054E50E46ECE6C0F80090FFDEC3F80090FFDE034A16
:20B620001A60FFDE002D3101404B4C00FC4800200146014846F0FABC544A002001448842D0
:20B640000ED010B40346074C074813F8012B04FB00F0994280EA0200F7D15DF8044B7047CD
:20B660000148704793010001C59D1C81094B93F86231042B08D9053B032B08D801231A46E2
:20B6800000B103701046704700230122F8E700231A46F5E7482B0020F0B40D6800240CE039
:20B6A000BCF1050F18D8A0F137030A2B14D104EB840415F8010B03EB4404A0F13003DEB2DA
:20B6C000092EA0F16107A0F1410CF0D9052FE7D8A0F157030A2BEAD00D601460F0BC704782
:20B6E0009FED727A07EE901A20EE070AF8EE677A27EE800AFDEEC07A17EE903A2033402BFC
:20B7000000F2C480DFED6A7AB4EEE70AF1EE10FAF0EE407A0CDD9FED676ADFED676AB0EEAE
:20B72000677AB4EEE67AF1EE10FA77EEC67AF6DC9FED627AF4EEC77AF1EE10FA0CD59FEDE5
:20B740005D6ADFED5F6AB0EE677AB4EEE67AF1EE10FA77EE867AF6D49FED5A7AF4EEC77A71
:20B76000F1EE10FA00F38A809FED577AF4EEC77AF1EE10FA44BF9FED517A77EE677A27EEC5
:20B78000A76ADFED525A9FED527ADFED526AA6EE257A67EE865AE6EE076AB6EE007AE5EEA2
:20B7A000A67A27EE877ADFED476A70EE267ABDEEE76A16EE103A2033402B64D8B4EEE60A02
:20B7C000F1EE10FA0CDDDFED3B5A9FED3B6AF0EE676AF4EEC66AF1EE10FA77EEE57AF6DCC5
:20B7E000DFED366AF4EEE67AF1EE10FA0CD5DFED315A9FED336AF0EE676AF4EEC66AF1EEB1
:20B8000010FA77EEA57AF6D4DFED2E6AF4EEE67AF1EE10FA3DDDDFED266A76EEE77A67EEB1
:20B82000A75A9FED2A5A9FED2A6ADFED2A6AA5EE856A27EEA55AE5EE866AB8EE006AE5EE3B
:20B84000267A67EE867AC7EE206AB7EE006A76EE865A76EE666A86EE257A80ED091A67EE35
:20B86000277A66EE876AC0ED017AC0ED037A80ED007A80ED027AC0ED046A70479FED0C7ADC
:20B8800077EE677A7BE7DFED147ADCE79FED127A89E7DFED0D6AF4EEE67AF1EE10FA44BFEA
:20B8A000DFED066A76EEE77AB9E700BF27D4D236DB0F4940DB0FC940E4CB1641DB0F49C0C6
:20B8C000E4CB16C1DB0FC93FDB0FC9BF92E741B99730083C15A82ABE00000000E14B2DE919
:20B8E000F04103F56B63E04ED3ED000A96F83043F8EE600A2DED028BC6EDCB0A002C6FD16D
:20B90000DFF8C4C396F84073C6F83C439CF80040002F39D0B6F836339FEDD46A9FEDD47A84
:20B9200007EE903AF8EE677A20EE877AC6EE276AD04B0022012F1A6076EE876AC7EE267A9C
:20B94000C3ED017A20D0022F9A60C3ED037A1BD0032F1A61C3ED057A16D0042F9A61C3EDE9
:20B96000077A11D0052F1A62C3ED097A0CD0062F9A62C3ED0B7A07D0072F1A63C3ED0D7A7F
:20B9800002D09A63C3ED0F7ABB4B9FEDBC6A93F882319FEDBB7A9FEDBB0ABB4A07EE903AD3
:20B9A000F8EEE77A9CF8583BC6EE276A1C4414FB07F4E4B207EE904A60EE870AF8EEE77ADF
:20B9C000C2ED006AA7EEA00A60F0F4FCBDEC028BFCEEC07A17EE903A86F89034BDE8F0814E
:20B9E00096F831339FEDA96AB6F832239FEDA82ADFEDA86ADFF8D0C296F84073C6F83CC310
:20BA000007EE903AFCEEE05AB6F834338CF8004007EE103A15EE903AF8EE655AF8EE677AF2
:20BA200086EE255ACCF81430012386F8383306EE102AB8EEC77A27EE822AB8EE466A67EE7D
:20BA4000266A22EE252A8CED025ACCED017A8CED036ACCED046A002F96D0DFED8F7A9FEDEB
:20BA60008F4ADFED8F5AC7EE871AC7EB0715A7EB07180CEBC5054FEAC8084FF0000EB1EEAD
:20BA8000611A9FED886A08EB05009FED873ADFED873ADFED876A0346002207EE902AB8EE5E
:20BAA000E77A27EE027AFDEEC77A17EE901A2031402900F2D080B4EEC47AF1EE10FAF0EE16
:20BAC000477A0CDDDFED7B4A9FED7B5AF0EE672AF4EEC52AF1EE10FA77EEE47AF6DCF4EE2A
:20BAE000E57AF1EE10FA0CD5DFED724A9FED735AF0EE672AF4EEC52AF1EE10FA77EEA47A90
:20BB0000F6D4F4EEC67AF1EE10FA40F39A8074EE677A27EEA75AB0EE630AA5EE030ADFED33
:20BB2000684AE5EE004A65EE272AB7EE005AE2EEA47AB0EE458AF0EE454AA1EEA78AE1EE3C
:20BB4000274AC5EE088A84EE880A77EE067ABDEEE75A15EE101A203140296FD8B4EEC67A4A
:20BB6000F1EE10FA0CDD9FED535A9FED537AF0EE674AF4EEC74AF1EE10FA77EEC57AF6DC80
:20BB8000F4EEE57AF1EE10FA0CD59FED4A5A9FED4B7AF0EE674AF4EEC74AF1EE10FA77EE49
:20BBA000857AF6D4F4EEC67AF1EE10FA3CDD74EE677A27EEA75AF0EE632AE5EE032A9FED48
:20BBC000407AA5EE227A65EE274AB8EE005AE4EE877A67EE857A87EE887A0132A24203F10F
:20BBE000280343ED048A03ED037A03ED017A43ED028A83ED000AC3ED056AC3ED026AC3ED63
:20BC0000016AC3ED046AC3ED036AFFF646AF783085427FF43AAF0EF5707EBEF5346F05F588
:20BC200070757FF42EAF75E69FED267AF4EEC77AF1EE10FA48BF75EEE77ABAE7F0EE667A12
:20BC4000C9E79FED205AF4EEC57AF1EE10FA48BF75EEE77A5DE7B7EE000AF0EE408AB0EE20
:20BC6000408A72E7403C0020384D002083F9223EBD378635CC510020482B002055555540C6
:20BC80006E12833A48E1FA3EC45100200060EA4827D4D2360AD7233C00004842DB0F4940FF
:20BCA000DB0F49C0DB0FC93F92E741B99730083C00000000DB0FC940E4CB1641E4CB16C1A2
:20BCC00015A82ABEDB0FC9BF48A700202DE9F04F07EE900A2DED068B9FEDF27AF24EDFEDAB
:20BCE000F36AB6F8D43496F8DA54C6F82C05B8EE679A0AEE103A87EE095AB6F8D634C6F84F
:20BD0000E854002283B0C6F8EC2408EE103AB6F8D834DFEDE77AB8EE4AAA08EE903AB8EE9D
:20BD2000C88A3AEE0A7AF8EEE88AB4EEC78AF1EE10FA68EEA77AB4EEE65A06F2DC43B8BFEA
:20BD4000B0EE478AF1EE10FA83ED028A83ED01AAC3ED007A00F1FE8207EE905AF8EEE77AB3
:20BD6000B7EE007AC7EE279AD24B96F8A01E1A46143201929E4603F12C04F6EE005A65EEF3
:20BD8000256AF7EE007A86EE887ADFEDCB3ADFEDCB4A9FEDCB6AD3ED05AAB4EEE77AF1EE7B
:20BDA00010FAB8BFB0EE677ABDEEC77AB0EE004A17EE107AB8EEC77A29EE066AC5EE076A8E
:20BDC000C6F8887787EE875A66EEA36AAEEC015A8AEE267AC8EE267A37EE257A77EEA57A44
:20BDE000B4EEC47AF1EE10FAF4EEE47AB8BFB0EE447AF1EE10FA88BFF0EE647ABDEEC77A8F
:20BE0000FDEEE77A17EE102A17EE900A02F1FF3B00F10108BBF1230FA8BF4FF0230BB8F176
:20BE2000230FC1462BEAEB7BA8BF4FF02309C345C8BFD946012FB8BF0127A9EB0B08CEED9D
:20BE4000006A98FBF7F883ED046AC6F89427C6F8980708F10108002940F0E380DFED990A15
:20BE6000DFED995A9FED992A9FED995ADFEDA42A9FEDA43ADFEDA43A9FED964ADFEDA31A92
:20BE800003F5E36207EE901AB8EEE76A66EE207A37EEA57AFDEEC76A16EE903A2033402BF5
:20BEA00000F21182F3EE026AB4EEE66AF1EE10FA0CDDDFED914ADFED8F6AB0EE471AB4EEDF
:20BEC000E61AF1EE10FA37EE647AF6DCB4EEC57AF1EE10FA0CD5DFED884ADFED886AB0EEFF
:20BEE000471AB4EEE61AF1EE10FA37EE247AF6D4B4EEE57AF1EE10FA40F3FA81DFED766A85
:20BF000036EEC77A67EE076AB0EE431AA6EEA21AB0EE630AA1EE260A67EE264AFDEEE76AE0
:20BF2000A4EE807A16EE903A2033402B27EE047A00F2D381DFED696AB4EEE66AF1EE10FA96
:20BF400040F3FC819FED6C0A9FED6A1AF0EE676AF0EE664AF4EEC14AF1EE10FA76EEC06A7E
:20BF6000F6DC9FED5D1AF4EEC14AF1EE10FA13D59FED611ADFED614AB0EE660AB4EEE40A12
:20BF8000F1EE10FA76EE816AF6D4DFED546AB4EEE66AF1EE10FA0CDD9FED576ADFED556A79
:20BFA000F0EE674AF4EEE64AF1EE10FA77EEC67AF6DCF4EEC57AF1EE10FA0CD59FED4E6A51
:20BFC000DFED4E6AF0EE674AF4EEE64AF1EE10FA77EE867AF6D4F4EEE57AF1EE10FA40F3C7
:20BFE0007F81DFED3D6A76EEE77A67EEA76AF0EE434AE6EEA24AB0EE631AA4EEA61A27EEF6
:020000040800F2
:20C00000A66AE6EE017A67EE847A0131242982ED007AC2ED017A02F108027FF433AFDFEDBE
:20C0200030AA4FF0000A44E905AB44E902874FF490720021204644F80C9C61F042FC4FF4C8
:20C040009072A018002161F03CFC264B04F51574A342E8D1019BDFED247AC3ED00AA012367
:20C0600029EE279A86F8A03E002D00F02781DFED1F7A1F4E9FED182ADFED152AC7EEA81AA5
:20C08000A6F1140406F5117738EE4A8AB1EE611A69EE889ADFED0C5ADFED0C6A234630468E
:20C0A0003AE000BF00247449384D00200000FA440AD7233CC4540020398E633C00000C42B7
:20C0C0009C534937C3B8B23DDB0FC93F00000000DB0F49C072F97F3FDB0F494000001042B4
:20C0E000BC297E3FEC5B002027D4D2360000484228520020E4CB1641DB0FC940E4CB16C191
:20C1000092E741B99730083C15A82ABEDB0FC9BF000010C20000807F0022B7EE005A07EEA3
:20C12000902AF8EEE77AB6EE007A77EE877AB0EE4A7AA7EEA97AF0EE477A29EE077AE0EC5D
:20C14000017AFDEEC77A17EE901A2031402900F2D780B4EEC27AF1EE10FAF0EE477A0CDD37
:20C160001FED1B4A5FED1D4AB0EE676AB4EEE46AF1EE10FA77EEC47AF6DCF4EEE27AF1EEC1
:20C1800010FA0CD51FED244A5FED244AB0EE676AB4EEE46AF1EE10FA77EE847AF6D4F4EE29
:20C1A000E57AF1EE10FA40F3B58072EE677A67EEA74A5FED2D3A1FED2D4A1FED2D6AA4EEDD
:20C1C000A34A67EEA43AA4EE246AF0EE454AE3EE867AB0EE456AE1EE274AA1EEA76A84EE42
:20C1E000864AC5EE064A77EE257AFDEEE73A13EE901A2031402900F28A80B4EEE57AF1EE1B
:20C2000010FA0CDD1FED443A5FED463AB0EE677AB4EEE37AF1EE10FA77EEC37AF6DCF4EE18
:20C22000E27AF1EE10FA0CD51FED4D3A5FED4D3AB0EE677AB4EEE37AF1EE10FA77EE837AA9
:20C24000F6D4F4EEE57AF1EE10FA6DDD72EE677A27EEA73A5FED560A5FED563A1FED567A05
:20C26000E3EE203A63EE270AA3EE237AF8EE003AE0EE877A67EEA37A87EE867A0132AA42EE
:20C2800003F12803C3ED0B4A83ED0C7A83ED0E7AC3ED0D4A83ED0F4A83ED145AC3ED116AB3
:20C2A000C3ED106AC3ED136AC3ED126A7FF437AFC834A74206F114067FF4ECAE03B0BDEC43
:20C2C000068BBDE8F08FFDEEE76AB0EE427A16EE903A2033402B7FF62DAEF0EE427A94E623
:20C2E000F4EEE17AF1EE10FA48BF75EE677A7CE6B4EEE17AF1EE10FA48BF35EE477A01E6B3
:20C30000B7EE004AF0EE444AB0EE446A6BE7F0EE667AB1E71FED836AF4EEC67AF1EE10FACA
:20C3200048BF72EEE77A42E71FED887AF4EEC77AF1EE10FA48BF72EEE77A89E75FED8C6A78
:20C34000B4EEE66AF1EE10FA48BFF0EE676A3FF50FAE2EE65FED919AC6F8E824154603E5C3
:20C360000848002302461178022902F1060204D00133062BF7D10020704703EB430300EB5C
:20C38000430070477C1B002000B50021084B83B00846C3F8C41F33F08FFC0422054B0193EC
:20C3A0000DEB0201062033F07BFC03B05DF804FB384D00205475C52A70B5461E00F13105AE
:20C3C000344614F8011F601E801BFF29C0B201D033F072FCAC42F4D1A02055F0DDFA0121F1
:20C3E000022033F069FC40F2E93401E0013C04D04220FFF71DF90028F8D16220FFF718F96A
:20C400001321242033F058FC2520092133F054FCBDE87040A02055F0BFBA00BF10B58CB0B8
:20C4200000234CF20502044601A9CDE90633CDE90833ADF800208DF8023003220B9301235D
:20C44000CDE903128DF814308DF82830CDF808D046F028F8204602A945F012FC204646F088
:20C4600021F89DF806000CB010BD00BF2DE9F043784D794F83B005F596702422002161F0FF
:20C4800020FA97F8C94F0023C5F85031002C3CD1724ED6F8F83063B39B6A53B370489847D3
:20C4A000836833B303886F4F013B9BB2BC46384600210678032E00F106001ED00131062943
:20C4C000F7D100223978022907F1060700F0A1800132062AF6D1D5F85011052909D0481CBD
:20C4E00002FB01C2C5F8500102200021938010705180204603B0BDE8F083062303FB01511D
:20C50000B1F82E31013B9BB2DBE797F8C80F07F57D63C7F8CC3F10B9504E0024B9E744F05D
:20C520002BFDC7F8D80F18B183790BB1412BF3D121464D4845F01AFD04460028ECD0D7F837
:20C54000CC3F474A9868C3F8942008B12023C380092143F0C7FAD7F8CC3F404E986844F0D7
:20C56000F5FF4248D7F8CC8F45F036FD4FF00109A8F804003220C6F8188186F81C9143F0B7
:20C58000FFFF0423D7F8CC0F4FF0000C0DEB03029F21CDF804C045F04BFE9DF805809DF80E
:20C5A00004309DF806104FEA082848EA034848EA0108414606F1F80050F04EF900287FF4E3
:20C5C00068AF4046FCF7B6F9034600287FF461AF9DF806009DF805209DF80710000240EAFB
:20C5E0000240234A0843904217D0C6E94033A6F8FC30A6F80831FCF79DF9804600287FF4DB
:20C6000048AF97F8C80F44F0B7FC45F019FB44463FE7062101FB02C266E7164AC6F8FC206F
:20C620004FF400334FF00062C6F800314023A6F80831C6F8042186F80A91FBF779FD06F15F
:20C64000F80086F8119150F053F80B4BC6F8F8301FE700BF501A0020384D0020482B002074
:20C66000402C00207C1B0020085D0020404B4C0021AAEF000004000864D906082DE9F041C3
:20C68000BC4BBD4EBD4DBE4C0822C3F88820336B82B043F00103336307464FF4C05228463A
:20C6A00040F2023388466946CDE9002308F016FB6B6AC4F8548523F470436B626B6AC4F822
:20C6C0005C7543F420436B626B6AAE49C4F8581523F470236B626B6AAB4844F8900C43F4DF
:20C6E00020236B62736CA94944F88C1C43F480437364736BA648A74944F8800C43F080036A
:20C7000002257363A44F04F8885CA44EA44D44F83C1C4FF0A04344F8843CA24A44F8747C9C
:20C7200003F53463A1F5D07144F8385C44F8706C44F8343C44F86C1C0123DFF898C244F8AA
:20C7400078CC07F51077A5F5E465A6F5A066A1F58C6144F8307C44F87C5CE66304F8853C09
:20C7600005F5A075536106F5B076216084F8823019468D4B8D4AA560A7F5BC67A0356661B8
:20C780008B4E2761A36107F5D45703F56953E5614FF050250020DFF840E22264ACF5687C3B
:20C7A00002F5A0426764A66407F5A04706F5A046E3642565A3F54853A4F19005C4E91676A0
:20C7C0006265E367C4F804E0C4F80CC002462B4684F88400402683F81C21A3F82221013238
:20C7E000042AC3E9496083F81D1183F81F01C3F8300103F12803EED1002211462B4640205E
:20C8000083F87423A3F87A230132042AC3E9DF0183F8751383F87713C3F8881303F1280364
:20C82000EED14FF0A04363489A6822F001029A60DA6842F04002DA6007F00EFB14F8873C9C
:20C840000022212161F317420BB142F4801214F88D1C54F8843C01299A6300F0E280DA68C7
:20C86000E66F54F8800CC2F3076121F0600141F0400161F31F620021DA603160026861F30B
:20C88000CC22026014F8852C012A00F0B7801021494807F033FE484807F016FE54F8800CDC
:20C8A00014F88F3C00224FF0FF31026142618161C26153B305F11407404E114607EB83078D
:20C8C0004FEA830C4FF0FF0E56F8042F1368002BACBF00234FF09043B74213601161C2F8E5
:20C8E00008E0F1D105F15003354963440027FF2651F8042F1568002DACBF00254FF090450A
:20C900009942156017619660F2D1036914F88D1C43F480730129036160D054F8842C294820
:20C920000023936100294FF0FF336FF0804151615360516114BF00231023906143F470133B
:20C940009069D4F8581543F4605343F00803034393619368096843F00103936088471A4B79
:20C960001A4ADA6068461A4B0093FDF7FBFA02B0BDE8F08100E100E0003802400000024045
:20C98000305E00205C040020080401004000400100080050000B0050200900504009005016
:20C9A000200B0050003C0140C00500500010005000300050AC5D0020A05D0020B45D002013
:20C9C000F05D00200008008000ED00E00005FA0543020001000900502005005054F8842C81
:20C9E000144B03636FF08041134D00234FF0FF30936151615060516195619FE701680F4A1B
:20CA00000F4E41F003010160802159629E62C3F80421E022C3F80821C0F24002C3F80C2125
:20CA200035E79A6822F03E0141F02A0161F307029A6014E70301810000080080A0004000EC
:20CA40008000200010B5194C94F86505B8B9184B83F85100586594F86835012B05D0022B62
:20CA600020D0D4F86C351BB910BD124BC4F86C3511495B68BDE81040A1F10C00184744F0BB
:20CA80007BFA94F867250A49003A18BF012281F8512048650028DED01F22C280202143F01E
:20CAA00021F8D8E7054BC4F86C35E1E7305E0020501A00209C040020A06300207804002072
:20CAC00099B10A6B824216D9154BD3F8AC25914221D34C3991421ED30B6B9842F9D38B6BC6
:20CAE0009842F6D80B46184670470D4BD3F8AC150A6B904212D30B680BB9F4E70A6B9042BF
:20CB00000B4602D38A6B9042EDD951F84C3F002BF4D1184670470023184670470A46D8E742
:20CB2000305E00202DE9F047CC0143D10346224A43F8082B4FF0FF324260022418467E26BC
:20CB4000DFF87880D8F8B0952644013E051D49466FF070474FF0010A08E0A3421CD0631CFF
:20CB600045F8043C321B1C460435CAB10B6BA34202D88B6BA34204D22046FFF7A1FF0146AC
:20CB800090B10A794B6B002AE7D1A34204D0E6D245F8042C631CE5E745F8047C631CE1E70C
:20CBA000C8F8B015BDE8F08745F804AC321B631C4946D8E78026C3E7F8FFFF0F305E0020CA
:20CBC00070B4447941BB03684FF400524FF40076202502213CBB1A8C22F001021204120C71
:20CBE0001A841A8B188C22F0F30280B2120420F00A00120C014342F0010241F001011A837E
:20CC000019841A8B22F00C021204120C1A831A8B92B270BC1A837047002203681646154634
:20CC20001146002CD7D0042C21D0082C38D0198C21F480510904090C19849C8B1D8C45F618
:20CC4000FF7040F6FF4128402140024342F4805241F4807199831A849A8B22F44062120406
:20CC6000120C9A839A8B92B270BC9A8370471A8C22F010021204120C1A84188B198C89B2F1
:20CC800040F6FF4221F0A00102400D4342F4807245F010051A831D841A8B22F44062B3E732
:20CCA0001A8C22F480721204120C1A84998B1A8C21F0F30192B2090422F42062090C3243B2
:20CCC00042F4807241F0010199831A849A8B22F00C02C4E738B50E4D0446006807F002FF5D
:20CCE000D5F83025204652084FF6FF7140F034FD20460021FFF764FF064BC5F89C3D05F67A
:20CD00009C5120460022BDE8384040F033BC00BF482B0020F50E0208036870B55E6A26B1D4
:20CD200033460522BDE87040184704460D464E1D00E023689B68204698470028F9D0236868
:20CD400015F8011B1B6820469847B542F1D170BD0A44914217D010B40139541E11F8013F3B
:20CD600008225840430010F0800F08BF400083F0D50314BFD8B2C0B2013AF3D1A142EDD15E
:20CD80005DF8044B704770472DE9F047164D0746002095F9BD9505F2C45684B007EB010844
:20CDA00005F6640504464FF0B60A3368ABB193F83830142B11D019F1020F01D04B450CD163
:20CDC000002269463046CDE90244CDE90078ADF808A08DF80D4034F051FAE036B542E4D192
:20CDE00004B0BDE8F08700BF305E00202DE9F0479AB0DDE9226ADDF8909004460D4617461E
:20CE0000984602E0206844F021F8206844F026F80028F7D10146642201A860F052FD264B2D
:20CE20008DF80450CDF85CA00293002D40D0AB1E012B3FD9042D14BF002203221F4B03962B
:20CE4000D3F884308DF805201E440123CDE9059404968DF85B3037B14246394607A860F03C
:20CE6000CFFC8DF85A80164E96F8A69800231893B9F1000F19D196F8A508642202FB0060C9
:20CE800001A900F6A80060F0BBFC012386F8A59886F8A638236843B143463A4629462046AB
:20CEA0001AB0BDE8F04712F01FBC1AB0BDE8F0870522C3E70222C1E794660020482B0020BF
:20CEC000305E00200C480D4BD0F8281910B40C4CC0F818398A1E2231B0F846391B01A4FBED
:20CEE00003C3DB08A3F5B06322F8023F9142F3D15DF8044B704700BF305E00203D8102085C
:20CF0000CDCCCCCC70B5084C251D2E4614F8010B34F01CFC28B1037805F8013BB442F5D114
:20CF200070BDFF23F8E700BF9C6700202DE9F0471D4F012607F10805B2464FF03C094FF041
:20CF4000000817F8010B44F017F8044690B180F80690C671FB7803F07F02012A18D013F09E
:20CF6000800F20460DD185F8048044F0E9FA85F805802C600136052E05F10805E1D1BDE874
:20CF8000F08785F804A044F0E1FA85F805A0F0E71B0605D40121204642F0A4FDFB78DEE764
:20CFA00044F0D4FAF6E700BFA46700202DE9F04FDFF8FC91DFF8FCA183B009F10C06012417
:20CFC00019F8018BB8F1000F00F0C6804FEA1815013D042D08F00F0200F2C1800AEB450378
:20CFE000B3F8840040FA02F717F0010700F0D28001239340013B184055445EF069F995F81D
:20D000009030664F184407EBC00704237761FC71BB71002302E0152B00F09E8003EB430268
:20D020005F49895C41454FEA430B03F10103F2D15C4B1A4492F84512002900F0AD804046E9
:20D0400040F0ECFC0546284640F008FD0378002B40F08280534B5B44042283F8854283F8D2
:20D060008422002D78D0002F5DD03B68287A03F13F4202F57E020AEB92224FF0010C92F889
:20D08000982002F01F015209032A0CFA01F171D0042A67D0022A75D0B7F804E0BEFA8EF264
:20D0A000C2F11F02C2F3CC0103EB810102F007020F6A92004FF00F0C0CFA02FC27EA0C0722
:20D0C0000F620F6A90403843002208624FF0010B11460BFA01FC3CEA0E0001F101011ED1D4
:20D0E00018680327974020EA07001860D3F800800220904040EA08001860986820EA07002E
:20D10000986098689860586820EA0C00586058685860D86820EA0700D860D868D8601029DF
:20D1200002F10202D5D1204B204AB3F89C19B3F89E390091002001340190B2FBF3F330461B
:20D140009BB22946E4B232F0E1FD0123092C737406F118067FF434AF03B0BDE8F08F0027D4
:20D16000776156E7DFF850C0DCF830200A43CCF8302091E7DFF840C0DCF840201143CCF893
:20D18000401089E7DFF830C0DCF844201143CCF8441081E777613CE70D4654E7F82D00202E
:20D1A0008C2D0020482B0020305E002040420F00D067002064D90608003802402DE9F04161
:20D1C000214E224F96F86F3A87F8083F06F66C2607F60C7500244FF0050816F8010B20BB01
:20D1E00028600134032C05F10405F6D197F8081FD7F80C0FC94301F0010144F0ADF997F875
:20D20000081FD7F8100F81F00201C1F3400144F0A3F997F8081FD7F8140F81F00401BDE8FD
:20D22000F041C1F3800144F097B943F0A5FE013401212860E3B210B180F80680C371286837
:20D2400042F050FCCEE700BF305E0020482B00202DE9F0412A4C2B4DB4F8746AA5F8186FB8
:20D2600082B0EEB994F8700A43F086FE94F8712AC5F81C0F003A18BF012285F81A2F48B116
:20D2800094F8721A2B22002914BF11210121C28042F028FC002002B0BDE8F04144F064B948
:20D2A00094F8708A002240462B2140F00FFC0746404643F061FEF8B1F7B12B22C5F8340FB6
:20D2C000C280397AFCF78EFE4FF000080E4AB2FBF6F3C3F34F0000909BB23946CDF80480FB
:20D2E00005F57260A4F8766A32F010FDD5F8203FC3F8008085F8318F02B0BDE8F08100BF8C
:20D30000305E0020482B002040420F002DE9F84F254C94F8843A84F8783A04F67B27002633
:20D3200004F698245FFA86FB0BF101085FFA88F8012117F8010F42460E448A4640F0C6FBA3
:20D340004FF00009054640B3387804F80E9C04F80D9C04F80FBC04F810AC44F8045C43F0FE
:20D360000BFE18B180F806A080F80780297AFCF739FE0E4A0021284640F0EEF90C4B236019
:20D380000C4B221D21462846C4E9013940F0F2F8697928684A4632F035FC082E04F11C0481
:20D3A000C0D1BDE8F88F00BF305E002040420F003DFC030875DE030870B52C4C2C4B94F870
:20D3C000B00BC4F8A83B00220221C4F8682BC4F86C2BC4F8702BC4F8A42BA4F8AC2B40F087
:20D3E00075FB002841D0234B0268054603F1C000597C11B159688A422BD018338342F7D1B6
:20D40000002394F8B00BC4F8945A84F8883A43F0B3FD08B10223C380297AFCF7E3FD2846D2
:20D42000154A002140F098F9144A1549C4F8981A0026111F2846134BC4F89C3AC4F8A06A07
:20D4400040F098F8697928683246BDE8704032F0D9BB138D0C490D4A9BB2D2F8302501332B
:20D46000B2FBF3F381F82833CAE770BD305E002000FFFF00CC2C002040420F00CC680020BE
:20D480009DDE030839E0030898010020482B00202DE9F04FC14FC24C85B08B460546C022F0
:20D4A00007F5C2700021CDF808B060F00AFA94F81C3C002B00F0DA8094F81D3C002B00F0F3
:20D4C000F48097F87031012B67D0022B00F0F980B44BB54E03931D460FCE0FC50FCE0FC552
:20D4E00097F866C197F8623196E80700AF4EC4F8006CBCF1000618BF0126072B85E8070053
:20D5000084F8256C00F22A81042B00F26381DFF8C0A20026AAF1120B029BB3424FF0030170
:20D5200039DD1BF8019B07EB090309F1010893F867515FFA88F82846424640F0C7FA0346D9
:20D5400028461D46002B00F0218143F015FDCAF8140020B14FF00303837180F8078097F88A
:20D56000632197F86231F1B2002A00F00D81EA7982F00102009228464A46013658F050FC87
:20D58000002800F003814FF00103082E8AF811300AF1180AC0D1039B66E0854E029BC4F8F5
:20D5A000283C0FCE834DDFF828920FC50FCE0FC596E8070097F8663197F8626184F8686CF7
:20D5C00000269B1B85E8070018BF012305F1980031464FF44C7284F8253C84F8266C60F0BF
:20D5E00070F9A9F1120305F57275B2460393D4F8283C534540F3AA80039A12F8013B039207
:20D600003B4493F86761304642F014F98046304643F0B2FC97F863310646002B00F09880C4
:20D6200098F8073083F0010B0BF0010894F8252C08F1010884F8248C0AB18BF0010B002E25
:20D6400000F09380B279002A59D0412A57D05A4B5A495B4AC4F8D03B012384F8263CC4F845
:20D66000CC1BC4F8D82B0023C4F8203CD4F8203C63B10022029883F82C00012183F82D1050
:20D680001A6383F82E2005B0BDE8F08F4D4E4E4D0FCE0FC50FCE0FC596E80700A5F1200395
:20D6A00085E80700C4F8203CEDE797F864210299003A284618BF0122FBF718FAC4F8200CCD
:20D6C000D4E797F86631002B3FF402AF97F86231082B7FF462AF344EDFF8D0C00FCE04F6C1
:20D6E000E83503950FC50FCE0FC596E80700012385E8070084F8253CC4F800CC31E03046E7
:20D7000043F088FF4FEA48180AF1010A48F009014FF0030369616860EE6085F810B086F88E
:20D7200007A0B371304642F0DDF91BF0010F304611D043F005FFEB68C9F81430BAF1080FDD
:20D7400005F1200509F118097FF451AF194B8BE798F807B068E743F0F9FEECE7082B7FF411
:20D76000D6AE1A4BC4F82C3CD1E6304643F052FF4FEA481848F009010AF1010A6961686078
:20D78000EE6085F810B0CDE7EA79F3E60C4B0A4AC4F80C3CC4F8042C002365E7482B002071
:20D7A000305E0020186A002054DA06083137060880DA0608E46900206DE0040871E00408DC
:20D7C00065E0040828DA0608646A0020E1E00408CC2C002097F86531064AC4F82C2C012B60
:20D7E00005D0022B06BFBCFA8CF35B09002384F8303C8CE611E104082DE9F0416E4F97F8BB
:20D80000400997F8415943F0B7FB60B12D23C3802021044642F066F90A2042F093FD20469F
:20D8200043F0EEFE28B9DFF8988158F85C3CDA0001D5BDE8F081013D092DFAD897F83F49ED
:20D84000D4B940203DF066F80028F2D090F9043097F81119092BC8BF143B43440A2913F821
:20D86000584C00F09B8013F84C3C97F83E29002A08BF1C46002CDCD0204643F07DFB0546E9
:20D88000002800F083802D23C380012142F02AF90121084643F09AFE2B68AA881A833C206A
:20D8A00042F06EFE0021012043F090FE97F84139002B4CD0414C00261FE02B68AA885A8323
:20D8C00042F040FD94F8081FD4F80C0F01F0010143F042FE94F8081FD4F8140FC1F3800102
:20D8E00043F03AFE2B68AA881A83782042F02AFD97F8413901369E4229DA94F8081FD4F8C8
:20D900000C0FC94301F0010143F026FE94F8081FD4F8140F81F00401C1F3800143F01CFEFC
:20D920007820002DC9D1782042F00CFD94F8081FD4F80C0F01F0010143F00EFE94F8081F36
:20D94000D4F8140FC1F3800143F006FECDE797F83F399BB9D7F8403903F0FF13B3F5803FA9
:20D960007FF467AF58F85C3C13F080537FF461AF87F84139BDE8F0414BF0D8BA322042F0BD
:20D98000FFFD2846002142F0ADF8E3E7012142F0A9F80121084643F019FE80E758F8343C85
:20D9A0005B057FF546AF09F0FBFC00287FF441AF002C7FF461AF3CE7305E0020482B002010
:20D9C000286F0020084B53E90C02904253F8283C02DC114602460846984204DD9A42B8BF99
:20D9E0001A46104670477047286F00200B6810B414681B1B036054684B681B1B43608B68C5
:20DA000092685DF8044B9B1A836070472DE9F047041E0D4612DB092C26DC824A0B4682484C
:20DA2000A0FB0410C00800EB8000A4EB40000021125C1A7059702846BDE8F08764422D23D3
:20DA4000092C01F8013B24D8764A774BA3FB0403DB0803EB8303A4EB43030020D35C487006
:20DA60000B702846BDE8F0876F4B632CA3FB04264FEAD60621DC6B4A0B466B49A1FB060121
:20DA8000C90801EB8101A6EB4101515C03F8011BC5E7654A632CA2FB04364FEAD60637D8CB
:20DAA000604A614BA3FB0603DB0803EB8303A6EB4303D35C01F8013BC7E7A3FB0627B4F5B5
:20DAC0007A7F4FEAD7070DD2564A0B465649A1FB0701C90801EB8101A7EB4101515C03F868
:20DAE000011BCAE7A3FB072842F20F7294424FEAD80836D84B4A0B464B49A1FB0801C908EA
:20DB000001EB8101A8EB4101515C03F8011BDDE7A2FB0637B4F57A7F4FEAD7070CD2414A3E
:20DB2000414BA3FB0703DB0803EB8303A7EB4303D35C01F8013BB4E7A2FB073842F20F73F1
:20DB40009C424FEAD80821D8364A374BA3FB0803DB0803EB8303A8EB4303D35C01F8013B96
:20DB6000DEE7324AA3FB080994424FEAD90921D82C4A0B462C49A1FB0901C90801EB8101AA
:20DB8000A9EB4101515C03F8011BB5E7274BA2FB08099C424FEAD90921D8224A224BA3FBC6
:20DBA0000903DB0803EB8303A9EB4303D35C01F8013BCAE71E4AA3FB090394424FEAD30A15
:20DBC00021D80B461849174AA1FB0A01C90801EB8101AAEB4101515C03F8011BCAE7144BA8
:20DBE000A2FB09029C424FEAD20A13D80E4B0D4AA3FB0A03DB0803EB8303AAEB4303D35CE3
:20DC000001F8013BCAE70A22BAFBF2F04AF07EFF0346D7E70A22BAFBF2F04AF077FF0146E3
:20DC2000E4E700BF045C0708CDCCCCCC9F8601003F420F0070B4334810F8243CA3F1300138
:20DC4000092956D8A0F124042246153812F8015FA5F13001092904D88242F7D1002070BCDF
:20DC60007047141B022C4ADD2748002101E010F8013B01EB810103EB4103161A303B022E49
:20DC8000044603F0FF01F2DC204B03FB01F1A2424FF000030DD903EB830314F8016B5B00CB
:20DCA000303B3344A24203F0FF03F4D1184800FB03F32E2D06D01748A0FB032301EB9300C3
:20DCC00070BC7047013204200024157804EB8404303D6400092D00F1FF30A4B202D82C441B
:20DCE000A4B2013210F0FF00EFD1642202FB0433E1E700211D46A0F124020B46D9E7064CBC
:20DD00000021C4E7286F0020056F00208096980040420F00ABAAAAAA046F002038B504463A
:20DD20000D460A460068FF215FF0CBFD21682944216038BD83B50C46164605463BF096F84B
:20DD400020463BF093F80021204B0846002E08BF1E4643F03BFC0021012043F037FC2846F4
:20DD600043F07CF8B0B10121002043F02FFC284643F06CF80746204643F06CF80028FAD0BA
:20DD80003946204643F06EF83846B0470021084643F01CFC204643F061F80028DFD00121EB
:20DDA000002043F013FC204643F050F801462846019143F04FF801990028F8D0284643F034
:20DDC00051F80021084643F001FCC8E7694C0408F0B50023C1E90033C1E902330B61026891
:20DDE000DFF888C089B004ADC2F385572E4647FA03F0C007344604D513F80C0004F8010BA8
:20DE000026460133062BF2D1164CDFF864C0C2F303200023205C33708DF81800C2F3053769
:20DE20000DF1190647FA03F0C007344604D513F80C0004F8010B26460133062BF2D10023A1
:20DE40003370C2F3834406ABCDE90134084602F00F0305490095C2F303124DF0A1FA09B077
:20DE6000F0BD00BF445C07082C5C07084C5C07083C5C070870B5094C54F8142C054662B12E
:20DE8000002654F8140C2D21013644F063FCAE42F7DBBDE8704049F02DBB70BD286F0020BC
:20DEA0002DE9F04F5FFA81F9002185B007460846164643F08BFB0021012043F087FB42F00B
:20DEC000FBFF022E0AD0042E44F6C01818BF4FF49648B9F1070F07D900200CE0B9F1FF0F9E
:20DEE0004FF41648F5D10326BE4D15F8103C2BB9002045F80C0C05B0BDE8F08F032EBA4CC5
:20DF00000DD0A144002299F8670103213FF0DEFD0028EDD0C4F87805C3799A07E8D415F832
:20DF2000100C84F8936D002203213FF0CFFDC4F87C090028DCD0AD4AAD4BC4F8343502F1EC
:20DF4000480003234FF48061A4F83835C4F84805002302F24C404FF0010A032EC4F83C8582
:20DF6000C4F86035C4F84015C4F85435C4F85035C4F84C05C4F84415C4F85C35C4F8583501
:20DF800084F8843DA4F880ADC4F88C3DA4F8903D84F8923D91460ED0D4F878B59BF80400FD
:20DFA00042F0EAFFC4F87405584614F0C3FB5146484614F0D3FB322042F0E2FA012E09D151
:20DFC000D4F87C094146FAF783FFD4F87805FEF781FE0AE0022E3BD1D4F8780514F099FB32
:20DFE000D4F87C094146FAF773FF45F80C9C4FF0060A022E11D055F80C0C42F02FFF60B1CB
:020000040800F2
:20E000000121002043F0E2FA55F80C0C42F026FF014600287FD143F0D9FA384642F01EFF61
:20E0200080B10121084643F0D1FA4FF0050B4FF00008384642F012FF0146002874D1012015
:20E0400043F0C4FA042ED6D0052042F099FAD0E7032E58D14FF0000A5146664884F894ADB1
:20E0600040225FF02EFC8DF80FA04FF0010A9DF80F30072B09D95D48012114F06FFBD4F85E
:20E080007C094146FAF724FFAFE79DF80F3003EB430304EBC30393F895316BB39DF80F30CA
:20E0A00003EB430304EBC303D3F8983123B39DF80F30234493F86701F0B1002203213FF0C9
:20E0C00005FD8346C0B114F024FB9DF80F3094F8942D03EB430304EBC30305EBC201D3F859
:20E0E000983141F8083C9BF807300132DB0748BF01F804AC84F8942D9DF80F300133DBB279
:20E100008DF80F30B3E7042E7FF46FAFD4F8780514F0FFFA54E755F80C0C42F097FE0146EA
:20E12000384642F09FFE6FE7384642F08FFE95F8463001468BB9242803D14FF0010385F891
:20E140004630012E04D13846019142F08BFE019955F80C0C42F086FE6BE7012B06D14D28FB
:20E160000CBF0223002385F84630EAE7022B06D13C280CBF0323002385F84630E1E7032B63
:20E1800010D10A2802D985F84680DAE7042385F8390085F8388085F83B8085F83A0085F80F
:20E1A0004630CEE7042B09D195F83A3085F84700434085F83A3085F846B0C2E7052BC0D129
:20E1C00095F8383095F8399095F83A004B4513D25A1C2B44484085F83A0085F8382083F844
:20E1E0003C10AEE7286F0020482B00207C300020ACDA0608206F00208842C4D195F8473082
:20E2000085F846A0F42B9CD1B9F1000F99D12421384685F8469042F025FE4D21384642F063
:20E2200021FE3E21384642F01DFE4946384642F019FEF421384642F015FEF421384642F0A2
:20E2400011FE032E1BD0D4F87805437901689D080223AB40DB439BB20B828D892B408B81EB
:20E260000079202114F044FAD4F878054A4649463FF080F9D4F87835186806F033FC002252
:20E28000D4F87C0911463FF075F9D4F87C39186806F028FC01202EE630B583B04D1C0093D5
:20E2A00003688572C2729C690023A04703B030BD03685B6C0BB102211847704770B51C4C65
:20E2C0000968E56C1B4EA46CD6EDCB7ADFED1A6A491B00EE901A0168F8EEE00A091B60EE04
:20E2E000A70A00EE101A20EEA07AB8EEC00A1C46A0EE007AB1EE400AF1EEC77A67EEA67AD5
:20E30000FCEEE77AC2ED007A4DF0E0FC9FED0B7ADFED0B7AE0EE077AFDEEE77A17EE902AB4
:20E32000002ABCBF02F50C42A032226070BD00BF286F0020980100202C7D8E3FA00CB34529
:20E3400000A00C4638B50F4C94F8671001F03F018B1C024601F10A0584F8653084F8625020
:20E3600004F1600084F8632008311EF03FFD254485F85E0094F862301C44000A84F85F001F
:20E3800038BD00BF286F002038B50B4C00250122802120463CF0AAFA30B194F904003CF011
:20E3A000D7FA08B1006838BD0135062D04F10C04EDD10020F7E700BFB06F002038B5041F3E
:20E3C00000F1080554F8043FD81780EA430016F039F9A542F6D138BDF8B5C94CDFEDC97A68
:20E3E00094ED357A94F83C31B4F83E712DED028BB8EE478A28EE278A002B5FD1D4F8483114
:20E4000094F85921002B40F30E8107EE902A9FEDBE6ADFEDBE6AF8EEE77AB7EE007AA7EEB7
:20E42000867AF0EE477A07EE103AF8EEC78AB7EE087A87EE270AC6EEA87A20EE270A5DF098
:20E440003BFF0F28B8BF0F2094F83D3185B2A4F83E51002B00F04781AF4234D0B4F8403154
:20E460009FEDAB6A94F8D86007EE103A07EE905AB8EE477AF8EE677AC6EE076A86EE277AB1
:20E4800076EE887A37EE087AC8EE276AC8EE077AB6B394F84231B4F84451C4ED3A7AC4ED32
:20E4A0003E7AC4ED427AC4ED466AC4ED4A7AC4ED4E7A002B5BD0BDEC028BF8BD94F83D31AD
:20E4C000002B00F0858094F8D860002E40F00381B4F84031DFED8E6A07EE907A07EE103A57
:20E4E000B8EE676AB8EE477AC6EE877A86EE867A77EE887A37EE087AC8EE276AC8EE077A89
:20E5000094F84261B4F844510023C4F8DC30C4F8E030C4F8E430C4F8EC30C4F8F030C4F894
:20E52000F430C4F8FC30C4F80031C4F80431C4ED3A7AC4ED3E7AC4ED427AC4ED466AC4EDA4
:20E540004A7AC4ED4E7AC4F80C31C4F81031C4F81431C4F81C31C4F82031C4F82431C4F8A4
:20E560002C31C4F83031C4F83431002E66D1D4F8483194F85921002B40F38E8007EE902A35
:20E580009FED616ADFED616AF8EEE77AB7EE007AA7EE867A07EE903AF8EEE77AB7EE086A75
:20E5A00086EE070A86EEA77A20EE070A5DF084FE0F28B8BF0F2080B2A4F84401002E3CD029
:20E5C000A8423FF478AF00286DD1BDEC028BF8BDD4F8483194F85A21002B40F3878007EE00
:20E5E000903AF8EEE78A3D4607EE902A9FED466ADFED466AF8EEE77AB7EE007AA7EE867A15
:20E60000F0EE477AB7EE087A87EE270AC6EEA87A20EE270A5DF050FE0F28B8BF0F2080B2CF
:20E62000A4F8400118E794F83D310F25A4F83E51002B7FF411AF2846F2E7054694F85831A0
:20E6400084F89534002D3FF436AF07EE905A9FED306AD4ED576A2F4BF8EE677ABDEC028B32
:20E6600086EE277A1946002241F8042B012084F894040A609A601A615A619A611A625A629A
:20E680009A6237EE267AC6EE877AC3ED037AC3ED077AC3ED0B7AF8BD0F20A4F8440146B3B3
:20E6A0000F2D3FF408AF07EE900A9FED196AD4ED576A194AF8EE677ABDEC028B86EE277A9F
:20E6C00037EE267AC6EE877AC2ED007AC2ED087AC2ED047AF8BD94F84231B4F84451002B19
:20E6E0007FF4E9AE43E794F85A217DE73D460F2096E794F8583184F895340546A5E700BF5C
:20E70000286F0020BD378635CDCCCC3D002474494E2DA63D8C730020987300201D4911F8F9
:20E72000242CA2B3F0B4002605463346304637461BB911F8244C2D2C23D02E2A19D0CA18F7
:20E7400000EB800012F8244CA4F13002092A4FEA40009CBFA0F13002A0180E2B14D8013332
:20E76000CA1812F8242C002AE2D106B14042F0BC70470133002DF8D0CA182A4402F8247CD1
:20E78000DDE701231E46EBE70020F0BC70470020704700BF286F00202DE9F0410C4F0124C4
:20E7A000A0231825E6B2FF2B0BDCC5F11B0103F10108D7F8E804DBB23246C9B2FFF76CFD47
:20E7C0004346013DEFD10134052CEAD1BDE8F081286F00201FB503AC8DF80C3000940023C9
:20E7E0008DF80D300DF0B8FB04B010BDF8B50546262027F059F9154C014610BBD4F8EC0450
:20E8000090F838301E3B012B02D894F8F9340BB142F028FB0E4F0026AE420ADBB4F81A358C
:20E820000133A4F81A350B4BD3F88430C4F82C35F8BD17F8011BD4F8EC0442F013FB0136B4
:20E84000EAE7002384F82835EDE700BF286F002022740020482B002010B58021044604F0B4
:20E86000E1FF2046002104F0DDFF2046BDE8104005F018BB2DE9F041B14C94F84335C4F83A
:20E88000300582B088465A2B00F2B980DFE813F0CC00B700B700DC00B700B700B700B700D7
:20E8A000B700B700B700B700B700B700B700B700B700B7000F01B700B700B700B700B7008F
:20E8C000B700B70033017400B700B7007400B700B700B700B700B801B7006201B700B70023
:20E8E0007C00B7000902B700B700B700B7005B00B700B700B700B700B700B700B700B700EB
:20E90000B700B700B700B700B700B700B700B700B700B700B700B700B700B700B700B70087
:20E92000B700B700B700B700B700B700B700B700B700B700B700B700B700B700B700B70067
:20E94000B700B700E40194F844359B0700F16982B4F84A35D4F84525D4F884155BBA9BB2B9
:20E9600012BAD0188842C4F89035C4F88C2503D904F018FF002854DB0020A4F87C05054665
:20E98000284602B0BDE8F08194F88835002B40F0FF8094F94035002B31DAD4F8783508461F
:20E9A0009B689847002840F01E82B4F84A05D4F84525D4F8843540BA80B212BA15189D42C3
:20E9C000C4F89005C4F88C2507D904F0EBFE002827DBD4F88C25D4F89005D4F88035D4F867
:20E9E0003C6503FB00F003FB02F20225B042C4F88C25C4F8900584F8885500F0CF8094F89B
:20EA000054355A1CD2B204EBC30305204FF40051042A84F8542583F85805C3F85C1500F0EE
:20EA2000A0814FF0FF35ABE7D4F83C35002BE6D1D4F8783508469B6898470546002840F045
:20EA4000D281A4F87C059BE73E4B002203F1120103F8012F8B42FBD13B4994F87E3594F8FF
:20EA6000540570250D7098424FF00C05CD7110D004EBC300013390F858558D70B0F85C05C2
:20EA8000DBB2042B40BA888114BF84F87E3584F87E2594F8473512229342A4F87C2598BFF1
:20EAA000A4F87C350025284602B0BDE8F08194F84435DA0700F13E81D4F8783594F84705C7
:20EAC000DA6901EBC10102EB81010A79531D834228BF0346A4F87C35002BE3D0013B1A4825
:20EAE0009BB201331944034411F8012D03F8012D8342F9D1D6E7154E154F35460823073E93
:20EB0000C5F10700A4F87C35002202E092F880211D462B46B54203F8012900EB030217FACB
:20EB200082F2F3D1D4F878354046DB6898470028B8D0AB7863F07F03AB70002520E700BFCE
:20EB4000286F002047970020489700204F97002064D90608D4F87835C74A5B680846111DE7
:20EB600098470546002840F03E81D4F88435C34AD4F88015013B180E1070180C09BAD37055
:20EB800050701B0A082093705160A4F87C05F7E6D4F89065D4F88C25D4F88035D4F8785562
:20EBA000B2FBF3F24FF48057BE4228BF3E462D69B249A4F87C754046B6FBF3F39BB2A847C7
:20EBC0000028C0F2BC803346AC4AD4F83005812104F05CFED4F88C25D4F89005D4F89C3544
:20EBE0003244851B9E1BC4F88C25C4F89055C4F89C65002D7FF456AF032384F88835BFE6D2
:20EC00009E4E0027334606F10C0203F8017B9A42FBD1D4F8783540465B686A4601A9984749
:20EC20000546002840F0E980019BBDF80020013B190E52BAF3713171190C1B0A717108208E
:20EC4000B371022172810C23BDF80220F07031727272A4F87C3593E6894E8A4F3046082376
:20EC6000073EC0F10705A4F87C35002202E092F8882118460346864203F8012905EB030285
:20EC800017FA82F2F3D1D4F878354046DB68984700283FF407AFF37863F07F03F370002531
:20ECA0006EE694F88835002B61D194F94035002BFFF6A5AED4F8783508469B689847002814
:20ECC00040F09180D4F878354046DB6898470546002840F0BA80B4F84A35D4F84525D4F8C8
:20ECE00084155BBA9BB212BAD0188842C4F89035C4F88C2500F29F80D4F88015D4F83C052E
:20ED000003FB01F302FB01F28342C4F88C25C4F890357FF474AEB3F5805F28BF4FF4805345
:20ED20000121D4F83005554A84F888159BB204F0D7FE25E607235449A4F87C35CEE694F883
:20ED400054355A1CD2B204EBC30304204FF48851824284F8542583F85805C3F85C157FF40B
:20ED600060AE002384F854354FF0FF3508E6D4F89065D4F87805D4F88035D4F88C25456946
:20ED8000B2FBF3F2B6F5805F28BF4FF480560846B6FBF3F339499BB2A847002862DBD4F883
:20EDA0008C25D4F89055D4F89C353244AD1B9B1BC4F88C25C4F89055C4F89C352DB9D4F813
:20EDC0003005294604F0E0FEDAE5B5F5805F28BF4FF48055ABB2D4F83005284A012104F090
:20EDE0007FFE0025CCE594F854355A1CD2B204EBC30302204FF468510AE694F8543504EBEA
:20EE0000C3020133DBB202204FF46851042B82F85805C2F85C1522D084F854354FF0FF35B3
:20EE2000AEE594F854355A1CD2B204EBC30305204FF41051ECE504F0B5FC0028FFF6F1AD81
:20EE4000D4F88C25D4F8903556E794F854355A1CD2B204EBC30302204FF41C51D8E584F898
:20EE60005475DEE594F854355A1CD2B204EBC30304204FF440716BE7A8740020489700209D
:20EE80004F97002064D90608DCDA060810B51C2042F072F81121044640F024FE204642F05A
:20EEA0004FFBC82041F06CFB2046BDE8104042F04DBB00BF08B5002042F05EF8054BC3F8C4
:20EEC000A40508B12A23C380BDE80840402140F009BE00BF286F00202DE9F04FB34C54F8E5
:20EEE000843C5A69D2078BB002D50BB0BDE8F08F5A699B6912EA030AF7D0CAF307431AF419
:20EF0000002F009340F00281009B5D0743D41AF0020F5FFA8AF503D054F8843C02225A61B5
:20EF2000BAF1000FC0F20C821AF4006FCAF3072740F082812E0708D59D4B9E48D3F83C3322
:20EF4000984754F8843C08225A61ED0600F1E481F80600F1A481B90600F12E81009BDA06AA
:20EF600009D5934B9348D3F84C33984754F8843C4FF480125A61009B9B06B6D58C4B8D48C2
:20EF8000D3F85033984754F8843C4FF400125A610BB0BDE8F08F54F8802C9369D2691340C7
:20EFA0001FFA83FBBBF1000FB1D0DFF80882CDF80CA045464FF0000909E05FEA5B0B09F147
:20EFC000010908F1040805F1280500F0D4811BF0010FF2D054F8801C5FFA89F708694A6BF6
:20EFE00004EB8703FA4053F8783CD2019B68D2B202431A40D007D3B216D54B6BD8F8182061
:20F00000012000FA09F023EA00034B63684B6948D3F83433012191603946984714F88D6C12
:20F02000012E00F0F58101231A0703D5D8F8182008239360DE0603D5D8F81820102393600E
:20F04000580603D5D8F8182040239360990703D5D8F81820022393601A06AED5D5E94C6077
:20F06000D5F82431D8F818C0311A8B42DCF8182028BF0B46033392B2B2EB930F9DD954F8EF
:20F08000802C323704EB8703CDE9019890469946B04238D2BEB3D5F8241114F88D3CD5F8CD
:20F0A0002821371AB94228BF394601F1030E4FEA9E0E83B98FB20337BF1059F888AC0AD088
:20F0C000013352F8040BCAF800009F42F8D1D5E94C60D5F82821DCF8183008440A44B0420F
:20F0E000C5F82821C5F834010AD195F81C11D8F83420012707FA01F122EA0102C8F8342021
:20F100009BB29E45C4D3DDE9019856E754F8803C9D69DB691D402D0C3FF4F6AEA4F19006A2
:20F12000DFF88CB0B046B146002708E06D0807F1010706F1040608F128083FF4E5AEEB0769
:20F14000F4D5F9B204EB810254F8803C52F83C2C92685B691A40D007D3B218D514F88D0C09
:20F16000726D01239842936007D11269D8F87C33C2F312029B1AC8F88C33DBF8303348462C
:20F18000984714F88D3C012B00F0508101239A0702D5726D022393601B07C7D5DBF838333F
:20F1A00048469847736D08229A60BFE7305E002098010020A05D002054F8803C54F8781CCC
:20F1C0009A680868C2F34102022A08BF03224FF0000514BF65F30A0062F30A0008605A68AB
:20F1E00042F480725A6006A805F02AFD54E92120D368BD49079D6FF38D23D3608068C0F320
:20F200004100014491F89011032900F0CA80B749B7480126294404F88E6C81424FF0400607
:20F2200024F88C6C00F210810E2161F38D234FF40051D360516191E6AE4B94F88220D3F822
:20F240004433AD4800218DF817108DF81720984754E9212114F8863C88684FF40061516147
:20F26000002B3FF467AEC3077FF564AE94F88530012B7FF45FAE9DF81730032B7FF45AAE59
:20F28000E36F9E491A6842F001021A601A6842F003021A600B6943F006030B614AE654F839
:20F2A000802C954853684FF0000823F001034146536005F023F914F88F6C414656B1904BF1
:20F2C000FF2203EB860653F8045FD86BAA609E428260F8D154F8803C87484FF0FF329A61CB
:20F2E0004FF00112DA610B2262F3070162F30708C3F8148019611A686FF30A121A6004F05C
:20F30000D1FD54F8842C7B4B7B48D3F840334FF48051516198471EE654F8843C9A6922F092
:20F3200010029A611A6AC2F34340022802F00F0142D0062822D09A6942F010029A6107E677
:20F3400014F8863C33B1E26F136823F0030161F30703136054F8802C66495368D1F84813C1
:20F36000654823F001035360884754F8843C4FF000425A61D8E5DDF80CA0C8E501EB8101A6
:20F38000256C04EBC1012E68D1F8FC02C4F83C65C2F30A1202442868C4F84005C1F8FC22F2
:20F3A000C9E700214FF4007004F88E1C092124F88C0C61F38D233AE747F6F0701042BAD0A7
:20F3C00001EB8100C2F30A1204EBC00002F1030C5FEAAC0CD0F8F052D4F840E04FEA810885
:20F3E00018BF002006D00130DEF8006045F8046B8445F8D1414404EBC101D1F8F052D1F891
:20F40000FC0215440244C1F8F052C1F8FC2292E7B9F1000F7FF407AE94F88130042B7FF444
:20F4200002AE354804F03EFD3346FDE5002F7FF4ADAE94F88120052A7FF4A8AE48460193D1
:20F4400004F030FD019BA2E62E48A5F57401A1F51051814203D80D2161F38D23E7E62A49DB
:20F460002A482944814203D20C2161F38D23DEE62748A5F18C71A1F54341814203D80B213A
:20F4800061F38D23D3E6234923482944814203D20A2161F38D23CAE62049214829448142F2
:20F4A00003D2092161F38D23C1E61E48A5F1B771A1F55851814203D2082161F38D23B6E6DE
:20F4C00019491A482944814203D2072161F38D23ADE6174917482944814234BF0621052175
:20F4E00061F38D23A3E600BF64D90608401E1BFF3F420F0098010020A05D002000ED00E0CA
:20F50000B45D0020DFC810002013FBFE20D61300FF69180000D3CEFE40771B00C05BB3FE11
:20F52000C091210040AC2700C01D6AFE40E13300803C36FEE09C4100704700BF704700BF14
:20F54000704700BF704700BF2DE9F0414FF0FF35324A33482C46002304E001330B2B02F138
:20F56000100215D0917A0429F7D103F5B17100EB0111C979CF07F0D4661C116801D0A942EA
:20F58000EBD21C4601330B2B0D4602F11002E9D1631C02D10120BDE8F081214D04F5B177B8
:20F5A00005EB07139988F1B9DFF880802601AB19D8F86C251B4916691B4A41F2186001EB74
:20F5C000442118580023B047D0B1022808D141F2CC6205EB0717AB58013B0121AB50B971C3
:20F5E0000020BDE8F081DFF8448005EB0413D8F86C2541F21860D268185826019047D6E7C2
:20F6000041F2CC6205EB0717AB580321B97141F2D061013B0124AB506C54BCE714D40020FF
:20F62000F8BD002010BE002049F60008305E0020044B41F2E472995C09B901219954012251
:20F640005A707047F8BD002038B5174D174B41F2D0640020285504E001300B2803F110034E
:20F6600014D053F80E4C8C42F6D11C78032CF3D16AB10F4B03EB40239A4201D0FFF7D8FFA5
:20F6800000F5B17005EB00100123837138BD41F2CC6100F5B1736A5805EB031304200132AF
:20F6A00098716A5038BD00BFF8BD00201ED4002010BE002038B5134B00209C7B14B11D6832
:20F6C0008D4205D001300B2803F11003F5D138BD72B10D4B03EB40239A4210D0FFF7A8FF3B
:20F6E0000A4B00F5B17003EB00100123837138BD064B00F5B17003EB0010827138BD022C19
:20F70000ECD1EDE710D4002010BE0020F8BD00202DE9F84F12F0020E9B4606D028B9FFF794
:20F7200087FF02252846BDE8F88F804C41F638056559002D5BD14FF0FF367D4FB146B046FE
:20F74000B24600253B68984200F0B68097F80EC0BCF1000F5BD0BCF1010F15D105F5B17CDB
:20F7600004EB0C1C9CF807C01CF0010F0CD11CF07E0F09D15FEADC1340F0A880D7F808C084
:20F78000D44501D2E246A94601350B2D07F11007D8D1751C04D1B8F1FF3F00F09F80464658
:20F7A00041F2C86806F5B17754F80850013544F8085004EB061C41F21C694FEA07184CF8F0
:20F7C000095044F8085041F2186904EB07154FF000084CF80900C5F8048004EB0715AD7977
:20F7E000042D9CD8DFE805F01A330F334D0004F5C25741F63C063F68A65907FB0565A84245
:20F8000099D3FFF715FF00252846BDE8F88F2E4601350B2D07F1100794D1BAE712F0010CAD
:20F8200070D104EB0710D51090F80780BBF1030F65F3C71880F8078062D94FF6FF708345E2
:20F840005B4628BF03469BB204EB07108380BEF1000F16D004EB061303F5B0531833987B7C
:20F8600004280ED041F2C8654FF0040C60590130605141F2CC65586083F80EC063590133DF
:20F880006351500705D504EB0710C37943F00103C371D30608D504EB0714E379C3F34502BD
:20F8A000013262F34603E371224B012503EB46260E602846BDE8F88F05F5B17704EB071600
:20F8C0004FEA071CB67986B92E4669E7A84601350B2D07F110077FF435AF5AE7B9F1FF3FAF
:20F8E00018BF4E467FF45CAF8DE741F2C8682E4654F80850013544F8085044F80C506CE77B
:20F900006346A1E70C4B0B49D3F86C350B4AD3F8088001EB46210023C04700283FF473AFFD
:20F9200004EB07140223A371FCE600BFF8BD002010D4002010BE0020305E0020B5F60008BB
:20F94000F0B5124D2B7841F63002022B0BBF070AC0F3D417C4B200F07F04A85883B00E4681
:20F9600000230122384401A9FFF7D2FE01280AD12B78022B019B16BF53F8243033F8143002
:20F9800023F07043336003B0F0BD00BFF8BD002010B5144602070B4610D50B4941F2C472FF
:20F9A000581C8B58834204D305D100232360012010BDFFF73DFE2060012010BD2146184686
:20F9C000BDE81040BCE700BFF8BD00202DE9F0414268C2F308030B44B3F5007F82B0044658
:20F9E0000D4657D390F91A30591C0AD0304A03F5B17302EB0313FF21DA796FF30002DA71AD
:20FA0000817694F91B305A1C0FD0294A03F5B17302EB0313FF20DA79C2F34501013921EA7E
:20FA2000E17161F34602DA71E0762378022B37D01F4A02F5C2531B68B5EB432F4FEA4328BA
:20FA400024DC41F648036768D6583E407342AB421CDCAB19434511D32169207E01AAFFF716
:20FA600097FF012812D16768236963614744019B2361A5EB0801BF1B67608D192046F8F7E5
:20FA8000B9FD20B93D446560012000E0002002B0BDE8F08115444560012002B0BDE8F081C1
:20FAA000616801202944616002B0BDE8F08100BFF8BD002070B5154604460E46FFF786FF39
:20FAC00050B994F8280028B9022384F82830C4E90B5670BD022070BD1DB12046A8470120C1
:20FAE00070BD012070BD00BF10B4D0E9011390F91A208B4238BF0B46511C83600AD0144BDA
:20FB000002F5B17203EB0212FF21D3796FF30003D371817690F91B305A1C0FD00C4A03F546
:20FB2000B17302EB0313FF24DA79C2F34501013921EAE17161F34602DA71C4760022436AA6
:20FB40005DF8044B4261426011460361B2E700BFF8BD002038B54422002111485DF0B1FE0B
:20FB6000104B41F602011A784FF6FF745C52022A41F2E87118BF032203F5C05041F64C05B4
:20FB80005A5441F60C0441F6010203215D5900F8181910211D519954FFF7A6FF012038BDF6
:20FBA000E0D50020F8BD00202DE9F041B1F904300F2B82B00C461646054632D02846F8F7B2
:20FBC0003DFD95F91B80B8F1FF3F074633D02D4B41F2186203EB08118A58904211D118337E
:20FBE00003EB4823A188013109B203EB4113A18028463360F8F722FD2060012002B0BDE82C
:20FC0000F081FFF715FD2846F8F7F4FC28B100230120336002B0BDE8F081002002B0BDE82F
:20FC2000F0814FF40071FFF7D1FE0028F5D04FF6FF73A380C2E72846F8F7DCFC0028E2D15A
:20FC40000FB9FFF7F5FC38460023112201A9FFF75FFD0128D7D1019B0B4A9A1A48BF02F2B4
:20FC6000FF12B2F5B05F4FEA622106D24FFA81F885F81B80002BB5D1C5E7FFF7D9FC019B8B
:20FC8000F6E700BFF8BD002010BE002030B50446C06983B010B9012003B030BD0D4600237A
:20FCA000032201A9FFF734FD0128F5D1B4F92030002B03DAFFF7BCFC0220EDE7019A012DED
:20FCC0004FEA431102EB431303D0022D12D1E5255554A268DA612278032A04D100221A7728
:20FCE0005A779A77DA77626A5A83C2F30F429A8203B030BDE268DA61EDE700BF10B503780E
:20FD0000023B012B0446037E02D913F0060F5AD198063AD494F91A30591C0AD02D4A03F550
:20FD2000B17302EB0313FF21DA796FF30002DA71A17694F91B305A1C0FD0264A03F5B173AA
:20FD400002EB0313FF20DA79C2F34501013921EAE17161F34602DA71E076237E1B070BD5BC
:20FD60001C4841F2C873C35C072B01D0FFF760FC41F2C8730022C254E26A0023237084F819
:20FD80002830FAB1BDE81040104700231249E0691A018A58904206D001330B2BBAD01A0199
:20FDA0008A589042F8D10B4A03F5B17302EB0313DA79C2F34501013921EAE17161F34602D1
:20FDC000DA71A7E710BD0121FFF760FF0128F9D1237E9DE7F8BD002010D4002030B10278BA
:20FDE00022B190F828201AB1002070470120704710B5D0E90142A242C16238BF224603219B
:20FE0000826080F82810FFF779FF012010BD00BF2DE9F04FDFF868918A4699F80010DAF8CD
:20FE200000300229174683B0834641F6300240F08B8059F80250DEB2A6EB030805EB132573
:20FE4000B8444FF480729044BB4208F1FF38B8FBF2F875D2A844032906EB0704A4EB0304E2
:20FE60000CBF80224FF48072944228BF1446A8EB050366B994422CBF0A220B2201A92846DD
:20FE8000FFF746FC012809D003B0BDE8F08F0B2201A92846FFF73CFC0128F5D199F800203E
:20FEA000DAF80010022A01F1010321D0A64210D2019906F18042013A081F00EB840001EB73
:20FEC000820242F8043F824203F10103F9D1DAF80010A61B7318BBF1010FCAF800301BD0D4
:20FEE0009F4205F101052BD999F800100026B2E7A642EED2DDF804C006F10042013AACF16F
:20FF0000020000EB44000CEB420222F8023F904203F10103F9D1DCE7BB42E1D199F8003053
:20FF2000022B21D004F18044019B013C4FF0FF3243F82420DAF800309F4205F10105D3D898
:20FF4000012003B0BDE8F08F59F8022003F07F060329C3F3D415A6EB03081544B84414BF2F
:20FF60004FF4807280226EE704F10044019B013C4FF6FF72584623F8142003B0BDE8F08FC9
:20FF8000F8BD00202DE9F04190F838300446032B51D8DFE803F002323B462D4BC068197814
:20FFA000E76A03F5C252032911680CBF80264FF4807601FB06F141F2C47C00EB412041F2B0
:20FFC000A87841F2AC7E53F80C20E06053F80E0053F808502261A5EB4125A0EB41219019E2
:20FFE00043F8085043F80E1043F80C00C4E90C205FBB6262012384F8383016480021FFF79A
:020000040801F1
:2000000045FE012811D1022384F83830626B04F130010120FFF7FCFE012806D1032384F8E3
:20002000383000212046FFF731FE431EDBB2012B02D9BDE8F081022094F82830062B04BFA7
:20004000002384F82830BDE8F081921B2263D1E7F8BD002098D500202DE9F04FDFF8248176
:2000600098F80060012887B08CBF00230123032E02930C460B68154639D0022E62D14FF409
:2000800080724FEA1329DFB201920138012823D8012203929D421AD9384E06F1880A06F1E8
:2000A0001C0B32681AB1DBF8001099424ED0DAF8000000234844092205A9FFF729FB01283B
:2000C0001FD002280FD020B123689D42E9D82560032007B0BDE8F08F87B1FFF7A9FA0220B6
:2000E00007B0BDE8F08F022007B0BDE8F08F80220192C3F3D41903F07F07C6E7019A0392FA
:20010000C8E7DDE902C1059ADDF804E098F80030022B14D0032BE6D152F8273023F0704332
:20012000B3FA83F35B0963450F44236823D00B4477452360EAD309F101090027C5E732F873
:200140001730EDE74FF480720192D2E70C490968013A02EB41224902B2FBF1F203991344E4
:20016000B3FBF1F201FB12320AB10B449B1A9D42236096D8ABE7AB42ABD3A8E7A0D50020FE
:2001800038D60020F8BD0020F0B5104D2B7841F63002022B0BBF070AC0F3D417C4B200F042
:2001A0007F04A85883B00E4600230322384401A9FFF7AEFA012807D12B78022B019B0CBFF1
:2001C00023F8146043F8246003B0F0BDF8BD00202DE9F04390F83C30002983B0044614BFE6
:2001E00002210021042B7BD8DFE803F0030C3C476900FFF74BFD012870D1626B002A75D19F
:2002000084F83C00404EDFF80881404D4FF6F7771DE01FFA80F9B94594BF4FF000094FF091
:20022000010901A9B9F1000F46D1FFF789FB0128494650D1206BFFF7A7FF01284BD1019BDF
:200240002A682363013B934228BF13462B603378206B032BDDD1404594BF4FF000094FF039
:200260000109DEE7426B04F130010020FFF7D0FD012833D1032384F83C30234BE16A41F2D2
:20028000C47003F5C2521D581268195041F2A87741F2AC76D8596D1A995902FB05F200EB96
:2002A000422501EB422203F5BD500021DD519A51FFF7ECFC012811D1042384F83C3094F8C4
:2002C0002830042B04BF002384F82830A36B8BB120469847012003B0BDE8F0830228FAD16D
:2002E00094F82830042B09D00220F4E7022384F83C30B8E7012003B0BDE8F083002384F8DE
:2003000028300220E7E700BFF8BD00203CD60020F7FFFF0F38B590F834300446052B46D85A
:20032000DFE803F01F033F101963006B4FF0FF31FFF72AFF01283AD1E06A002839D1032347
:2003400084F8343000212046FFF7A0FC01282ED1042384F8343094F82830082B2DD0012040
:2003600038BD41F63803224DEA5800F1300102320120FFF771FE012824D00238C0B2012897
:2003800015D8052384F8343094F82830082B04BF002384F8283041F2E5730122EA54022089
:2003A00038BDC06A216BFFF7EFFE0128C7D0002038BD022384F83430F4E7002384F8283003
:2003C000012038BD05F5C252E3681168D4E90B2003EB412341F644016850C4E9033002B92C
:2003E0006062012384F83430A0E7014DCCE700BFF8BD00202DE9F04F436883B0C3F3080822
:200400001646002A00F0E180714B05468946A3F1180B4FF0000AC8F5007495F91A70B442F0
:2004200028BF3446791C28462ED0F8F707F90BEB071341F218629B58984205D0FFF7F8F826
:20044000504603B0BDE8F08F614B03EB47202246494640445DF0D4F9002221462846FFF7AC
:2004600029FBA2440028EBD02B7E1B0706D5594B2A691B689A4201D3FFF7DAF8361BA14481
:200480004FF00008C7D1DBE7F8F7B4F8002849D12846F8F7D3F86968C1F308032BBB21F42B
:2004A000FF7323F0010303F50072AB689A422CBF062207222B7E03F00C030C2B1CD000232D
:2004C00001A9FFF725F90128BAD10198404BC31A48BF03F2FF13B3F5B05F4FEA63224FD205
:2004E00057B2AF760028B2D1AAE72B7E03F00C030C2B4FF00702E2D19BF800C0364BBCF134
:20050000030F1B680CBF4FF0800C4FF4807C03FB0CF34FEA432C0CF1FF3C0CEA0101A3EB0E
:200520005123CDE72B7E1A072ED59BF800102A4B95F828201B6803290CBF80214FF480718A
:2005400003FB01F3062A4FEA43233FF479AF23490868834230D891F83D30002B7FF470AF23
:20056000002A7FF46DAF6B6985F83820062185F82810EB622846FFF705FD012888D05FE7C3
:20058000FFF756F80198ACE7154B1A78002A7FF457AF95F82820002A7FF452AF082185F83D
:2005A000342085F82810D3F85F206B692846C5E90B32FFF7AFFEE0E741F2E573012250460D
:2005C0000BF8032003B0BDE8F08F924638E700BF10BE0020BCD5002038D60020A0D5002006
:2005E000DDD500202DE9F04390F8384083B00546032C00F29F80DFE804F0021A890BFFF7C1
:2006000089FE012811D002280BD1032385F838302B6C002085F82800002B00F087809847DB
:200620000224204603B0BDE8F08385F838002B78022B77D0404A6F6841F64803D3581F402A
:20064000C7F34F272846F7F7F9FFDFF8F08006463F1A0AE0D8F80030013B99454AD2FFF714
:20066000B5F908B9FEF7E4FF0136022201A900233046FFF74DF8BC1901281FFA84F94FF483
:2006800000724FF000010446CBD101985DF019F9EB694FF400712846002BDBD06B68002B80
:2006A000D8D1019B4FF020324FF02E0C1A605A6083F800C0C3F807204FF0100E6C6A1A62EB
:2006C0005A6283F820C083F821C0C3F8272083F80BE0EA6B5C83C2F30F4CC4F30F4483F876
:2006E0002BE09C825A87A3F834C0D8F80030013B9945B4D3C3EBC35359022846FFF766F9DE
:2007000008B9FEF795FF022385F838302B6C002285F8282063B1284698470124204603B068
:20072000BDE8F0836F68C7F34F278BE7022478E7012476E7002474E7F8BD002038D600209F
:200740002DE9F04F90F8303089B00446042B00F2A880DFE813F0A900B20005008A00E800F4
:20076000B64D41F61003EB5C002B40F09A80B44F04F11C09B84607F1380BBA4601AE3246F3
:2007800049464046FFF710FA012840F018810198002800F0FA800378E52B01D0002BEED1E1
:2007A000A84A821A48BF02F2FF12B2F5B05F4FEA622380F03C811B01A34A13449A7B042A5B
:2007C0000CD041F2C86104266A5801326A5041F2CC615A609E736B5801336B5041F60202F0
:2007E000AB565E1C09D003F5B17305EB0313FF26D979AE546FF30001D97141F603016B5661
:200800005A1C0ED003F5B17305EB0313FF26DA796E54C2F34501013921EAE17161F34602FA
:20082000DA71202200215DF04CF82346019A53F8311F58685060116019899B7A93721181AB
:20084000019B627EDA7205A848F0B2F9BDF81430002B40F02F8144F28172019903200A82CA
:20086000CB810A83CB8284F83000237E980600F1A9802046FFF738F92369002B00F0AE80EB
:20088000237E03F0F70213F00403227640F0B480122A00F0BA80002384F828302046E36AB5
:2008A000984709B0BDE8F08F6548FFF71DF94FF6FF720123228484F83030614F04F11C089E
:2008C00001AE04F13109324641463846FFF76CF901282FD00228E4D1584D41F60202AB567A
:2008E000591C09D003F5B17305EB0313FF20D979A8546FF30001D97141F603016B565F1CF7
:200900000ED003F5B17305EB0313FF20DA796854C2F34501013921EAE17161F34602DA7130
:20092000042384F830300020E36A2070984709B0BDE8F08F019D0B2249462846002D00F016
:2009400087802B78002B00F0838095F80BA01AF0080FB8D15CF0E1FF0028B4D1637E8AEABF
:200960000303DB0640F1C780344D41F602016B565F1CC1D003F5B17305EB0313FF26DA79F6
:200980006E5460F30002DA71B6E73B782F49022B4FF009025046C3D00B78002BC0D1C1E9A4
:2009A00005330A708BF800304A6B0B7351F8143CC1E90132FFF716FE01283FF4E0AE02280B
:2009C000AED06EE7E0690023112205A9FEF7A0FE01283FF44EAF09B0BDE8F08F237E19076D
:2009E0007FF559AF154A41F2C873D15C00297FF458AF0721D1544EE70023E26AA16884F868
:200A000028302046FFF756F84BE7626AE06AA0630421C4E90233C4E90B2284F83C306363FA
:200A200084F8281063622046FFF75EF839E7FEF7FFFD01986FF00F03BEE600BFF8BD002038
:200A4000E0D5002010BE002010D4002008D60020474D41F60202AB565E1C09D003F5B17392
:200A600005EB0313FF20D979A8546FF30001D97141F603016B56581C0ED003F5B17305EBFC
:200A80000313FF20DA796854C2F34501013921EAE17161F34602DA71237EDA067FF540AFB5
:200AA0003448FFF721F84FF6FF720223228484F8303056E6304B05A9B3F9A82502A848F08E
:200AC00095F89DF80C309DF80D609DF80A509DF80B20BDF808109DF80E00DB0243EA461334
:200AE00042EA4512A1F2BC7143EA500342EA41229BB292B2B1E6A98A6B8B204A43EA014378
:200B000012686362EB69A3605202B3FBF2F102FB113109B113445B1A154DE36041F60201B6
:200B200084F819A06B565E1C09D003F5B17305EB0313FF20DA7968546FF30002DA7141F636
:200B400003016B56581C0ED003F5B17305EB0313FF20DA796854C2F34501013921EAE1719C
:200B600061F34602DA71032384F830307DE600BFF8BD0020E0D50020286F002038D60020DB
:200B80002DE9F04390F82830013B83B00446082B41D8DFE803F048054D525865406A4300D7
:200BA000384B4668056B41F6480103F5C2525F5813683740EA19B2EB432F4FEA432816D2C1
:200BC00058E02169207EFEF7E3FE012823D1256B666823696361A5EB08053D444644F61B5B
:200BE000019B6660A84525634F46236142D82046F7F700FD01AA81460028E2D06668A36875
:200C0000E26A9E4238BF1E460023A66084F828300AB12046904703B0BDE8F083FFF7E2FCB9
:200C200003B0BDE8F083FFF78BFD03B0BDE8F083FFF764F803B0BDE8F0830021FFF7C8FAAA
:200C400003B0BDE8F0830121FFF7C2FA0128E2D10023216C84F828302046FFF7BFF8DAE7C1
:200C6000FFF790F903B0BDE8F083FFF753FB03B0BDE8F0832046F7F7BDFC0028BFD12E44E4
:200C80006660BCE7F8BD00202DE9F04782B0054602AF18461C460E4690465AF0C1FA083074
:200CA00020F00700ADEB000D0DF1080A013CD14614F8013F5BB989F800304246CDF800A016
:200CC0003146284640F072FFBD46BDE8F087184647F016FEC3B2A3F120023F2A88BF2023A8
:200CE00009F8013BE4E700BF2DE9F04704460D469046002144221E46089F5CF0E2FD01238C
:200D00004FF6FF722676628384F828302B782E2B4CD02E4604F1310A307804F1390968B114
:200D20002E280BD047F0ECFDC0B20AF8010BCA4506F1010607D030780028F1D120200AF82A
:200D4000010BCA45F7D130782E2808BF707804F1380908BF013604F13B0A58B147F0D0FD88
:200D6000C0B209F8010FD14506F1010607D030780028F3D1202009F8010FD145F7D118F03A
:200D8000100F14BF0323012384F819802370E7622B782E2B26D16B7823BB0323204684F86A
:200DA0003030FFF7CDFC2046BDE8F0876B78002BAFD1114B41F2F47241F60C0041F2F07138
:200DC0009A5818585958E26041F601026062A1609A5C627641F2E8729B5C2370E7622B78F0
:200DE0002E2BD8D00023204684F83030FFF7A8FC2046BDE8F08700BFF8BD002010B5104CBC
:200E000014F8863C23B90F4B4FF480225A6110BD0D4A136823F0060313605AF0CDF914F8E4
:200E2000863C002BEFD054F8803C9B68DB07EAD5E26F136823F0030161F307031360E2E7DD
:200E4000305E0020003C014010ED00E008B50121032003F041FD72B64BF0B2F82DE9F04FF5
:200E60008DB0CF4CDFF84C93CE4D00904FF0000854F80B0C002800F0FE803FF0EFFF064610
:200E8000002800F0DB81D9F8843044F8073CE0260023C54F04F8033CA4F10B0B06FB08F6B8
:200EA00054F80B0C3FF0DAFF002800F0E48054F80B0C3FF0CBFF14F8023C5A1E82460B2A30
:200EC0000DD8DFE812F01F003A004600530083009B00E30017013701420179019101242886
:200EE0000CD0009A3AB995F8D220824240F08281012204F8032C0D2BD2D186E0012304F864
:200F0000023CCDE700234D28C4F8C53084F8CD3084F8CE3004D0582808D004F8023CBFE797
:200F2000022204F8022C84F8C430B9E7032304F8023C022384F8C430B2E704233C2804F83E
:200F4000023C0BD0BAF13E0F0CD0002304F8023CA6E70A233C2804F8023CF3D1002304F80C
:200F6000013C9DE7012304F8013C99E7D4F8C500BB190344421CC4F8C52083F8CFA594F8AD
:200F8000CD00022A8AEA000184F8CD1088D12378C02BDAD86278FF2A08D1052BD5D901231B
:200FA00084F8C430072304F8023C79E7A4F8C12000229342C4F8C93014BF0523062384F834
:200FC000C320C4F8C52004F8023C69E7D4F8C500BB190344421CC4F8C52083F8CFA594F8DD
:200FE000CD00D4F8C9308AEA00019A4284F8CD107FF456AF062304F8023C51E794F8CD3019
:201000008342A2D10D2304F8023C14F8017C002F40F0F680654B08940FCB04AE86E80F007B
:20102000D4F8C930D4F8D100ADF82A7023440993B4F8C130ADF8283094F8C3308DF82C3012
:2010400001238DF82D30324603AB08A9039730F0C7FB48B1049B059394F8C420544B049361
:201060003146584630F00AF9039E002304F8023C002E40F0DB8008F10108B8F1030F04F1CF
:20108000E0047FF4F5AE0DB0BDE8F08FD4F8C500BA190244431CC4F8C53082F8CFA594F841
:2010A000CD2094F8CE0001938AEA020284F8CD205146D52247F0E2FD019B84F8CE00072BB8
:2010C0007FF4EEAEB4F80530C02B3FF63EAFB4F80320A4F8C120A27884F8C3200022934257
:2010E000C4F8C93014BF08230923C4F8C52004F8023CD5E6D522014694F8CE0047F0BEFDF1
:2011000094F8CD3084F8CE008AEA0303D4F8C50084F8CD30BB190344421CC4F8C52083F8E3
:20112000CFA5D4F8C9309A427FF4BAAE092304F8023CB5E694F8CD30434084F8CD3094F8AD
:20114000CE3083427FF401AF54E7D4F8C500BA190244431CC4F8C53082F8CFA594F8CE006C
:201160000193D522514647F089FD019B84F8CE00052B7FF495AEB4F80120B4F80330A4F87C
:20118000C120227884F8C32000229342C4F8C93014BF0B230C23C4F8C52004F8023C7FE659
:2011A000FF630020286F0020305E0020F8DA060878A00120482B0020D522014694F8CE0004
:2011C00047F05CFD84F8CE00D4F8C500BB190344421CC4F8C52083F8CFA5D4F8C9309A42FA
:2011E0007FF45EAE0C2398E694F8CE3083427FF4ACAE07E7232804BF022204F8032C7AE6FC
:20120000012F4FF0000602D004F8026C33E7D4F8C93008942344099308A8B4F8C130CDE99C
:201220000A66ADF828302DF0EFFDEDE754F80B0C37F01CFE54F80B0CB0471CE714F8033C18
:20124000002B3FF418AFD9F8842054F8071C521A632A7FF610AF012B29D0022B7FF40BAFD9
:2012600054F80B3CC5F8AC350122C5F8B035C5F8B835402385F8AA2585F8BD050D4A0E4833
:2012800085F8BC350D4BC5F8B42545F8143CC5F8003646F033F94FF400503AF0FBFA08480E
:2012A00046F020F985F8046685F80566E3E6FFF7CDFD00BF09E004085C5C0708DC7400209C
:2012C000925C0708202301480B807047F4040020642301480B807047140500204323014831
:2012E0000B8070477805002010B5074CD4F8C800FF2807D0054951F8042BF7F7A3F8FF23F4
:20130000C4F8C830002010BDF404002050D60020EAE700BF08B5D0F8E4355B6A98470020DC
:2013200008BD00BF08B5D0F8E4351B6A9847002008BD00BFD0F8E43510B504461B68984731
:20134000D4F8E8359B689847002010BD08B5D0F8E435DB6903B19847002008BD08B5042298
:2013600090F81211D0F8E83580F8131180F81221DB689847002008BD10B5D0F8E83504469B
:201380001B699847032384F81231002010BD00BF0B0630B41CD401EB810200EBC202002333
:2013A00000EB810582F8741382F8753301241A4604FA01F16D6D61F31F4201696FF3CF33C7
:2013C0002B60CB6923EA0203002030BCCB61704701F07F0101EB810400EBC404012200EBAA
:2013E0008105002384F81C1184F81D2102FA01F11A46AD6961F30F02DFE700BF10B581212C
:201400000446FFF7C5FF20460121FFF7C1FF024B0020187010BD00BFB074002010B581215E
:201420000446FFF7B5FF20460121FFF7B1FF82212046FFF7ADFFF7F74DF8002010BD00BF00
:2014400038B50D4604468321FFF7A2FF29462046FFF7E4FF002038BDF0B416460A063AD4E6
:2014600001EB810500EBC5052824002204FB0104022B85F87413C5F87C6385F8773385F862
:20148000752304F55D7448D0154600EB8107012202FA01F17F6D61F31F45D7F800C01CF4B0
:2014A000004F11D1E488204946F0805242F4004242EA834204F00F041C4B42EA84521140F4
:2014C0000CEA0303194339600269D3692B430020F0BCD361704701F07F0101EB810500EB81
:2014E000C5052824012204FB0104022B85F81C11C5F8246185F81F31A5F8221185F81D213E
:2015000004F58E740CD0002500EB8107012202FA01F1BF6961F30F05BFE722711546B4E78C
:2015200000252571F0E700BFFF87CC13007833EC002310B5194604464022FFF78DFF802148
:20154000204600234022FFF787FFD4F8E835A078012284F812215B689847002010BD00BF03
:2015600070B44B78012B26D00B784A6900EB83035C6D25682369D2B18A684A6102F07F0246
:2015800023F4002323F07F0342F4002213432361C378012B04BF0B696361C5F3076363F073
:2015A0007B0363F31F652560002070BC70478A6802F07F02E4E782694C691568136944B38B
:2015C0008E68B4428CBF06F07F0404F07F0423F4002323F07F0344F4002443EA040388BF3E
:2015E0004E611361C378012B1DD0C5F3076464F07B0464F31F651560002BD5D14B69002B7E
:20160000D2D002690878516B012383400B435363CAE723F4002323F07F0343F40023136148
:20162000C378012BE1D10B780C6900EB8300C5F30763816963F07B0363F31F654C610020A7
:20164000156070BC704700BF2DE9F0434B78012B30D00B784C6900EB83035E6D356837698A
:201660001CB38B681C44013CB4FBF3F4C4F3090203FB02F3C3F312034B61144643EAC443BB
:2016800063F31C073761C378012B04BF0B697361CB78012B44D0C5F3076363F07B0363F3FB
:2016A0001F6535600020BDE8F0838A680124C2F31203E3E791F800804E6900EB880EDEF817
:2016C00018C0DCF80050DCF8107076B3D1F80890384A06EB0904013CB4FBF9F402EAC444E3
:2016E000C6F312022243CC7807F060473A43012C174649D0CCF81020C278012A55D00269CD
:20170000516B03FA08F30B435363C5F3076363F07B0363F31F65CCF800500020BDE8F083F8
:201720004B7973B345F00055B5E707F0604747F40027CC78CCF81070C378012B2FD0012C7E
:20174000E3D102699268D20554BF45F0005545F08055C5F3076262F07B0262F31F65CCF865
:201760000050002B9ED1B0B203308010DEF8D04098D0CA6852F8041B216001339842F9D118
:2017800090E745F0805586E764F35E77CCF81070C378012BD5D10A69CCF81420D1E70A6948
:2017A000CCF81420012CB0D1CBE70B69CCF81430ABE700BF0000F81F0E4BDA68D20310D499
:2017C000DA68D1060FD4DA68D20510D4DA6812F0E00F0AD1DB6813F0020F14BF0820092087
:2017E00070470120704706207047072070470220704700BF003C024000207047104AD06820
:20180000A8B113699BB188420FD88B4234BF00230123DBB243B193695161994204D0094BBD
:201820009161142083F8CC0070470023F1E7A1F59C53083BB3F57A7F2CBF00230123E9E71E
:2018400050D60020F4040020054B5A7F19778A4204D0044A5977142082F8CC00704700BFC3
:2018600050D60020F4040020704728B1034B987F012894BF00200120704700BF50D600209C
:2018800008B5FFF7F2FF50B1054AD37F127F5B0003F00203002A18BF43F001030B6008BDB6
:2018A00050D6002008B5FFF7E0FF10B1014B1B6A0B8008BD50D6002070B5FFF7D6FF50B137
:2018C0000A4A958C35B1966A0023B3421C4603DB002000E00D7070BD02EB44040133A48D11
:2018E000AC42DBB2F1D10B70F5E700BF50D6002008B5FFF7BAFF10B100230B70137008BD3C
:201900000420704728B1034B93F9CE00003818BF01207047F404002008B5FFF7F3FF50B1C6
:20192000054B93F9CE20012AC3BF93F8D130C3F340030B60002008BDF404002008B5FFF790
:20194000E1FF18B1024B93F8D0300B7008BD00BFF404002070B5FFF7D5FF38B10E4C94F831
:20196000D130DB0703D500230B70137070BD0B4D94F9CF3095F83C6093FBF6F301330B702B
:2019800094F9CF4095F83C1094FBF1F301FB134301331370EAE700BFF404002050D6002068
:2019A0000320704770B50A4A92F8403006255E1CB6FBF5F405FB146492F84150AC4205D045
:2019C00002EBC303C3E9110182F8404070BD00BF50D60020002230B504461046914200DC14
:2019E00030BDA35C0825584010F0800F4FEA400318BF83F0D503013DD8B2F5D10132EDE774
:201A000010B5D9B10E4B586F814217DCB2B1DB6B9A4213DC0B4C013A013903FB012184F8C5
:201A2000DC1004F1D8000521FFF7D4FF062184F8DD0004F1D800BDE81040B3E710BD00BF96
:201A400050D60020F40400200023038083708380C3800381704700BF074A084992F878307B
:201A600009780133DBB2994282F8783004BF002382F87830704700BF50D60020785000207B
:201A8000F8B5794CE36F83B1784B1B6893F82E305BB1774B94F88020A3FB0013012A4FEA10
:201AA000931330D0022A08D002B1F8BD714B9842FBD9012384F88030F8BDD4F8842064329F
:201AC0009A423ED894F8783004EB031393F8F824FF2A06D068490132012083F8F82481F820
:201AE000DE00FFF7B9FF654B1B780122092B84F88020DAD1B4F87A35614A01339BB2A4F8D6
:201B00007A355380F8BD94F878105C48C4F884308C2303FB0143007883F89A20002384F829
:201B2000963004F18C050A2202230928C4F8885084F8972084F88030B7D1514B01311980F5
:201B4000F8BD94F8962094F897309A42ADD104F18B0004F19405002310F8012F08215340BC
:201B60005A0013F0800F08BF5B0082F0070214BFD3B2DBB20139F3D18542EDD194F8952033
:201B80009A4239D194F8786094F8935094F89430B4F88F00B4F8912094F88DC004EB0617BF
:201BA00043EA052394F88E5087F8F81440BA52BA81B292B245EA0C202F4DC7F8FC141BB2EB
:201BC00094F98C10C7F80025032E4FF00102A7F8FA04A7F8043587F8F91485F8DE2008D829
:201BE000264A12780C2A29D00D2A02D1244B23F81610FFF731FF5CE794F8783004EB031360
:201C000093F8F824FF2A06D01B490132012083F8F82481F8DE00FFF71FFF184B1B7801224B
:201C2000092B84F880207FF440AFB4F87835144A01339BB2A4F878359380F8BD1149124AF3
:201C400091F822100E4803EB830303EB830349089B0093FBF1F382FB0312DB17C3EBA20356
:201C600020F81630C5E700BF50D60020506A0020D34D62103F4B4C00F4040020404A002051
:201C8000484A0020A82C0020676666660B4B93F8961093F8972091420ED010B493F8962086
:201CA000D3F88840511CD2B2C0B2C9B283F89610A0545DF8044B7047704700BF50D6002087
:201CC000FD2870B522D0F02804D0EF2822D00224204670BD114D0320052641282E444FF054
:201CE000000405F1010580F080030DD0042B0BD9FFF7E6FF2044B542C4B2E9D015F8010B83
:201D0000412880F08003F1D10420F3E7044D0B200426E2E7034D0C200626DEE7D45C07088C
:201D2000DC5C0708CC5C07080E4BD3F88025B3F97C05530707D400EB8000400080B200F528
:201D4000C87080B27047084B084AD3F8C430323382FB0312D817C0EBA20080B200F5C8706C
:201D600080B2704750D60020283C00206766666600B5062983B00A464FF03203014628BF0E
:201D800006220DF101008DF800305BF039FD044B6846D3F88435984703B05DF804FB00BFC0
:201DA00050D600205E2810B511D05D2805D00D4BBDE81040D3F8883518470A4CD4F8883544
:201DC0009847D4F888353D20BDE810401847054C5D20D4F888359847D4F888353E20BDE828
:201DE0001040184750D6002070B5094E0546D6F888355E200C469847D6F888352846984715
:201E0000E0B2FFF7CFFFC4F30720BDE87040C9E750D6002003682DE9F041002B3D4D3E4F4F
:201E20003E4EB8BF5B42A5FB0321890D07FB0137C7EB0717BF0096F8923585FB0725FA17CD
:201E40000446C2EBA555002B57D101EB810101EB810105EB810109B2DFF8BC801320FFF7F9
:201E6000C3FF2F4908FB057581FB0531ED17C5EBA11109B21B20FFF7B7FF2368254D002BC9
:201E8000B4BF53214E212320FFF7AEFF636896F8922583EAE376A6EBE376A5FB0631890DD9
:201EA00008FB0168C8EB08184FEA880885FB08354FEAE873C3EBA5552ABB01EB810101EBE2
:201EC000810105EB810109B21220FFF78DFF124B134903FB058581FB0531ED17C5EBA11146
:201EE00009B21A20FFF780FF6368002BBDE8F041B4BF57214521222076E7C1EB011105EB0E
:201F0000810109B2A8E7C1EB011105EB810109B2DAE700BF6BCA5F6B806967FF50D60020F6
:201F2000D34D621030B40023022515244FF4167140F2D93205808471018130BC4281438033
:201F400083808381704707B50DF1060210F00CF968B1084BBDF80620B3F8B0159A84914254
:201F600005D00549A3F8B025142081F8CC0003B05DF804FB50D60020F404002013B50446DE
:201F8000FFF7C0FC08B300230DF106022046ADF8063010F0E9F8C0B10D4C9DF8062094F977
:201FA000CE1084F8E320032908BF62F07F024FF00501084808BF84F8E320FFF70BFD0621FE
:201FC00084F8E4000348FFF7EDFC02B010BD00BFF4040020D305002008B5044BD3F8B40599
:201FE0003EF03CFFB0FA80F0400908BD50D600202DE9F04F204B85B04FF0000804461E2046
:020000040801F1
:2020000093F800A093F801B09D78B3F80490DF881E7ACDF80480ADF80C8023F045FD18B16E
:2020200017B1B9460125C246144A92F8B835D9070AD492F8BF253AB9012E1BD0022E03D199
:2020400013F0020F08BF01258DF80C608DF804A08DF805B08DF80650ADF80890ADF80A70F4
:2020600001AB03CB1B88206020466160238105B0BDE8F08F3546E7E71874002050D60020E4
:20208000144B30B4D3F8E44514B300220F2583F8EA15090A83F8E90583F8EB15C3F8EC25AF
:2020A000C3F8F025C3F8F42583F8E85503F5BD60012110F8015F01312A440E29D2B2F8D101
:2020C00083F8F6252046044930BC10223EF096BE30BC704750D6002038DC0020034B00218B
:2020E00083F8F815C3F8FC15CAE700BF50D6002013B504462620019123F0D6FC019920B994
:20210000204602B0BDE81040BAE702B010BD2DE9F743B74CD4F8E4350D464BB14FF00208C2
:2021200000264FF00109D4F8E4053EF097FE58B90027A37F042B00F25781DFE813F08F000C
:20214000E400F7003D014601D4F8E4053EF07EFED4F8FC355A1C2344C4F8FC2583F8000688
:2021600094F8F835012B0AD0022B11D0002B70D10F280CBF84F8F895C4F8FC35D3E7A0F1E3
:202180007203012B01D9762863D184F8F885CAE7102AC8D197490023012211F8010F013203
:2021A00003440E2ADBB2F8D194F80E2684F8F8659A42C4F8FC65B6D194F80F36002BB2D1B2
:2021C00094F80176732F37D0762F0DD0722FAAD194F8032694F8023653EA0223A3D0E36024
:2021E000B4F804362361A4E794F8032694F8023653EA022397D094F8051694F8042694F8BF
:202200000906236242EA012294F80616E17794F8071684F8121694F80816A4F8102641EAE7
:202220000021A4F81416616901B96361A38C002B7FF47FAFA2847CE794F8072694F806366A
:2022400043EA02231AB2002B3FF46DAFA4F816266FE784F8F865C4F8FC6564E7722F44D1C1
:202260000123A3770022644B1B78402B2FD1634E94F812C6A08CA37FB4F810E63380050292
:202280004FEA0C33217F778005F4706503F440532B434FEA0E1543EA8133EDB22B43276A8E
:2022A00065691BB2BD4214BF0825002513432B43704514BF042000201843514B614514BF5F
:2022C0000221002193F8CC30F3800143B180636F1BB1A36A002B40F09D804A494A481F22C2
:2022E00003B0BDE8F0435BF02ABBD4F81836474AEB1A934201DC0022B5E77220FFF7EEFE8F
:20230000C4F81856F7E7762F03D10223A3770022A9E7D4F818363D4AEB1A9342EBDD762072
:20232000FFF7DCFEC4F8185600229CE7344ED4F8183696F8CC20EB1A82B3344A934230DD4E
:20234000E27FD2071BD46169226A91420ED089B24620FFF7CDFE96F8CC30C4F81856013BFB
:2023600086F8CC300423A37701227CE7A18CB4F810268A4203D05020FFF7BAFEEBE7217FDE
:2023800094F812268A4206D0B1FA81F149094920FFF7AEFEDFE7142286F8CC201C4A9342BC
:2023A000BDDC762FA7D17320FFF798FE0323A377C4F81856002256E7732F9CD0D4F8181677
:2023C000124B691A9942A0DC95E7D4F818360F4AEB1A93428FDD7620FFF780FE0223A37748
:2023E000C4F8185600223EE70023A3771A463AE750D6002050DC0020404A0020484A0020C0
:20240000F4040020975C0708D90500203F0D03003F420F00334DD4F81C662A2385F8E53018
:202420000DF1020220230DF10101304685F8E6300FF031FF30B19DF801109DF8027051EA56
:20244000070339D1552385F8E730462385F8E830202301A9304685F8E9300FF016FF034608
:20246000214813B1BDF804209ABB204948F098FFB4F814761E4D87B30DF1030130460FF077
:2024800007FF50B39DF803100DF1060230460FF06BFE10B3BDF8062016493B46BA420CBF62
:2024A00020222A22284648F07BFFB4F81636A4F8203603B0BDE8F08330460FF0D1FE3946F6
:2024C00085F8E70030460FF0B7FE037885F8E830BEE7094948F064FFCAE70849284648F024
:2024E0005FFFE2E7F4040020DE050020B95C0708E2050020B15C0708CEE80708B85C07086B
:2025000038B50B680E4D5A1C0A6005221A700B6895F8CE200C46591C21601A70236895F897
:20252000D120591C21601A70B5F8D410204645F0CDFF236895F8D620591C21601A7038BDAF
:20254000F40400202DE9F0472DED028BFFF7DAF9C8B31E4B93F9CE00012834DD93F804415E
:202560001B4F9FED1C8A15468E1E02EB44084FF03209454504D1BDEC028B2046BDE8F087EE
:2025800037F802AB26F802AF07EE90AAF8EEE70AB2EE040A60EE880A59F06AFFBCEEC00AD6
:2025A000BAF10E0F10EE103A9BB209D91933B3FBF9F39BB203EB830303EB83035B009BB219
:2025C00025F8023BD5E70024D5E700BFF404002072DC0020CDCCCC3D38B50D46FFF792F95D
:2025E000044638B10C4890F8D130DB0704D5B0F8D2002880204638BD084A90F9CF3092F82F
:202600003C2093FBF2F102FB11320132013100F584700FF0BDFDECE7F404002050D6002075
:2026200038B5134C94F8413094F840209A4219D004EBC3030F49D3E911200023984212DCBB
:2026400093780D4AC4F834065B081370FCF7CEF894F8413006210133B3FBF1F201FB123359
:2026600084F8413038BDD55C01F8015B0133E5E750D6002022740020507400202DE9F04FBD
:20268000A94B1B788BB08146002B40F0B580A74ED6F81C56002D00F0AF80A54AD2F80C419A
:2026A00004F0F021B1F1E02F6BD1C2F80C31D6F83826944265D004930593ADF818309D4BF6
:2026C000C6F838469A881F78ADF8142093F801C01A7A93F802A08DF810700DF110088DF87F
:2026E00011C08DF812A08DF8182098E807000DF11C0EAEE803009049AEF80020C4F34252E3
:20270000895CC4F303428F4202F101021F4601D1944508D028468DF81C108DF81D200FF049
:2027200037FDADF8200028460FF083FF032804F0070B33D0042835D000239A4501A9284632
:2027400018BF8DF81E300FF09DFD48B1019BC4F3001103F001038B4202D028460FF040FE98
:202760000A2207A940465BF084F850B19DF81E30BDF81C20BB703A80BDF82030BB8046F000
:20278000D5FB96F83CA6DFF8ACB104AF96F83C36032B7BD8DFE803F00A3376A3674B13F8C4
:2027A0000B30CAE7664B13F80B30C6E7394628460FF06EFD044658B107A8FFF719FC9DF890
:2027C0001E109DF810308B4260D028460FF094FE96F83C36013303F0030386F83C360CB918
:2027E0009A45D3D196F8B835DB0700D524B12B6849461B68284698470BB0BDE8F08F01A8D5
:20280000FFF7F6FB96F8B8859DF8044008F00108ECB1B8F1000F39D13A460DF103012846DD
:202820000FF039FD044688B307A8FFF7E1FB9DF81C109DF803309DF81D208B4203D19DF8CC
:202840001030934222D028460FF060FEC0E7B8F1000FBDD1394628460FF017FD0446A8B116
:2028600007A8FFF7C5FBBDF82010BDF810308B420CD086F83D8686F83E862B6828469B69E8
:202880009847A5E796F8B835D80701D500249FE707A928460FF0F6FC04460028F6D01E206E
:2028A00023F002F996F83F3683428046EED086F83F0660B1BBF80630002BE7D1079BD9079C
:2028C000E4D4012128460FF08BFD444680E7079BDA07DBD5014628460FF082FD78E73846F5
:2028E000FFF786FB97E8070007AB03C31A809DF810309BB10DF11D0207A928460FF0CBFCA7
:202900000DF11E0128460FF0C3FC0A2207A938465AF0AFFF041E18BF012459E708A928469F
:202920000FF0B3FCECE700BFD274002050D60020F404002018740020FC5C0708F05C070825
:20294000E45C0708024B0146D3F840063EF08ABA50D600202DE9F041FD2984B0044600F0F0
:20296000DD80F02900F0BC80EF2900F02F814AB10346861803AD002003F8010B9E4205F867
:20298000010BF9D1994B0B2003F1090501E013F8010F814200F0C780AB42F8D14B1E832B8D
:2029A00000F29280DFE813F03001370184004101AF01B501480153015F0190009000650131
:2029C000650165017B017B017B015F019000900086018E01900090009000900090009000C1
:2029E0009000900090009000900090009000900090009000900090009000900090009000D7
:202A00009000900090009000900090009000900090009000900090009000900090009000B6
:202A20009000900090009000A4019000900090009000900090009000900090009000900081
:202A4000900090009000900090009000900090009000900090009000900090009000900076
:202A6000900090009000900090009000900090009000900090009000900090009000900056
:202A8000900090009000900090009000900090009000900090009000900090009000900036
:202AA0009000900090009000900090001D011D014F4B93F89715002900F0628101922DF0FD
:202AC00087FB019AADF80C003AB1224403AB13F8011B04F8011BA242F9D104B0BDE8F08172
:202AE000444F03214FF00508B844002501370CE0FFF7E6F8064660193246FFF72BFF7019D4
:202B00004745C5B2E9D017F8011B412981F08003084601D0042BEBD80426ECE7364F0B21B1
:202B20004FF00408E0E7324BD3F8800580060CD4002AD2D0224403AB13F8011B04F8011B31
:202B40009442F9D104B0BDE8F08193F84406870741D52A4D287D052834BF022603261429C8
:202B600016D97C39C8B20628E2D80629E0D801A050F821F0592D0108592D0108432D0108D7
:202B8000312B0108692D0108632D01086F2D01080929CDD90A390A29CAD801A757F821F0FB
:202BA000292D0108752D0108312B0108312B0108312B0108312B0108312B0108312B0108AD
:202BC000312B01083B2D0108592D01080C4F0C214FF0060888E7094B0B29187DA8D101268F
:202BE000C9E0084BD3F8C03003936DE7C05C070850D60020D45C0708DC5C0708706F00203E
:202C0000CC5C0708283C00200192FFF78DF8019AADF80C0058E76A4BD3ED037AFDEEE77A22
:202C200017EE903AADF80C304EE701922DF0D0FA019AADF80C0047E7624D95F8B835DE07AD
:202C400000F1A780B5F86C36ADF80C303CE75D4B5D49B3F9E83681FB0301DB17C3EBA1032D
:202C6000ADF80C3030E7574BB3F8EA36ADF80C302AE7564BDFED566AD3ED007A0C39C9B2D6
:202C800003EB810393ED127A67EEA67A67EE877AFDEEE77A17EE903AADF80C3014E7494B60
:202CA00003EB4101B1F8C63603EB83035B00ADF80C3009E7434B93F8B83503F00103ADF8FD
:202CC0000C3001E73F4BB3F88816CD055ABFCB4303F00103032311F0440F18BF042311F094
:202CE000020F18BF072311F4806F18BF0923ABE70192FFF719F8374B019AD3F8C83043EA92
:202D0000C0400390E0E62F4BD3F87C36ADF80C30DAE62C4BB3F86C16002934D001922DF041
:202D20006FFA019A80B2CDE62B8A03EB830303EB83039B00ADF80C30FAE6EB89ADF80C305C
:202D4000F6E6EB89244903EBC3039B00A1FB03135B09ADF80C30EBE6B3F84636ADF80C3097
:202D6000E6E66B680393E3E62B680393E0E6AB680393DDE6F6B28DF80C608DF80D00D7E612
:202D8000B3F848069EE6D3F8840680F3100080B298E605F5CA65019222F0ECFED5ED037A37
:202DA000019AFCEEE77A17EE903A9BB200287FF44BAF0A49096811F0100F18BF002343E774
:202DC000A0DC002050D6002067666666DCDC002000007A44283C00201F85EB51F46E0020FC
:202DE00070B5214D95F8EC36EA181C4692F8F0268AB11E4E09225C1CA6FB04135B0803EB3A
:202E0000C303E31AE918DCB291F8F01609B1013AF1D185F8EC4602681549561C06600C2699
:202E200016700268561C0660002616700268561C066003EB430603EB8603147019440D221E
:202E400045F0FCFA95F8EC16084B4A1CA3FB02035B08294403EBC3030120D31A81F8F0065B
:202E600085F8EC3670BD00BF50D60020398EE3384CDD00202DE9F041684ED6F81C7684B0C5
:202E8000044638460D460FF0D4FB86F8710757B10DF1090202A938460FF0FDF9002840F0CC
:202EA0008E8096F871070023ADF808308DF80A301A46431EDBB20021FF20FD2B8DF80C20D8
:202EC000ADF80E108DF80B0003D9002004B0BDE8F0819DF80830042B00F09680052B00F0B7
:202EE0009980032B00F09880022B00F08C80012B08BF042100F088809DF809309DF80A10CD
:202F0000D6F81C06013B0DF10E028DF809300FF02BF996F87137032B73D0042B0CD1404A59
:202F20009DF80A000121002301E012F8011F81426DD20133082BF8D1D6F87427029B394FE2
:202F40009A420DF108084FD023680D22591C21601A7023680022591C21601A7023689DF8E1
:202F60000820591C21601A7023689DF80920591C21601A7023689DF80C20591C21601A7014
:202F800023689DF80A20591C21601A70BDF80E10204645F09BFA23689DF80B20591C216023
:202FA00020461A700721FAF7B9FE98E8030087E803000120C6F87C5704B0BDE8F08101A936
:202FC00038460FF05FF900283FF46BAF38460DF10A010FF05DF900283FF463AF019B96F834
:202FE000710703F0010264E77A68D8F804309A42AAD1D6F87C370C4AEB1A93427FF665AFA1
:20300000A2E70A4A8CE703218DF8081074E78DF80A3091E70121F7E70221F5E750D60020C8
:20302000E45C0708C4DD002080841E00F05C07082DE9F0412A4C2B4AD4F87C36B4F88077B0
:20304000B4F8846682FB0352DB17C3EBA2031FFA83F8474582B00D4603D1B4F88237B342F0
:2030600033D002680190511C34230160137002680023511C01601370414645F027FA019856
:20308000314645F023FA019847F6FF7145F01EFA019847F6FF7145F019FA019847F6FF7100
:2030A00045F014FA019847F6FF7145F00FFA01980221FAF733FE0120A4F88087A4F8826722
:2030C000C4F8845702B0BDE8F081D4F88437064ACB1A9342C5D8002002B0BDE8F08100BFBC
:2030E00050D600206766666680841E00026810B57F21541C0460117002680024511C01604F
:203100000E211470FAF70AFE012010BD2DE9F04FC24B1B68804613F0800083B000F07181D2
:20312000BF4B93F8440610F0020000F06A81DFF810B39BF81430052B40F26881DBF8003014
:20314000B84D0093002BB8BF5B42A5FB0342B648B649920D00FB0233C3EB03139B0085FB08
:20316000034502EB8202DC1702EB8202C4EBA55400FB043304EB8204A4B281FB0321DB17FB
:20318000C3EBA111BCB10025A94F2E46A7FB0432D20802EB8203A4EB4303E8B2A4469BB207
:2031A00080008340BCF1090F94B246EA030605F10105EBD8340489B2B9B100259C4F2E4668
:2031C000A7FB0132D20802EB8203A1EB4303E8B28C469BB280008340BCF1090F91B246EAC8
:2031E000030605F10105EBD83443DBF804E08D4D8D4E8E498EEAEE70A0EBEE70A5FB0032BC
:20320000920D06FB0200C0EB0010830085FB035002EB8202DD1702EB8202C5EBA05506FB7F
:20322000053305EB8205ADB281FB0321DB17C3EBA111C5B10020DFF8F8C10646ACFB05323E
:20324000D20802EB8203A5EB4303C7B2A9469BB2BF00BB40B9F1090F95B246EA030600F1AA
:203260000100EBD8350489B2C1B10020DFF8C0C10646ACFB0132D20802EB8203A1EB4303E8
:20328000C7B289469BB2BF00BB40B9F1090F91B246EA030600F10100EBD83543DBF8083069
:2032A000634A0193002B1846B8BF5842A2FB0030604E6149030AA6FB0363DB0901FB03F126
:2032C000C1EBD00189B2B9B1002691463746A9FB0132D20802EB8203A1EB4303F0B28C46E9
:2032E0009BB280008340BCF1090F91B247EA030706F10106EBD8B9B2BBF81070DFB10026E6
:20330000DFF82CA1B446AAFB0732D20802EB8203A7EB43035FFA86F938469BB24FEA89099F
:2033200003FA09F3092897B24CEA030C06F10106E9D81FFA8CF7BBF812303D4AA2FB030658
:20334000F608632E28BF6326092B63D9002093468146ABFB0632D20802EB8203A6EB43033D
:203360005FFA80FAB4469BB24FEA8A0A03FA0AF3BCF1090F96B249EA030900F10100E8D86E
:203380005FFA89F9009B019A002BCCBF392338231616BEF1000F26F07F0635DD274A334331
:2033A000964543F00206C8BF43F00606D8F800301622581CC8F800001A70D8F80030002219
:2033C000581CC8F800001A70404645F07FF82146404645F063F82946404645F05FF8404679
:2033E000394645F073F8D8F800305A1CC8F8002083F80090D8F800305A1CC8F800200120D6
:203400001E7003B0BDE8F08F1E43CFE7002003B0BDE8F08F4FF00009B4E700BFF46E002015
:2034200050D600206BCA5F6B806967FFD34D6210CDCCCCCCC55A7C0AA0860100FFC99A3BCC
:20344000706F00202DE9F047AB4B1B68064613F0800084B000F09E80A84B93F8440610F0CE
:20346000020000F09780A64F397D052940F29780632900F292800024DFF898C289B2254696
:20348000ACFB0132D20802EB8203A1EB4303E0B28E469BB280008340BEF1090F91B245EA05
:2034A000030504F10104EBD8EDB2BB68954A82FB0312D917C1EB623189B2002900F01881F8
:2034C0004FF0000CDFF84CE26446AEFB0132D20802EB8203A1EB43035FFA8CF088469BB208
:2034E00080008340B8F1090F91B244EA03040CF1010CEAD8E4B2FB8983494FF4F36707FBFF
:2035000003F7A1FB0737C7F38F1742F20F739F4249D8CFB10020DFF8FCE18446AEFB0732BF
:20352000D20802EB8203A7EB4303C1B2B8469BB289008B40B8F1090F97B24CEA030C00F115
:203540000100EBD81FFA8CF7704BD3E9002313433ED14FF0FF3833681722591C31601A7032
:2035600033680022581C306039461A70304644F0ADFF4146304644F091FF33685A1C3260C7
:203580001D7033685A1C326030461C700621FAF7C5FB012004B0BDE8F087992585E70020E6
:2035A00004B0BDE8F0870021DFF868C10F46ACFB0302D20802EB8200A3EB40039BB28B40E7
:2035C0000431102947EA030793B2F0D1BFB2BBE701A845F0EDFA9DF80810002900F08A8094
:2035E0004FF0000CDFF82CE1E046AEFB0132D20802EB8203A1EB43035FFA8CF089469BB28B
:2036000080008340B9F1090F91B248EA03080CF1010CEAD84FEA08289DF80910E1B1002090
:20362000DFF8F0E08446AEFB0132D20802EB8203A1EB43035FFA80F98A469BB24FEA890965
:2036400003FA09F3BAF1090F91B24CEA030C00F10100E8D848EA0C089DF80A104FEA082816
:20366000E1B10020DFF8ACE08446AEFB0132D20802EB8203A1EB43035FFA80F98A469BB282
:203680004FEA890903FA09F3BAF1090F91B24CEA030C00F10100E8D848EA0C08BDF80C3032
:2036A0001B49632BA1FB03214FEA08184FEA51117FF651AF0020DFF85CE08446AEFB013216
:2036C000D20802EB8203A1EB43035FFA80F98A469BB24FEA890903FA09F3BAF1090F91B213
:2036E0004CEA030C00F10100E8D848EA0C0832E70C4600E788468FE7F46E002050D600202F
:20370000706F002089B5F814D34D6210D8DD00201F85EB51CDCCCCCC08B5A0F10103B3FAE9
:2037200083F302284FEA531301D0184608BD0F2022F08AF930B9064B93F8B83503F00103E9
:20374000184608BDBDE808400F2022F0ADB900BF50D60020014B1B681B6A18479C630020DB
:20376000024B186808B18369184770479C630020024B186808B14369184770479C6300203B
:2037800010B5074C606D40B13DF03AFF94F8513013B180F00100C0B210BD012010BD00BFBF
:2037A000501A002030B40A490A480A78531CDBB20525042B00EBC20400F8325008BF00230A
:2037C0004FF404520B7062604FF0FF3030BC70477C74002080740020037870B4FBB1044649
:2037E000C0F10106A31914F8015FDBB2002DF9D101335B00DCB2032513800C704D700478D8
:203800005CB1022300255A1CD2B2CC548D5410F8014F0233DBB2002CF5D170BC7047022441
:203820002346E8E70B0617D401EB810300EBC30310B400EB81000124002283F8764383F80D
:20384000741383F87523426D5DF8044B136843F4001300201360704701F07F0101EB81038B
:2038600000EBC303012200EB810083F81C1183F81E2183F81D2182691368002B01DA43F04E
:20388000804343F4001313600020704770B501F07F0505EB850400EBC404282101FB0501C0
:2038A0000126C4F830310023C4E94A2284F81C5184F81D61C4F8343101F58E711DB9FDF7C5
:2038C0004FFE002070BDFDF7BFFE002070BD00BF2249F8B5D1F890370F2B04D05A1CC1F8AC
:2038E00090270020F8BD1E4C25780023C1F89037002DF6D11B4E1C4B3268B2F5006F17D037
:203900001B689A4227D017D9C2F50063402B15D9403B02F14005C1F894370123237035606B
:2039200092B2402311490A448121FFF7AFFFD8E71B6835607BB12A469B1AE7E74FF00005B8
:2039400002EB0307C1F894570CBF02210121376092B22170E6E700232370C2E750D60020DE
:20396000C4230020AC230020B0230020C8230020AEE700BFF8B51D4C2378012B03D0022B22
:2039800009D00020F8BD01461948D0F8943753B923700020F8BD00231A468121FFF776FF3A
:2039A00000232370F5E7402B11D9124C2268403B02F14005C0F89437256092B240230E4C7C
:2039C000084622448121FFF761FF0020F8BD094D2A684FF0000603EB0207C0F8946708BFC8
:2039E00002202F6092B208BF2070E8E7C423002050D60020AC230020C823002038B513461F
:203A000002250A46C0E94E3380F811510021FFF73DFF002038BD00BF10B50C7814F0600453
:203A200013D0202C0AD14B78023B092B18D8DFE803F01B21171717171717272E22490122F5
:203A4000FFF7DCFF0024204610BD4B78062B24D00A2BF3D01D4B8A78C3F8A027204610BD3F
:203A6000FAF7FAFE0224EEE719490122FFF7C6FF0024E8E717490122FFF7C0FF0024E2E70A
:203A80004B88124A1B0AC2F89C370024DBE70F4B8A78C3F898270024D5E74B881B0A222B64
:203AA0000CD0212B04D021462246FFF7A7FFCAE7CA880949092A28BF0922F6E7CA88074986
:203AC000362A28BF3622F0E7F0DD002050D60020ECDD0020E8DD00204E06002004060020D1
:203AE00038B501EB810400EBC4040D46002184F87453C4F88C1384F87513C4F88833C4F86C
:203B00008023C3782821012B01FB050108BFEDB201F55D7108BFC4F884231DB9FDF720FD15
:203B2000002038BDFDF790FD002038BD144B9A6870B5044662B1134A1B7B92F8A4572B4311
:203B400016D081212046FFF76DFE022D09D070BD0C4B93F8A45781212046FFF763FE022D76
:203B6000F5D12046064ABDE870401F230121B7E70121FFF757FE20468121BDE8704051E671
:203B80005C74002050D6002070B5094A094D1173094B13600021044629700D238121FFF70A
:203BA00075FE2046054ABDE870401F23012197E7BC740020B0740020555342535C740020E5
:203BC00010B5064B597B0446FAF754FE002800DB10BD20460121BDE81040D5E75C74002075
:203BE0002DE9F041314D2C7834B1012C01D1FFF7E7FF0020BDE8F0812D4FDFF8D080B0F81B
:203C0000B4337A68C8F804201F2BBA68C8F80820064606D1274B3A689A4202D1797B01299F
:203C20001AD9254A25491378052401F8334001EBC3000133DBB2042B08BF00234FF4005177
:203C400013701F4B41600222304683F8A427FFF76DFF0020BDE8F081BB7B013B0F2BE0D8FA
:203C6000FAF708FE002819DB2B78013B022BC0D9144B1988B1B1BB68D8F8082088F80C4043
:203C80008B4228BF0B46D11A0424C8F808100E4A2C7030468121FFF7F9FDAAE73046FFF73F
:203CA00045FFA6E73046FFF76FFFA2E7B07400205C740020555342437C740020807400204B
:203CC00050D60020A474002048970020BC74002008B5084B1B78022B07D0033B012B02D82C
:203CE0000021FFF751FF002008BDFFF769FF002008BD00BFB074002010B501EB8101084AAD
:203D000000EBC1010446B1F88C131046F4F7EEFA034A204640230121FFF7E2FE002010BD40
:203D2000F8DD0020E8E700BF70B50A7812F060050C46064611D0202D16D1CD88D5B113064B
:203D40002AD52A461F496078F4F77CFBE2881D493046FFF753FE00250AE04B780A2B16D0D8
:203D60000B2B0ED0062B03D13046FAF775FD0225284670BD022260781144F4F763FB284687
:203D800070BD8B78D3B9104BC3F8E857F0E70F490122FFF733FEEBE70D4964780A4AC1F888
:203DA000C8400321C0E9E45542F8045B2B4680F811110021FFF794FE0025D9E7FAF74CFD89
:203DC000D6E700BF54D6002050D6002038DE0020F40400200B7803F00303012B03D0022BE1
:203DE00004D0002070478B881BB915E68B88832BFBD099E710B50223044640228121FDF7FE
:203E00002BFB2046022340220121FDF725FB8221204603230822FDF71FFB064B02229A8063
:203E2000F4F760FB044A204640230121FFF758FE002010BDB0010020F8DD002038B50922EC
:203E40000D46044603238321FDF706FB29462046FFF7D0FF002038BD82B000230168019305
:203E60000B6901930E4B03E00A690192013B13D0019A002AF8DA019A094B42F0010201928B
:203E8000019A0A610A69019203E00A690192013B02D0019AD207F8D4002002B0704700BF97
:203EA000400D0300436D064A1A61C278012A06D100F2CC5058614FF0802219681A607047A1
:203EC0001800086010B5002304220446194680F811211A46FFF7DAFC2046FFF7E3FF002077
:203EE00010BD00BF10B5044629B990F81131032B0DD0002010BDD0F8E4359B69002BF8D0AB
:203F000090F81221032AF4D19847002010BDD0F89013D0F87C33994214D9C078D4F88023D7
:203F20000128A1EB030104BFD218C4F880238B4228BF0B46C4F890139BB220460021FFF78E
:203F4000CFFDD6E7D0F8E4351B691BB190F81221032A03D02046FFF7B5FFCAE79847F9E76C
:203F6000F0B5012190F8D17590F8D36590F8CFC590F8CE5590F8D03590F8D22580F811117F
:203F800090F8CC1585B005EB0C2503EB072302EB062201F01F06AFB292B290F8CD558DF84B
:203FA00008109BB2012E0446ADF80A70ADF80C30ADF80E20C0F840218DF8095017D0022E42
:203FC0001FD036B101F08001FFF72CFC002005B0F0BD092D0FD8DFE815F0BF00AC000E0097
:203FE000D5000E00EA0085000E007700540090F81221032A2FD02046FAF72EFC002005B059
:020000040801F1
:20400000F0BD01F060012029DAB234D0012D00F02081032D00F00681002DD7D190F81211E2
:20402000022900F0DF800329E5D11B0600F14B8102EB820200EBC20393F87633002B00F0D6
:204040004D81BF4B0122C3F8FC27BE4920460222FFF7D4FCBAE7DAB2012ACCD8D0F8E43553
:2040600002A99B689847BDF80E30002BAED12046FFF728FFAAE7D0F8E43502A99B68984794
:20408000A4E7F9B2AE4D012985F8EC17B3D890F81231022B00F02781032BACD1002900F066
:2040A000868190F810110129E1D0D0F8E4355B68984795F8EC1784F810112046FDF73AF938
:2040C0002046FFF7FFFE81E7012A94D190F81231022B00F01781032B8DD100F58871FFF79F
:2040E0008DFC73E73D0A022DADF8062000F05081032D00F00B81012D7FF47DAFD0F8EC3579
:2041000080781B680DF106019847BDF80620002A3FF45CAFBDF80E30002B3FF457AF9A42CA
:2041200028BF1A4601462046ADF80620FFF766FC4CE790F81231023B012B3FF65CAF012F91
:204140007FF444AFD0F8E43500229B68C0F8182102A9204698478AE790F81231023B012B6D
:204160003FF649AF764BD0F818210021C3F8F41712B10222C3F8F427734920460222FFF770
:204180003DFC23E7012F00F09880022F7FF41EAF13F0FF0F7FF41AAF02691B0A023B52685F
:2041A000032B00F21D81DFE803F0393531241A437FF421AF90F81231032B3FF41CAF0369C1
:2041C00007F07F0580F81451196867F30A120A431A60FFF777FE002D00F0E580022384F83B
:2041E0001231F3E651063FF4F1AE1146FFF71AFBECE6052363F30612514B012184F816114F
:204200002046C3F8F827FFF75DFEDFE6042363F30612F1E7032363F30612EDE7022363F3F8
:204220000612E9E790F81231022BDBD0032B7FF4E2AE27B9550602D01146FFF7F3FAD4F8AF
:20424000E43502A99B68204698472046FFF73AFEBCE690F812110229C4D003297FF4CBAE9A
:20426000002F7FF4B3AE12F07F013FF400AF180600F1A78002EB820304EBC30304EB81000A
:2042800083F8767383F8741383F87573282303FB0243416D03F55D73DA780B68023A6FF3EE
:2042A0005553012AD4F8E42598BF43F080530B602046936802A99847D9E6D0F8E435C0F84B
:2042C00018719B6844E702F07F0202EB820200EBC20393F81E31002B7FF4B3AE184B002235
:2042E000C3F8FC27B1E600293FF4C1AE0121032380F8101180F81231FDF71CF82046FFF77E
:20430000E1FD63E61149FFF779FB5FE6FDB2052D3FF671AEDFE805F0342C241C0B03D0F806
:20432000EC3580789B690DF106019847EDE6D0F8EC3580785B690DF106019847E5E600BF96
:2043400050D600204CDE002044DE002040DE0020D0F8EC3580781B690DF106019847D4E64A
:20436000D0F8EC358078DB680DF106019847CCE6D0F8EC3580789B680DF106019847C4E611
:20438000D0F8EC3580785B680DF106019847BCE6D0F8E43580789B6A0DF10601984745707C
:2043A000C4F8F005B1E6012384F812310EE60222D0F8E43580F8101180F812215B689847F3
:2043C00055E6282202FB014304EB810083F81E7183F81C1183F81D51816903F58E735BE7E7
:2043E000012363F3061207E770B5044649B990F81131022B1BD094F81631012B0DD00020EE
:2044000070BDD0F8E4355B69002BF8D090F81221032AF4D19847002070BD2A4A2369D2F834
:20442000F8275A60002384F81631002070BDD0F83831D0F82451AB4217D9C278012AD0F8F8
:204440002821A3EB050308BF5219C0F8383108BFC0F828219BB20021FFF718FA00231A4669
:2044600019462046FFF73CFBC5E7D0F83C31B3FBF5F605FB163666B99D420AD8D0F840217B
:20448000934206D233463246FFF700FAC4F84061E4E7D4F8E435DB681BB194F81221032A86
:2044A0000CD00023052284F8112119461A462046FFF716FB2046FFF7F5FC9CE720469847E7
:2044C000EFE700BF50D6002082B000230193019A094B42F010020192C168019A0A610A69B0
:2044E000019203E00A690192013B02D0019AD206F8D4002002B07047400D030082B00023C5
:204500000193019A0B4B42F020020192019A61F38A120192C168019A0A610A69019203E0F9
:204520000A690192013B02D0019A9206F8D4002002B07047400D0300F8B50B7813F06005F7
:204540000C4606461CD0202D17D14A78FE2A44D0FF2A3DD14A88002A56D1CD88002D53D19E
:204560001B0651D43749384B0D70012183F8A417364A1F23FFF7B4FA00E000252846F8BD8F
:204580004B780A2B4BD00B2B44D0012BF6D191F904308988002B47DBFFF796FF21792A4F11
:2045A0003046FCF7F5FE0223217940223046FCF753FF97F8A437022B3BD094F90420002A46
:2045C000DCDA012BDAD030460121FFF7DDFAD5E70225FAF741F92846F8BD4D88A5B9CC8832
:2045E000012C11D11A060FD5194B1B689B6998471549C0B281F8000830B1224601F50061ED
:204600003046FFF7FBF9B9E730460225FAF724F92846F8BD0C4B4A8883F80128AEE70D4914
:204620000122FFF7EBF9A9E701F07F01FFF766FFB4E730468121FFF7F5F8002387F8A4370E
:204640009CE700BFB074002050D600205C740020A074002051DE002038B50446FCF7CEFE25
:204660002046022340228121FCF7F6FE2046022340220121FCF7F0FE0C4B0D491B680D4A4D
:2046800000250D701B6882F8A457284698472046FFF71AFF20460121FFF730FF064A20465B
:2046A0001F230121FFF71CFA284638BDA0740020B074002050D600205C740020012905D07A
:2046C00008B50321FFF71AFF002008BDFFF752B90B88F0B433BB028C4C880E898B88C98882
:2046E00022F001021204120C0284058B028CADB225F0F30592B22B4322F00A0243EA06134B
:2047000022439BB242F0010203830284038B23F00C031B041B0C0383038B9BB21943F0BC47
:2047200001837047042B048C2CD0082B4E888A880D89C98851D024F480542404240C048494
:20474000838B078C2C0344EA022440F6FF421A4045F6FF733B4043EA063322439BB292B2E0
:2047600043F4805382830384828B22F440621204120C8283838B9BB243EA01239BB2F0BC00
:204780008383704724F010042404240C4D880F898A88C9880484068B038C12029BB242EAD7
:2047A000073423F0A00340F6FF42324043EA051322439BB292B243F0100302830384028B05
:2047C00022F440621204120C0283038B9BB243EA01239BB2F0BC0383704724F480742404D2
:2047E000240C0484848B038CA4B29BB224F0F30423F42063224343EA062342EA05129BB2D0
:2048000043F4807392B282830384838B23F00C031B041B0C8383838B9BB21943F0BC8183BB
:20482000704700BF214A038890429BB212D002F5806290420ED0B0F1804F0BD0A2F58032EE
:20484000904207D002F58062904203D002F58062904203D14A8823F070031343144A9042D4
:2048600018D002F58062904214D030B423F440730C894D6802F56C429BB2234390420C880B
:204880000380C56204850DD18B7A0386012330BC8382704703800B884A68C2620385012315
:2048A00083827047034B9842EED0EFE700000140001000400004014082B0064B0022019272
:2048C0000193019B03EB80000190019B186802B0704700BF5028004082B0064B0022019275
:2048E0000193019B03EB80000190019B196002B0704700BF502800400023C0E90033C0E9EC
:204900000233C0E90433C0E90633C0E90833C0E90A33C0E90C338363704700BF0B6870B4FB
:20492000D1E90524CD682B431343D1E9072523431343D1E909422B43D1E90D65234313439E
:2049400004680B4A334322402B4313430360D1E90B3442690D6922F0070223431343D1E9EC
:20496000014243614560846070BCC260704700BF3F801CF002683649002310B422F0010253
:20498000212488420260036043608360C3600361446138D02F4B98422ED02F4B98423CD0D7
:2049A0002E4B984240D02E4B984232D02D4B984241D02D4B984246D02C4B984217D02C4BC5
:2049C00098423CD02B4B984216D02B4B984224D02A4B984228D02A4B98421AD0294B9842A9
:2049E00029D0294B98422ED0284B984208D14FF03D5243F8AC2C03E04FF4746243F8202CE8
:204A00005DF8044B7047224B5DF8044B3D229A607047204A43F8642CF2E74FF474125DF8EE
:204A2000044B43F8382C70474FF074625DF8044B43F8502C7047184A43F87C2CE0E73D223F
:204A400043F8082CDCE7154A43F8942CD8E700BF10600240286002404060024058600240F4
:204A60007060024088600240A0600240B860024010640240286402404064024058640240F6
:204A80007064024088640240A0640240B8640240006002403D000020400F002000003D2063
:204AA00000B583B009238DF80730FCF785FE8DF807009DF80730012BF7D09DF8070003B016
:204AC0005DF804FB024A536A23EA00005062704700380240024A136A23EA0000106270478A
:204AE00000380240484B98422ED0B0F1804F32D0464B984236D0464B98421ED0454B98422B
:204B000037D0454B98423BD0444B98423FD0444B98424BD0434B984240D0434B98424CD021
:204B2000424B984251D0424B984256D0414B98425AD0414B98425ED07047404A136A43F04B
:204B4000040313620420C5E73C4A536A43F0010353620120B6E7394A136A43F00103136270
:204B60000120B7E7354A136A43F0020313620220B0E7324A136A43F0080313620820A9E7B0
:204B80002E4A136A43F0100313621020A2E72B4A136A43F02003136220209BE7274A536AFF
:204BA00043F4803353624FF480308BE7234A536A43F002035362022084E7204A536A43F4EF
:204BC000003353624FF400307CE71C4A536A43F4802353624FF4802074E7184A136A43F015
:204BE00040031362402075E7144A136A43F08003136280206EE7114A136A43F480731362CF
:204C00004FF4807066E700BF000001400004004000080040000C0040001000400014004098
:204C20000004014000400140004401400048014000180040001C0040002000400038024012
:204C4000224A936803F00C03042B10B421D0082B22D01F4B03601D4C1E4AA168C1F3031173
:204C6000114491F86C11CB404360A168C1F38221114491F86C1123FA01F18160A1685DF822
:204C8000044BC1F342310A4492F86C21D340C3607047114B0360DEE7546851685268630234
:204CA000C2F388124CBF0C4B094B01F03F01B3FBF1F303FB02F3054A5268C2F30142013205
:204CC0005200B3FBF2F30360C5E700BF003802400024F400F404002000127A002DE9F0479E
:204CE00000230F6801264FF0030C02E00133102B41D006FA03F232EA0704F7D1D0F800E0B7
:204D00005C000CFA04F52EEA050EC0F800E091F80490D0F800A009FA04FE09F1FF394EEA81
:204D20000A0EB9F1010FA846C0F800E06FEA050515D8D0F808E005EA0E0585604D79D0F8A6
:204D400008E0A54045EA0E058560456825EA020242608A7945689A4092B22A434260C268F6
:204D600022EA0802C260CA79C568A24001332A43102BC260BDD1BDE8F0870B4B93F8B82543
:204D8000D20703D5012283F80228704793F802284AB9D3F81C3633B1044B1A7810445A7823
:204DA000187011445970704750D600201874002010B50E4C40F0080284F8802194F9CE20B3
:204DC000022A06DD420704D583071CBF012384F8D63005210648FCF7FDFD062184F8810111
:204DE000BDE810400248FCF7DDBD00BFF40400207006002010B5FCF785FDA8B31B4C94F9F1
:204E0000CE30012B30DD59B3022B2DD094F8D6309BB971B180230521154884F88631FCF7D1
:204E2000D9FD062184F88701BDE810401048FCF7B9BDBDE810400420BAE7002914BF0020E5
:204E4000042094F8D1301A0748BF40F002005B0701D411B108B940F00100BDE81040A7E7D9
:204E6000022BD3D10420ECE710BD00BFF404002076060020F8B5224C04F5C477030A84F852
:204E80008D0105460621384684F88C31FCF7A2FD94F8D13084F88E01DB072AD4B4F8D220B3
:204EA000AA4226D1174DD4F88831C5F80338C3B285F8093841F26F714FF6FF738A4218BF8E
:204EC0000123134405F60306C3F307220621304685F8072885F80838FCF77CFD072185F85D
:204EE00009083046FCF75EFD052104F28F10FCF759FDBDE8F84004480721FCF753BD00BFC6
:204F0000F404002050D600207C06002008B5FCF7F9FC48B1A1F59C53083BB3F57A7F03D2B5
:204F2000BDE808400846A5E708BD2DE9F0476B4E3368002B3AD06A4D6A4C05F1CE0730683F
:204F40003BF08CFF002833D1674B198809291D4609D95F8864227A43B2FBF1F2452A40F349
:204F6000A1811880588094F84138012B00F0C581022B00F0E08133B95C480521FCF712FD02
:204F8000012384F841385A4B1D685A4B1B78002B00F0DB81584B1B68EB1A782B40F2D581C9
:204FA000D4F83406F9F722FCC4F84458BDE8F08730683BF04BFF94F80A388046052BBED802
:204FC000DFE803F00309171D3745AA28B7D1012384F80A38B3E7552803D1022384F80A3851
:204FE000ADE7414A938801339380002384F80A38A5E7032384F80B0884F80A389FE713288F
:2050000084F80C08C4F8240807DD374AD3880133D380002384F80A3891E718B9052384F803
:205020000A388CE70023C4F82838042384F80A3885E7D4F82838E218013382F80D08D4F876
:205040002428C4F8283893427FF479AFE6E7D4F824382A4803F1020A4FFA8AF1FCF7BAFCA4
:20506000804594F80B9840F01481262020F01CFD204B48B100221A701B4A538801335380B1
:20508000002384F80A385AE71A784A4519D100221A7009F1FF33102B00F2F680DFE813F09E
:2050A00030008E008E00DE008E00F400F400F4003000F400F400F400F400F400F400F40080
:2050C0003000B9F1090F02D0B9F1110F01D1012ADDD0054A538901335381DAE714740020FC
:2050E000F404002050D600204274002083060020CC2B002050740020547400205BDE002097
:20510000BAF1060F5ADDB9F1010F06D0B9F1090F0CBF4FF002094FF0030994F8100894F8B6
:20512000111894F80F2894F90DE894F90FC894F80E3885F8CE9041EA002109B2900785F8D5
:20514000CFE085F8D1C0A5F8D21006D512F00C0F14BF0122002285F8D620B9F1030F13D1F0
:20516000BAF1090F2ADD94F91328082AA8BF082222EAE27285F80421002043B29A4200F1F6
:20518000010059DC94F81238D4F828A0002002469BB25245904657DB7C4B85F8D0001B7874
:2051A000232B0BD109EB8903794A03EB83030CEB83031380A2F802E09180D08075497648A5
:2051C0000A2258F056FB10B1002384F83638714B3A681A607A685A603A891A8194F8363870
:2051E0002BBB95F8D6306D4A002B14BF0223012384F8363895F8D130117884F8381813F068
:2052000001031CBFB1FA81F35B09517884F83918D8B29188927884F83708A4F83A1884F8C4
:205220003C2813B109B1A4F83E1884F840080DF073FE0DF071FE1FE704EB4308234493F8CA
:205240001538A8F8223698E704EB48080132B8F82C8052B2984508BF10469AE7BAF1040F7F
:20526000ACDD94F80D2894F80E3843EA022359041AB204D5C3F30D03A5F8D4309EE7002AA8
:20528000F8DBA5F8D23099E7454A938901339381F2E619F0010F7FF4F3AE414A13890133C9
:2052A0001381EDE63F4BD3F89421B3F89811012A1AD141F25632914203D14FF0FF32C3F886
:2052C0009421D3F89421306802EB820202EB820201EB420189B2A3F8981103681B699847A3
:2052E00000232B806B803EE60132EAD1B1F5965F04BF0122C3F89421E3E72A4D95F9CE60F5
:20530000002E3FF440AE022E11D14FF48040FFF7B1FD84F8416895F9CE30012B7FF733AE51
:2053200095F8D130C3F3400385F8D6302BE6032384F84138EFE71B4BB3F8D430002B3FF4EE
:2053400022AE032384F841381DE694F8402094F841309A4204D0FDF763F9C4F8445825E613
:20536000D4F84438EB1AB3F57A7FBFF41FAE0E4B1B68ED1A952D7FF619AE0C480521FCF771
:2053800011FBBDE8F047FDF74BB900BF404A0020484A00207CDE0020C20500201874002005
:2053A00042740020F40400205474002083060020104BD3F81C0610B5D8B10F4C217841B1F2
:2053C00062780CF0E5FEA38883421ABFA08001210021E2885AB141F288339342B8BF1346E0
:2053E0009A4204D0E380BDE8104043F09FBD0029F9D110BD50D600201874002010B401445B
:205400000446002014F8013B08225840430010F0800F08BF400083F0070314BFD8B2C0B2F3
:20542000013AF3D18C42EDD15DF8044B704700BF30B54FF4806085B035F06CFA40B3154CAB
:2054400090F9040094F84838134A002B18BF08234FF4E1310125CDE90153009100234FF4AD
:20546000806135F0B8FAFF23E067003818BF012084F8F83484F8083584F8183584F82835D8
:2054800084F8383584F8483584F8583584F8683505B030BD50D600208D1C0108374B1B6869
:2054A00013F000635CD02DE9F04F354B1F78B84251D3FF2856D1334B93F8DE30002B47D029
:2054C000DFF8D4A00022CAF84C28CAF85028CAF85428AAF85828002F4CD00AF59F631046ED
:2054E000144611461546164603EB071BB946B3F802C09F8993F8008093F901E061443A4405
:205500004645D3E901C738BF464610337545B8BF75469B4509B212B264443844E7D191FB03
:20552000F9F192FBF9F28AF84C688AF84D58CAF85048CAF85408144BAAF84E181B781149E0
:20554000AAF85828092B4FF0000281F8DE200CD00E48BDE8F08F0E4A02EB0010BDE8F08F6E
:20556000184670470020BDE8F08F0A4B9AF84C28DA80EDE73A463946DDE700BFF46E002045
:2055800078500020F4040020404A00209CDE002048DB0020484A002050D600200268F8B575
:2055A0003A4E3B4CB6F95C38511C01607E2111700168054603EBC30384FB0302481CDC1768
:2055C000002328600B70FF20C4EB6204FFF766FF2034304BA4B200284DD01B78B0F90C1054
:2055E00023BB2D4BA1F57A729A4246D82B48B0FBF1F189B2284642F043FF96F897357BB136
:205600002AF0E6FD0146284642F03AFF2146284642F036FF28460821F8F780FB0120F8BD5A
:20562000B6F84816284642F02BFFEFE71C4B1F78002FD6D01B48002300EB830201339289A6
:20564000BB421144F8DB184B9FED186A93F8223007EE103A07EE901AB8EEC77AF8EE676A5B
:20566000C6EE077A67EEA67AFCEEE77A17EE901AB1FBF7F1B5E71B7813B94EF69C21B9E756
:20568000074B1F78002FF8D00146D3E750D6002067666666556A002017839303008793031E
:2056A00078500020B0DE0020A82C0020000048432DE9F8434A4C427894F8E43802F00F0586
:2056C000C3B9EDB92B46002184F8E818EB1AD9B20E290BD8234493F8981539B102F0F00283
:2056E000802A4AD0902A5FD0A02A0DD000273846BDE8F8830021AB4284F8E818F6D8E5E76D
:2057000084F8E4582B46DEE7412966D081F08003042B62D90846FCF7D3FA031D0246DBB29A
:20572000304884F8E83865F05F0584F8E958FDF711F994F8E878002FD8D0BE1E16F0FF003D
:2057400024D1FF25A946022756B1DFF89C80464418F8011BD4F80C093BF084FB4645F7D18A
:20576000D4F80C0949463BF07DFBD4F80C0929463BF078FB3846BDE8F88365F07F05042786
:20578000022684F8E95884F8E8783046164A4FF6FF71104412F8015B491B904289B2F9D1C8
:2057A0005FFA81F90D0ACFE7412914D081F08003042B10D90846FCF783FA65F06F0506273B
:2057C000042684F8EB0884F8E95884F8EA1884F8E8783046DAE70420EFE7082304229FE711
:2057E00050D600203ADF002038DF00202DE9F04FC31D85B0544C03F4FC7300AFADEB030D2C
:20580000D4F8103904F5126B0DEB00025B4506468A46FA60E9462FD094F8601A94F861CA02
:20582000D4F8145901F00F0040EA4C1001310DF101088DF8000084F8601AC7F8088007F1B6
:205840000800ED1AA2EB0808A845194644DD2A4642F0F4FDD4F81029B968C4F810B92A4483
:20586000A1EB09014846C4F81429C9B2D04700201437BD46BDE8F08F94F860CA94F8610A3A
:20588000B4F91A590CF00F0141EA401141F01001002DC9B2D4F81459B8BF41F080010CF117
:2058A000010C012884F860CA89F80010A5EB0B0822D1B8F1FE0F3ADDFF2394F8182989F8A8
:2058C000013007F1080009F103031FFA88F1786089F80220BB6020E0424642F0AFFDD4F83D
:2058E0001029424448463146C4F81029D04701201437BD46BDE8F08F94F81C39B4F8181987
:2059000089F8013007F1080009F102037860BB6042F0DCFD78681FFA88F142F0D7FDD7E9A0
:205920000282D4F81459D4F81039786889E794F8181989F8018009F1030889F80210C7F82F
:20594000088007F108007CE750D6002001297FD9F0B50378654CC3F34115032D83B084F8D8
:20596000615A03F00F0700F0848013F01003164606D0012D6ED0052912D8002003B0F0BD23
:2059800094F8342B002AF8D094F8352B013202F00F02BA4255D0184684F8343B03B0F0BD3E
:2059A000437884F8303B4388A4F82C3B85884318811DC02D7ED84E4AC4F8242B15444FF0F3
:2059C000000C0120C4F8285BA4F82ECB84F8340BAA1A5B1A934284F8357B66DB454D002AD4
:2059E0005CD1B4F92C3BFA2B53D0414A4249D4F8243BD1F89C01C4F8242B2946151FA2F532
:205A0000A276C4F81459C4F8283B0025A2F5AA7201ABC4F8106984F8345BC4F8185901959F
:205A20002BF0DEFE013058D0019B0BB100209847D4F81039C4F814390120C4F8106903B098
:205A4000F0BD4318D4F8285BD4F8242B411CBFE700207047022990D045788378A4F82C3BB4
:205A6000FF2D1FD1042988D94318B0F80350411D9FE70023214984F8203904F5126204F679
:205A80002113C4F81819C4F81029C4F81439012074E7002EA9D005233370A6E7284642F0CC
:205AA000CDFC9EE74318C11C83E712481A4642F0C5FC62E7124BB4F82C0BC4F81039032197
:205AC00001334FF6F672A4F81809C4F8143984F82019A4F81A29012050E7D4F810390222FA
:205AE000591CC4F810191A709EE700BF50D60020B4E0002074E10020F40400200000F6FF02
:205B000070DF00200B4B93F86A2612B1B3F8A8254AB9B3F9E836084AD81782FB0323C0EB0E
:205B2000A30000B27047D3F8840690FBF2F000B2704700BF50D6002067666666F8B5184C7F
:205B4000C6B205463146D4F8380B3BF08BF994F83C1BD4F8380BC5F307274E40394684F8EC
:205B60003C6B3BF07FF994F83C1BD4F8380BC5F307464F40314684F83C7B3BF073F994F888
:205B80003C1BD4F8380B2D0E4E40294684F83C6B3BF068F994F83C1B4D4084F83C5BF8BD80
:205BA00050D6002070B50C4DC6B231460446D5F8380B3BF057F995F83C1BD5F8380B240A3B
:205BC0004E40214685F83C6B3BF04CF995F83C1B4C4085F83C4B70BD50D6002038B50B4C11
:205BE000002305462421D4F8380B84F83C3B3BF039F9D4F8380B54213BF034F9D4F8380BA8
:205C00002946BDE838403BF02DB900BF50D600202DE9F043DFF894932DED028B99F83D4BDB
:205C200083B00E461546002C00F03982013C89F83D4B9FEDD88AD84FDFF874833378002BAC
:205C400062D099F83D4B002C5ED135B13AF01AFC2B68C01A002880F2028499F83E4B002CA5
:205C600040F0A68399F83F0B062840F2D781CB4A92F8A53192F8A411994200F00082D2F86D
:205C8000A01199F840CB31F8134064440130013302F5D072A4B2C0B2DBB2B4F5E06F89F827
:205CA0003F0B537100F0D18100F2AA80B4F5806F00F0F88264D9B4F5A06F00F0CC823CD92E
:205CC000B4F5A16F25D8601EC0B2FFF7E7FBC8B1B0F90C30B24AADF8014092F82210D9F879
:205CE000842503EB830303EB830349089B0093FBF1F31021CDF803308DF800106846904772
:205D000000233370002D99D103B0BDEC028BBDE8F083B4F5C06FF5D1B9F86C36002B00F019
:205D200054832AF06DFA10220024CDF8030006238DF800208DF801401FE2B4F5826F00F0CE
:205D40005082B4F5846F40F0358199F844369A07D8D5B9F84636CDF80330102120220423D7
:205D60008DF800108DF801208DF80230D9F884356846002498473470002D7FF45FAFC3E7FA
:205D8000B4F5067FBED8B4F5007FC0F02C81A4F50073182BB6D801A252F823F0196101085A
:205DA00007610108076101080761010807610108076101080761010807610108076101085B
:205DC000055D0108055D0108055D0108055D0108055D0108055D0108055D0108E36001088A
:205DE000CD600108CD600108CD600108CD600108CD600108CD600108CD600108CD600108F3
:205E0000B4F5116F00F0E0815BD8B4F5026F00F0BF8121D9B4F5036F00F07282B4F5046F76
:205E20007FF470AFB9F9E836D9F8842503EB83035B001020CDF80330402108238DF800007E
:205E40008DF801108DF802306846002490473470002D7FF4F3AE57E7B4F5E46F00F0788144
:205E6000B4F5006F76D199F8442691077FF54AAF13F0010F4B4B00F005835A6882EAE2731F
:205E8000A3EBE27303EB5303A7FB0313DB08002AACBF43F0004343F0404310210024082200
:205EA000CDF803308DF800108DF80140D9F884358DF80220684698473470002D7FF4BEAE21
:205EC00022E745F230239C4200F0B1811DD945F240239C4200F0298245F250239C427FF42B
:205EE00011AFD9F88436CDF803301021502252238DF802308DF80010D9F884358DF80120CB
:205F0000684600249847347036E7B4F5376F00F031826FF437616318072B3FF6F3AEA4F10A
:205F20007100C0B2FFF7BAFA00283FF4EBAE90F90130CDF8033010238DF80030ADF8014060
:205F4000D9F884356846984700233370002D7FF475AED9E6B4F5E26F7FF4D4AE124B93ED16
:205F6000130AD3ED007A20EE270A002420EE080A56F0A2F910230722CDF803008DF800308D
:205F80008DF801308DF80220D9F8843568469847347092E70000C8421F85EB51F40400206E
:205FA000A82C0020706F0020DCDC002050D60020C5B3A29140F201439C427FF4A3AEB9F95B
:205FC0005C38CDF803301021012204238DF802308DF80010D9F884358DF80120684600246C
:205FE00098473470C8E6B4F5807F00F01481B4F5887F7FF487AEB9F9EA36CDF803300122FE
:020000040801F1
:2060000010238DF800308DF801308DF80220D9F884356846002498473470ADE60130CD4A81
:20602000C0B292F8AD1192F8AC318B4222D04B1CDBB24900D2F8A841C74A645A89F83F0BF6
:20604000B4F5E06F53717FF42FAEC44B93ED120AD3ED007A20EE270A002420EE080A56F086
:206060002BF910220723CDF803008DF800208DF8014082E0002182F8AD110123DAE7B849CC
:2060800099F8403B097882F8A5410133DBB201318B4289F8403B00F087810120C1E700286E
:2060A0003FF4C7AD0378303B012B3FF6C2AD013009F63D320621FFF749FC99F83D3B89F8F8
:2060C0003E0B002B3FF4B5AD3470B2E5A4F11100C0B2FFF7E3F900283FF414AEB0F902309A
:2060E00027E799F89735002B40F0B081B9F84806CDF80300102302228DF800308DF8013020
:206100008DF8022083E7601EC0B2FFF7C7F900283FF4F8AD43680CE7D9F87C369149D9F8FC
:20612000842581FB0301DB17C3EBA10300241021CDF8033002238DF800108DF801408DF8A0
:206140000230684690473470002D7FF477ADDBE5824B93ED140AD3ED007A20EE270A002458
:2061600020EE080A56F0A8F8102320228DF80030CDF8030007238DF801208DF802306846F2
:20618000D9F8843598473470002D7FF457ADBBE599F844369B077FF5B5AD734AD9F88435E4
:2061A0009268CDF80320102220218DF8002008228DF801108DF80220684600249847347029
:2061C000002D7FF43BAD9FE52AF002F810230922CDF803008DF800308DF801308DF8022067
:2061E00015E7D9F8803513F0200440F0F1805F4B1B681B0640F13981102304228DF80340FB
:206200008DF804408DF805408DF806408DF800308DF801304AE6D9F8443BCDF8033010220B
:20622000002401238DF800208DF80140A5E7B9F9E636CDF803301021302252238DF80230AA
:206240008DF80010D9F884358DF80120684600249847347090E5FF20FFF720F900283FF426
:2062600051ADB0F90C304249D9F8842591F8221003EB830303EB83031020490800249B0053
:2062800093FBF1F305218DF80000CDF803308DF801408DF80210684690473470002D7FF4C3
:2062A000CDAC31E599F8483B0133DAB2042A00F0D08042F2107389F8482B03FB02F3D9F89E
:2062C0004C2B002A00F0C080023399F8B825D207B9F8882648BF0433D40748BF0A3390071E
:2062E00048BF1433D10548BF2833540748BF6433500648BF03F57A63102100240422CFE5BE
:2063000099F8443698077FF5FDAC174BD9F88425D9894FF4F36303FB01F3A7FB03135B09D1
:206320001020CDF80330302187E5B9F9E436CDF803301021402252238DF802308DF8001060
:20634000D9F884358DF80120684600249847347012E500BFF40400209C060020DCDC002050
:206360007850002067666666706F0020F46E0020A82C0020FF20FFF791F800283FF4C2ACC0
:2063800090F90130CDF80330102170220B238DF802308DF80010D9F884358DF80120684630
:2063A000002498473470E7E489F8404B012038E65C490620FFF71AFA002389F83E0B3370BB
:2063C00003B0BDEC028BBDE8F083D9F88406AAE4554A99F84416538A643BC3EB4370C3EBBE
:2063E000C00388FB03401844DB17C3EB20230933092BA8BF092323EAE37303EB830311F0FA
:20640000020F03EB830314BF4FF47A7000209B00C90748BF00F5FA60117DD9F884259BB2C1
:2064200003440B44042010218DF80200CDF803308DF800108DF8011068460024904734707A
:20644000002D7FF4FBAB5FE401333EE729F0C0FE4EE6012389F8483B42F210732FE73470B6
:2064600003B0BDEC028BBDE8F08399F89635002B3FF448AC99F8503B032B4ED8DFE803F043
:2064800043392A111A6882EAE273A3EBE27303EB5303A7FB0313DB08002AB8BF43F08043A9
:2064A000FBE4D9F8582B537A907AD17A03F1407303EB0023002203EB014389F8502B10224D
:2064C0000421CDF803308DF800208DF801208DF802104BE4D9F8541B8A7D087C897A1204AA
:2064E00002EB00220A44591C89F8501B02EB0363E5E7D9F8541B4A7DC87B497A120402EBAF
:2065000000220A44EFE7D9F8541B0A7D887B097A120402EB00220A44E5E75A1C89F8502B37
:206520001B06CCE7711D0108706F002030B5A0F17D03012B044683B00D46104608D9214661
:206540003AF090FC15B1288804442C8003B030BD7D2101923AF086FC019884F020013AF046
:2065600081FCEFE730B50F4B85B0D3F8B42500230446C51DADF80E3014F8010B01920DF1D5
:206580000E01FFF7D3FFA542019AF5D10DF10E0016F0F2FB019A9DF80E000021FFF7C6FFC3
:2065A00005B030BD50D600207E28F8B50F4652D0324E96F8B04164B9314D95F8641B51B181
:2065C0001B2885F8644B3DD00D2837D0012386F8B0310020F8BD7D284AD095F8682B1AB101
:2065E00080F0200085F8681B95F8632B062A14D8B5F8664B511C2A440444C9B2A5F8664B8A
:2066000085F8631B82F85C0B002BE2D10729E0D101231C4886F8B031F8BDB5F8663B184499
:20662000C0F3072353FA80F0FF284FF00103A5F8660B86F8B031CCD11248F8BDA5F8664BEF
:206640002046F8BD90470028C0D0012320463B7086F8B031F8BD0A4B084A0024012183F8DF
:20666000634B83F8641B3C7082F8B0412046F8BD0123084685F8683BF8BD00BFF404002022
:2066800050D60020ACE10020044AD2F86C3B43F4DF2343F48063C2F86C3B704750D6002097
:2066A000013070B5094EC4B203E045F001FB013448B9E5B2152D21463046F6D9162D04BFE2
:2066C000034B93F8705B284670BD00BFBCE1002050D6002000B1D7E7044AD2F86C3B23F474
:2066E000DF2323F48063C2F86C3B704750D6002070B5114C84B00546D4F8740B0E4634F07C
:20670000C7F894F8902594F89135003A18BF01220BB142F00802CDE9016200234FF49641A5
:2067200095F9000000911A46082134F054F9C4F8740B04B070BD00BF50D6002010B5064C08
:2067400003E0D4F8740B3AF081FBD4F8740B3AF085FB0028F5D110BD50D6002010B50D4C51
:20676000D4F8783B1B791E3B012B0DD9D4F8740B01213830FFF7BCFF0023C4F87C3B84F803
:20678000803BBDE81040D9E7D4F8740B01213AF055FBF1E750D600200B2814D810B401EBB5
:2067A0004103094C01EB83032344184490F8FC36934205D02144002380F8FC2681F8F036E6
:2067C0005DF8044B7047704750D60020F0B5444C94F8813B012B83B005464FD994F8821BE9
:2067E0004048DFF810C194F8837B4A1CA0FB026000F4FE7606EB90001944121A5CF8216035
:2068000084F8822B2FB1D4F8841B04F6883291420DD06EB9344A0133A2FB031222F0010101
:2068200001EB52029B1A84F8813B03B0F0BD2F4E94F89C3B93B92E4B019348F2A501123B65
:2068400015226F46A4F8A01B009384F8A22B29463846B04758B994F8813BDBE76F463846E7
:2068600015F058F929463846B0470028F3D094F89C1B49B1384615F0C7F8ECE71D4A52F8F0
:206880002360002EC6D0D3E7009E1B4A964214D9013A013E41F2210512F8013F81EA032183
:2068A000082311F4004F85EA41000ABF490081B289B2013BF5D19642EED1384641F006FEDD
:2068C0000E49009D6D1A152DA8BF15252A4601F1180056F095FF94F8813B84F8CD5B99E79A
:2068E00050D60020CDCCCCCCABAAAAAAE12D010805E2002020DB0608F3E10020F0E100206C
:2069000070B50C4E054606F6D231D52242F094F92C686C6006F53D61641A182CA8BF18249A
:206920002960224606F6E83056F06AFF86F8004C70BD00BF50D60020026810B40421541CE4
:206940000460117002680B24511C016014705DF8044BC82141F094BD70B50C4E054606F692
:206960000641D52242F068F92C686C6006F60441641A402CA8BF40242960224606F644407F
:2069800056F03EFF86F8844C70BD00BF50D6002010B5104B0A4682B001467B24101D83F8C4
:2069A000050C83F8064C93F8850C83F8070C03F6444403F609400194C824009083F8044CB0
:2069C000684683F8084C41F039FD6846FFF7C4FF02B010BD50D60020F0B5454C94F8883C21
:2069E000D90785B005463BD594F8893C0F2B5AD9002217463F4E94F8883C84F80C2CA6F1C2
:206A00003702CDE90226C3F3820340F6C822DFF8F8C084F80B3CA6F13E01712302A8A4F802
:206A2000082CBA2284F80A3CC4F804CC42F004F9029A3F3E961B84F8056C15F08DF802A8DE
:206A4000FFF78AFF15F088F894F8883CC4F88C5C23F0030343EA470384F8883C05B0F0BD0C
:206A60009A0728D5D4F88C0C2D1AB5F57A6FF5DB94F8893CD4F8900C0F2B97BF1E4A1F4951
:206A800002EB8303D969036801911B69984701990620FDF721FF94F8883C6FF3410384F89B
:206AA000883C05B0F0BD164B93F834301F1E18BF01273A469EE7134B1B685B05CED4104BE1
:206AC00093F83430002BC9D004F6444104F60542C82302A8CDE9022184F8043CFFF72CFFF8
:206AE00015F03AF802A8FFF737FF15F035F8B5E750D6002094E2002020DB0608A0680600C8
:206B000064670020F46E0020C80032EC044BD3F8AC3530EA030314BF01200020704700BF7D
:206B200050D60020AB4A38B50820002382F8AD31FFF7ECFF002800F08C80D2F8A8314FF49F
:206B4000806102204FF48264198082F8AD0101465C804FF40020FFF7D9FF50B14B1CD2F8C2
:206B6000A801DBB240F2014482F8AD3120F811401946994C94F86936002B6CD194F86A36A4
:206B8000002B40F088804FF40070FFF7BFFF50B14B1CD2F8A801DBB24FF4046582F8AD31BF
:206BA00020F811501946D4F88045A50700F11881600700F1EB80894B1B681B0600F1A380E7
:206BC00000234FF4803082F8AC1182F8AD3182F8A531FFF79BFFD0B3D2F8A03101214FF4AD
:206BE000047082F8A51118804FF40040FFF78EFF50B14B1CD2F8A001DBB24FF4007482F8C2
:206C0000A53120F8114019464FF40030FFF77EFF50B14B1CD2F8A001DBB24FF4A06482F8CF
:206C2000A53120F8114019464FF48020FFF76EFF38B1D2F8A0014FF437644B1C20F811406E
:206C4000D9B2002382F8A41182F8A53138BD0146CAE701467DE70120FFF758FF00288DD07C
:206C60004FF48030FFF752FFD2F8A85128B94FF4047325F811300131C9B20BB2481CC1B2DD
:206C80004FF4116082F8AD1125F8130094F86A36002B3FF478AF0220FFF738FF00283FF47D
:206CA00072AF4FF40040FFF731FF50B94B1CD2F8A801DBB24FF4007582F8AD3120F8115011
:206CC00019460420FFF722FF50B14B1CD2F8A801DBB24FF4C06582F8AD3120F8115019461A
:206CE0004FF48010FFF712FF00283FF44CAF4B1CD2F8A801DBB245F2502582F8AD3120F8E1
:206D0000115019463FE74FF40050FFF7FFFE50B14B1CD2F8A801DBB24FF4036482F8AD319D
:206D200020F8114019464FF48050FFF7EFFE68B1D2F8A8014B1C4FF40064DBB28D1C20F8AD
:206D40001140E9B282F8AD1120F813404FF48040FFF7DCFE50B14B1CD2F8A801DBB24FF426
:206D6000846482F8AD3120F8114019464FF48060FFF7CCFE00283FF423AFD2F8A8014FF445
:206D800002644B1C20F81140D9B219E74FF48060FFF7BCFE50B14B1CD2F8A801DBB24FF4B4
:206DA000807482F8AD3120F8114019464FF40060FFF7ACFE00283FF4FEAE4B1CD2F8A8019B
:206DC000DBB24FF4887482F8AD3120F811401946F1E600BFF404002050D60020F46E002051
:206DE0008020FFF793FE50B14B1CD2F8A801DBB245F2302582F8AD3120F8115019464FF405
:206E00008070FFF783FE50B14B1CD2F8A801DBB245F2402582F8AD3120F8115019461020A7
:206E2000FFF774FE50B14B1CD2F8A801DBB24FF4E06582F8AD3120F8115019462020FFF794
:206E400065FE50B14B1CD2F8A801DBB24FF4E26582F8AD3120F8115019464020FFF756FE03
:206E600000283FF4A5AE4B1CD2F8A801DBB24FF4E46582F8AD3120F81150194698E600BF04
:206E8000F0B5CA4C94F8983CD4F88015C4F8940C0133880785B084F8983C12D411F0340FA8
:206EA00035D1090794F8982C42D412F007055BD0282A00F0DB80D4F888355E20984705B0E5
:206EC000F0BD7020FFF722FE0028E7D004F2D466242504F28C67F6EC017A97ED007A67EE6E
:206EE000877A2846FDEEE77A013517EE901AC1EB411301EB8301C90009B2EDB2FAF774FFFB
:206F0000272DE8D1D4F8801511F0340FC9D04FF40060FFF7FBFD002840F0278194F8982C45
:206F200012F0030100F0FD80D4F880150907BCD54FF40070FFF7EAFD0028B6D012F0030594
:206F4000B3D19B4AB4F9E836D91782FB0323C1EBA30109B21420FAF747FF29461C20FAF758
:206F600043FF94F8982CA0E7FF20FEF797FA002800F001810378FF2B00F09A8090F9011070
:206F80000220FAF731FFFF20FEF788FA002800F091800378FF2B00F08D80B0F90C20854BA8
:206FA000834893F8221002EB820202EB82029300490893FBF1F3D91780FB0320C1EBA00037
:206FC00001B20320FAF710FF94F86936002B79D1D4F880359A0640F198804FF40050FFF748
:206FE00095FD002840F0CB80734D4FF48060FFF78DFD002840F04C816B8A94F8982C297DE9
:20700000B3F5967F02D9100740F1118194F89335002B40F0B280A1F1200307EE903A9FED1D
:20702000677AF8EEE77AF6EE006A67EE877ABEEE007AF5EEC07AF1EE10FA58BFB0EE667AC3
:2070400077EE877AFDEEE77A17EE903A19B20520FAF7CAFE4FF48050FFF758FD002840F050
:20706000BD8094F8982C282A7FF425AF544A554B15685549A3FB0535AD09A1FB05367609AD
:20708000A1FB06314909C1EB0111A6EB81010902C6EB0616002309B21720A5EB860684F875
:2070A000983CFAF7A1FE31B21820FAF79DFE02E7294665E700210320FAF796FE94F869362D
:2070C000002B85D00120FFF721FD002840F0F28094F86A36002B3FF47BAF0220FFF716FD52
:2070E000002840F040810420FFF710FD00283FF46FAFB4F86C36002B00F0428129F080F81A
:2071000001B20420FAF770FE62E71B07A9D52F4B93E8030002AB83E803001846FAF77AFE76
:207120009FE74FF48060FFF7F1FC00283FF4FCAE274BD4F8942CD4F8445B9A4240F2F080D7
:20714000244BE91783FB0523C1EB6313642101FB13510DB219B21020FAF746FE2946212074
:20716000FAF742FE94F8982CDEE6B4F9EA163020FAF73AFED2E6014602E709B267E794F827
:2071800044369F0759D44FF48060FFF7BFFC0A4D00283FF431AF002631460120FAF724FE6B
:2071A00031460920FAF720FE26E700BF50D6002067666666A82C0020706F0020E4380E3F19
:2071C000CC2B0020D34D6210898888887CDB06083F4B4C001F85EB510050C34794F844267A
:2071E00000239207CDE9003347D494F89C3C012B43D0B4F98C355FED086A07EE103AB4F914
:207200008E3507EE903AB8EEC77AF8EEE77A27EE267A67EEA67ABDEEC77AFDEEE77A02A8B2
:207220008DED027ACDED037AFAF7F4FD19E742F20F719942A8BF1946E8E6544D544BE9896A
:207240004FF4F36606FB01F14909A3FB0131C9091120FAF7C9FDE9894E4B06FB01F1A3FB27
:2072600001214909A3FB01235B09642202FB131109B21920FAF7B8FDB7E6D5E90023012193
:207280006846CDE9002384F89C1CFAF7C3FDE8E694F844369E077FF57EAFAB683D4AD917DE
:2072A00082FB0302C1EB6211642606FB113636B209B272E794F8991C00293DD10B46062070
:2072C000A4F89A3CFAF790FDB4F89A3C0133A4F89A3C28F089FF94F8943594F8992C012B24
:2072E00094F897351ED000EB800086B213B10AB1B6FBF2F6274BA3FB062343F34F113A2064
:207300005D09FAF771FD642101FB1561224B89B20531A3FB0131C9083B20FAF765FDD7E6C7
:207320000D4618E71BB112B1B0FBF2F080B201B23920FAF759FDCBE6B4F89A0CB4F848263D
:20734000B0FBF1F301FB1303642000FB02129BB24900B2FBF1F2110241EA0311C2F30322A7
:20736000114309B2ABE7D4F87C360C49DA1781FB0313C2EBA30319B22820FAF735FDB2E6F5
:20738000D4F8843683F3100319B2BAE6706F0020C55A7C0A1F85EB51CDCCCCCC6766666625
:2073A00003685A0607D513F4057F04D007298CBF00200120704703F48253B3F5825F03BF3D
:2073C000C81FB0FA80F040090020704770B5BC4C94F89D3C012B84B000F04D8194F8A90C9B
:2073E000FCF79AF994F8AA3C834205461FD0002800F0D680D4F8783BCBB194F8912593F95F
:207400000400002A18BF08224FF4964100230325CDE9015200911A46082133F0DCFAC4F800
:20742000740B20B1FFF79AF9012384F8AA3C94F8AB3C012B00F0C180D4F8B46C3EB1A14B56
:2074400030465978FFF7ACFF002840F0F28094F8B90CFCF761F994F8B83C8342054621D05B
:20746000002800F0F680EEB1337A002B00F01881954A02EB8303DB6994F8902596F9040014
:207480000093003A18BF012202210023CDE901121A46102133F09FFAC4F8380B10B10123E5
:2074A00084F8B83CD4F8BC6C3EB1864B30465978FFF776FF002840F0AC8094F8C80CFCF71F
:2074C0002BF994F8C03C8342054622D0002800F0C980F6B1337A002B00F0E5807A4A02EB18
:2074E0008303DB6994F8902596F904000093003A18BF012202210023CDE901121A464FF475
:20750000007133F068FAC4F8C40C10B1012384F8C03C94F8C90CFCF7FFF894F8CA3C8342EA
:20752000054631D090B3694BD4F8CC6CD3F880344FF47A721A613EB34FF4805240213046FE
:2075400033F0D4F90546F8B994F8903596F90400002B14BF0921082103224FF4E133CDE9D8
:20756000012100932A462B464FF4805133F033FAC4F8D00C40B10123C4F80C0984F8E458DB
:2075800084F8D45C84F8CA3C04B070BDD4F8D00C33F07EF9C4F8D05C84F8CA5C04B070BD2F
:2075A000D4F8740B33F074F994F8AB3CC4F8745B012B84F8AA5C7FF43FAF94F8AC0CFCF7AC
:2075C000ABF80546002871D0D4F8B435002B7FF433AFD4F8B02C002A3FF42EAF94F89155CB
:2075E00094F8901592F90400002D14BF08220022002908BF42F0010203254FF46141CDE997
:20760000015200911A46202133F0E5F9C4F8B40512E794F8C03C002B7FF47BAFD4F8A43C7A
:20762000002B3FF476AF0122C4F8C43C84F8C02C6FE794F8B83C002B7FF434AFD4F8A43C7D
:20764000002B3FF42FAF0122C4F8383B84F8B82C28E7D4F8380B33F01BF9C4F8385B84F81C
:20766000B85C1FE7D4F8C40C33F012F9C4F8C45C84F8C05C4DE7D4F8A05C124B284659781A
:20768000FFF78EFE20B3D4F84036002B7FF4A6AED4F8A43C002B3FF4A1AEC4F840369DE653
:2076A0004FF49643E8E64FF461431BE7D4F8B40500283FF4C1AE33F0EBF8C4F8B455BBE63C
:2076C00050D600204067002020DB0608F43D002094F8A80CFCF720F80646D8B1D4F84036E1
:2076E000002B7FF47BAE002D3FF478AE94F8902595F90400B2FA82F252094FF4165102251E
:20770000CDE9015200911A46042133F064F9C4F8400663E6D4F8400600283FF45FAE33F0E2
:20772000B7F8C4F8406659E670B5C94C94F89D3C002B00F0BF81082033F0ECF8C4F8780B91
:2077400000283CD0082133F0DBF800260346C149C14884F8A93C0522C4F8DC6C3AF0F4F9B1
:2077600041F208530122BC48A4F8E03C84F8E42C0CF074FC31462B22B84856F0A2F848F6C2
:207780007C607D25E02331462B22A4F8EC0CB44884F8EF3C84F8175D56F093F848F67C21D1
:2077A000A0224EF27B0384F8435D84F8466D84F8EF5DA4F8181D84F81B2DA4F8443D94F8F8
:2077C000AB3C002B00F06081102033F0A3F81021C4F8B40C33F094F8A24B84F8B90C3A21F3
:2077E00040F23B1094F8692618809F254AF21E40197100219D7198601973002A40F00E81D5
:2078000094F86A36002B72D1D4F88035580700F1FE80990700F1F2801A0700F1E880924D23
:207820002868C0F3C010FEF755FF0020FEF738FF03464FF4007084F8703B33F06BF84FF4B4
:207840000071C4F8BC0C33F05BF8D4F8F03D84F8C80C002B14BF0123002384F8F43D40F052
:207860009280D4F8903C002B14BF0123002384F8FD3D43D1D4F8A42F0023C4F8A03F002AC8
:2078800000F0DC80012284F89C3B84F8A82F002376487749C4F88C3B06223AF055F940F6D9
:2078A00009437248A4F8903B0CF0D8FB4FF4805033F030F84FF48051C4F8CC0C33F020F84B
:2078C000D4F8B03F6B4A6C4D84F8C90CC4F8102902F5A070591C0022C4F81409C5F89C3138
:2078E000C4F8B01F84F8CA2CBDE870406EE5D4F86C3B43F00403C4F86C3B85E7D4F8800516
:20790000002310F0020084F8FE3D84F8FF3D40F0EA80024694F869362BB10120FFF7F6F8E5
:20792000002840F0F28094F86A36002B40F0E7800820FFF7EBF820B1A318042183F8001E44
:2079400001322B681B0600F101814C4B10219818053300F8011B8342FBD10521092042F2F5
:20796000090384F8051E84F8290F45494548A4F8343F2025042284F82A5F3AF0E5F841487E
:207980000CF06CFB76E794F869362BB10120FFF7BDF8002840F0BF8094F86A26002A40F047
:2079A000E2802B681B0600F1BA80D4F880154E070CD54FF48060FFF7A9F838B1A318082168
:2079C00083F8F81D013284F8FC2D4AE7080705D54FF40070FFF79AF80028EFD10905F2D52D
:2079E0004FF40060FFF792F80028ECD0E6E7D4F86C3B43F48073C4F86C3B10E7D4F86C2B59
:207A000042F4601242F0C002C4F86C2B04E7D4F86C2B42F40272C4F86C2BFAE6D4F86C3BD9
:207A200094F86A2643F00201C4F86C1B002A3FF4EBAE43F03603C4F86C3BE5E6D4F8AC3F6A
:207A4000002B4BD0012384F8A83F84F89C3B1EE750D6002084DB060828E300203CE30020E4
:207A600068E30020886F0020F46E0020D8E100202CDC060870DF0020F404002050E4002038
:207A8000D8DB06087CE50020202032F043FFC4F8B00C00283FF498AE202132F031FF354BD4
:207AA000C4F8843584F8AC0CFFF73CF8012384F8AB3C89E6042032F02DFFC4F8A00C0028FB
:207AC0003FF439AE042132F01BFF2B4A84F8A80C0123C4F8882584F89D3C2CE684F8A83F2F
:207AE00084F89C3BE2E64FF46070FFF70FF800283FF40FAF012084F8000E02460AE7062038
:207B0000FFF704F800283FF413AFA318022183F8001E01320CE7012284F8F82D41E74FF48A
:207B2000A050FEF7F3FF20B1A318022183F8F81D01324FF40850FEF7E9FF00283FF435AF45
:207B4000A318042183F8F81D01322EE74FF45850FEF7DCFF00283FF4F8AEA318082183F852
:207B6000001E0132F1E60620FEF7D0FF0028D2D1024616E76565010845290108084B5A8864
:207B80001B88801A9B1AC00090FBF3F00628A8BF062020EAE070C0F19600C0B2704700BF81
:207BA000B0DC0020074B084A33F81010127802EAD122520705D0DA6F511CD967134483F8CB
:207BC00080007047ACE60020A806002010B5164B42681B7803F00303032B21D1134B1B8871
:207BE000DBB1134B1349B3F9BE30B1F904100A2491FBF4F15B1A1B0103F5B95314334FF429
:207C0000B471B3FBF1F3C3F1080303F00F0360331370436800225A7010BD05231370F8E7E5
:207C20002D231370F5E700BF94DC002096DC0020ACE6002034DD0020436872221A7043685D
:207C400073225A70436874229A7043680022DA7070470F4B4268B3F904300A2193FBF1F32B
:207C60001B0110B503F5B9530A4C4FF4B4711433B3FBF1F303F00F031919E35813604B68F0
:207C800053600B7A1372436800225A7210BD00BF34DD002030640708044B93F8C53013F05C
:207CA000FD0F14BF9E209D20704700BFACE60020094B93F8C53013F0FD0F06D142F21073D1
:207CC0005843064B90FBF3F07047242358434FF47A7390FBF3F07047ACE6002040D2060092
:207CE000064B07EE900A93F8C530B8EEE70A1BB9DFED037A20EE270A704700BFACE6002009
:207D000048F9514010B5104B93F82C21012A10D1D3F83021811A00290BDD0221B3F8264190
:207D200083F82C110949B1FBF4F142B10A44C3F8302193F82C01013818BF012010BD084459
:207D4000C3F83001F5E700BFACE6002040420F00831E00F17A02EA2123F8021F9342FBD163
:207D60004E2243F64913C280CE2243850281CD2323228380A0F87220A0F87830704700BF69
:207D800008BB1F48B0F8343103F001036BBB30B490F83841ACB11B4A02F1F00502E00133EA
:207DA000A3420ED052F8041B4904F8D590F8241200EB8101D1F8BC1145F823100133A34233
:207DC000F0D130BC70470E48B0F83421032A4FEA52030BD90A68A0F8343102F5C332A03220
:207DE00003F001030A60002BD1D070470B6803F5C333A03348F205020B60A0F8342170471B
:207E0000ACE60020E8E700202DE9F04100283AD12D4A92F8380180B32C4A2D4B92F804E07E
:207E200092F905C092F90680CEF1FF07AEF17F06FFB2F6B203EB800003F1F002002403E044
:207E4000834202F1040218D053F8041B8904F7D5E1B2A1EB0C0181EAE175A5EBE175012DB8
:207E60000DDC71B1414514BF394631468342D17004F1010402F10402E6D1BDE8F0810821B9
:207E8000F4E77146F2E7114B1A79F02A09D802F10F000D4A18710B6803F582431A330B60C3
:207EA000B7E7094A93F9054092F83A017F2584421D71987905DB4042C0B298712044587128
:207EC000E9E7002CFADAF6E7ACE60020A8060020E8E70020F0B5384E78B196F8AC32002B9B
:207EE00046D0364A013BDBB286F8AC321378DC0741D4334B0A681A440A6096F838414CB386
:207F0000304B2E4F03EB840403F1F001002503E09C4201F104011DD053F8042BC2F30320F2
:207F20000628F5D13878C00715D596F8AC0296F83BE100EB050CBCFBFEF00EFB10C0012863
:207F4000CCBF0020012058B99C4205F1010501F10401E1D1F0BDE84300F001000028F3D00D
:207F6000C2F3834206EB8202D2F8BC210A60EBE796F83B31B5E7D6EDAF7A134B134CFDEE05
:207F8000E77A642017EE902AA2F57A7200FB02F283FB0230D317C3EBA01303EB4303C3EBEE
:207FA000031384FB0302DB17C3EB62130533084A92FBF3F39EE700BFACE6002008DC00201B
:207FC000400D0300E8E70020D34D62101F85EB5140420F00F0B4524C002868D194F8F80236
:207FE000002856D04F4BD3ED007AB3EE097AF4EEC77AF1EE10FA4EDCBBEE097AF4EEC77AB6
:020000040801F1
:20800000F1EE10FA4CBF08270027D3ED017AB3EE097AF4EEC77AF1EE10FA3EDD47F0010751
:2080200094F83851ADB3404ADFF808C102EB850502F1F00014E094F9FB62B142ACBF0221E8
:20804000002194F9FC62B3421CDB41F004010F421CBFDCF80C300360954200F1040018D09F
:2080600052F8043BD903F7D594F9FA6203F00F01B142C3F30313DEDC94F9FC62B3424FF04B
:208080000101E2DA94F9FD62B342D8BF41F00801DDE7F0BC70470427B7E7BBEE097AF4EE72
:2080A000C77AF1EE10FA48BF47F00207B8E794F8F93263B31B4B1D4DD3ED007A93ED017ADE
:2080C0000A6894F8F802F0EEE77AB0EEC77AF4EEC77AF1EE10FAB8BFF0EE477AFDEEE77A1C
:2080E00080F0010017EE903A193B03EB4303C3EB031385FB0365DB17C3EBE51305330C4DE3
:20810000B5FBF3F31A440A6084F8F80268E70B6894F8F80203F5433303F5A0730B605FE719
:20812000ACE60020A0DC0020E8E70020353AFC4440420F00B4DC0608F0B40B4F97F83861FE
:2081400086B107F59E72054607F50B77002352F8044B35EA040004BF086847F8230001336B
:20816000B342F4D1F0BC7047ACE6002030B42A4B60B92A48027DCAB993F8253228492033A4
:2081800001EB830130BC4FF4A060D5E793F8FE22F2B1013A214883F8FE220A6802F5C322A9
:2081A00002F520720A60027D002AE5D01D4A12689106E1D51C4A93F8FE12127892071AD52D
:2081C00011BB93F827321649203301EB8301D9E7124893F8FF42057DA54205D8042483F8FE
:2081E000FF2283F8FE42D8E70134012283F8FF4283F8FE22D1E70029BED193F82632084991
:20820000203301EB8301BDE793F823320449203301EB8301B6E700BFACE60020706F0020FA
:20822000E8E70020D0DB002094DC002010B41E4A48B91E4C92F800030B6823440B6098B142
:208240005DF8044B704792F8013303B3012B16D092F800030B68164C80F00100234482F889
:2082600000030B600028EBD192F8233211495DF8044B203301EB83014FF440705CE792F84C
:2082800000030D4C80F0010082F80003D4E70B685DF8044B03F5742303F5107301200B602C
:2082A00082F80003704700BFACE6002040420F0048E80100E8E7002020A107003C4AA0B9C1
:2082C00092F802336BB192F803138A081341DB070AD501F00101032A06D8DFE802F050482D
:2082E000403892F8053353BB704792F80333013303F00F0382F803333BB192F802330868BB
:2083000000F5C330A0300860DCE72A4882F80233437A002B44D12848C07818B143F00403B1
:2083200082F8023325480078C00730D592F804030028E4D043F0080382F80233DFE792F833
:2083400012331F4901EB83014FF40030F4E61C4B03F13002002914BF19461146F4E7194B35
:2083600003F1180200290CBF19461146ECE7144B03F10802002914BF19461146E4E7104B3D
:2083800003F11802002914BF19461146DCE70E4800680028CAD043F0010382F80233C5E748
:2083A00092F80133002BB6D0022382F80233B2E7ACE60020B0DC00200CDC002008DC002077
:2083C000B4DC0608C4DC06089CE1002030B4022340F203154FF4FA74322146F20142C370AF
:2083E00000238580C480018130BC42810380704770B40B4C0B490C4B22680E680D6883F890
:208400002C03002122F0200283F83013C3F81C63C3F828532260C3F8241370BC704700BF94
:20842000D0DB0020CC2B0020ACE6002090F8603043B942690121072082F84430A2F84600D2
:2084400082F84810704700BF034A0123E021C37351701846704700BF94E300204FF0FF3092
:20846000704700BF4FF0FF30704700BF704700BF002070470020704770B4067AAEB1427ABF
:208480000B4800212025002352B1142B05DC072903DCC45C202C18BFC55401339342F4D1A4
:2084A00001318E4200F11500EDD1002070BC704797E3002010B50024C4730121FFF7DCFF46
:2084C000024B01225A70204610BD00BF94E3002070B403980378ABB10C4C02EB4205C5EB07
:2084E000C5052544142901F1010406D8072A294403D8CE789E4218BFCB7010F8013FE1B2AB
:20850000002BEFD1002070BC704700BF94E3002014299DF800000CD8072A0AD8064B02EB10
:208520004202C2EBC2021A441144CB78834218BFC8700020704700BF94E30020027A407A59
:2085400002FB00F0704700BF027A407A02FB00F0704700BF002070474FF0FF30704700BF64
:20856000034B93F82121027293F822314372704758E4002000207047002070470120704740
:2085800000207047027A407A02FB00F0704700BF002070470123C373184670470123C373CB
:2085A000184670474FF0FF30704700BF704700BF002070470120704700207047027A407A90
:2085C00002FB00F0704700BF002070470120704700207047914201D0012A01D90020704732
:2085E0000129FBD808B5074BC1EB0110C2EB021203EB421103EB40104FF4F07255F000F98F
:20860000012008BD3845002001299DBF024B012083F8341300207047ACE6002001298CBF23
:2086200000200120704700BF4FF0FF30704700BF034B1B68186A003818BF0120704700BFA6
:20864000FC48002030B41D299DF808000DD80F2A0BD8074B074D93F834431E23C4EB04143E
:2086600013FB021202EB44125055002030BC7047ACE6002038450020014B1889704700BF7B
:20868000A80600200020704700207047074BB3F88A14B3F88C24034610B4054C1C6001206D
:2086A0005DF8044B19815A81704700BFACE60020ECDC0608064AB2F880340BB9184670471C
:2086C00092F88834037292F88934437201207047ACE6002000207047034B93F8890493F891
:2086E000883400FB03F07047ACE6002000207047034B0449B3F90A304068012242F050BE04
:20870000A8060020B25C0708064B07491A88074B40681B68534342F2107293FBF2F242F0BE
:208720003FBE00BF98DC0020025D0708CCDC0020054A064992F8A53492F8A4244068013384
:20874000013242F02DBE00BFACE60020075D07080B4B4068B3F904300A2293FBF2F31A014D
:2087600002F5B9524FF4B4711432B2FBF1F2C2F1080202F00F020349603242F011BE00BF5B
:2087800034DD00200D5D0708034A044992684068072342F005BE00BFCCDC0020145D0708CD
:2087A00007B5144A406892F8B414B2F8B634012909D1009392F8B8340F497B2242F0F0FDF0
:2087C00003B05DF804FB022906D10C497B2203B05DF804EB42F0E4BD0A22534340F2FF32AF
:2087E000B3FBF2F39BB2092B054928BF09237B22EDE700BFACE600201A5D0708525E0708DD
:20880000245D070813B54468FFF746FA0F4B1B789B07024612D50E4B93F8C3140D4B59B143
:208820009889FFF745FA0C49009203467022204642F0B6FD02B010BDD889F2E7009007493C
:208840002D237022204642F0ABFDF3E794DC0020ACE60020706F00202C5E07082A5D0708AC
:208860002DE9F0413F4F90F800C03C78416890F803E0BCF1170F0CBF4FF098084FF08908C6
:2088800014F0040486B0064605D0374BBCF1170F0CBF5C681C68354D84EAE473A3EBE473E1
:2088A000BEF1010FB3FBF5F201F1010005FB123343D0BEF1020F44D181F800803C214B4360
